:020000040800F2
:10000000C8B40020B1020008474400082D3C000895
:10001000FD4300089F080008615000080000000030
:100020000000000000000000000000004D44000837
:100030002F0A0008000000004B4400084F4400084D
:10004000CB020008CB020008CB020008CB0200085C
:10005000CB020008CB020008CB020008CB0200084C
:10006000CB020008CB020008CB020008A50800085C
:10007000CB020008B5080008CB020008C50800083C
:10008000D5080008E5080008CB020008CB020008EC
:10009000CB020008CB020008CB020008CB0200080C
:1000A000CB0200081D450008CB020008CB02000867
:1000B000CB0200082D450008CB020008CB02000847
:1000C000CB020008CB020008CB020008CB020008DC
:1000D000CB0200080950000835500008CB02000888
:1000E000CB020008CB020008CB020008CB020008BC
:1000F000CB020008CB020008CB020008F50800087C
:10010000CB020008CB020008CB020008CB0200089B
:10011000714800089D480008CB020008CB02000887
:10012000CB020008CB02000805090008CB0200083A
:10013000CB020008CB020008CB020008CB0200086B
:10014000CB020008CB020008CB020008CB0200085B
:10015000CB020008CB02000815090008CB020008FA
:10016000CB020008CB020008CB020008CB0200083B
:10017000CB020008CB020008CB0200080000000000
:10018000CB020008CB02000800F002F800F066F88D
:100190000AA090E8000C82448344AAF10107DA45E2
:1001A00001D100F05BF8AFF2090EBAE80F0013F0CE
:1001B000010F18BFFB1A43F001031847741C01001C
:1001C000941C01000A444FF0000C10F8013B13F09E
:1001D000070408BF10F8014B1D1108BF10F8015BA0
:1001E000641E05D010F8016B641E01F8016BF9D193
:1001F00013F0080F1EBF10F8014BAD1C0C1B09D1EA
:100200006D1E58BF01F801CBFAD505E014F8016B5B
:1002100001F8016B6D1EF9D59142D6D370470000ED
:100220000023002400250026103A28BF78C1FBD8FF
:10023000520728BF30C148BF0B607047642900F0E7
:100240003B81732900F09882002070471FB511F0A0
:10025000CBFC00F082F91FBD10B510BD00F0F4FA20
:100260001146FFF7F3FF07F06BFB00F012FB03B43E
:10027000FFF7F2FF03BC04F055FF00000B49D1F873
:1002800000C04A685CF8043B1068184442F8040B4C
:100290008C4528BFA1F1DC0C8A4228BFA1F1DC0209
:1002A000C1F800C04A6020F0004070475CAE0020FA
:1002B0000948804709480047FEE7FEE7FEE7FEE7FA
:1002C000FEE7FEE7FEE7FEE7FEE7FEE70448054936
:1002D000054A064B704700000945000889010008DF
:1002E000C8AE0020C8B40020C8B00020C8B00020AC
:1002F0007047704753EA020C00F069802DE9F04B1B
:100300004FF00006002B1FBFB3FA83F503FA05F484
:1003100024FA05F65E4012BF1643B2FA82F502FADD
:1003200005F4C5F120051EBF22FA05FC44EA0C04C1
:10033000203556EA044C4FEA144418BF641C4FF0B1
:1003400000084FF00009904271EB030C39D30029EB
:1003500019BFB1FA81F701FA07F6B0FA80F700FA8F
:1003600007F6C7F120071EBF20FA07FC46EA0C0675
:100370002037B6FBF4FCA7EB0507103F07F01F0B77
:10038000CBF120060CFA0BFB2CFA06F644BFB34661
:100390000026202FA4BF5E464FF0000B5BEA060C40
:1003A00008BF4FF0010B19EB0B09ABFB027C48EBCC
:1003B0000608C01B06FB02CC0BFB03CC71EB0C0147
:1003C000C1E70B46024641464846BDE8F08B13B5EF
:1003D0004FF000004FF00001AFF30080BDE81C407B
:1003E000704700000FB4044910B503AA029800F04A
:1003F000C7F910BC5DF814FB480000202DE9F0415E
:100400000E460446002020622046E168884730B34B
:10041000252805D0D4E901219047206A401CF2E745
:10042000E168204600278847050018D0A5F1410063
:10043000192802D820354FF4006732462946204655
:100440002760FFF7FBFE40B1012804D0F61D26F01F
:1004500007060836D8E7361DD6E72846DAE7206AC9
:10046000BDE8F08170B50C460546012A05D0287814
:10047000800600D5EA69002302E0012305E05B1C49
:10048000934202D2E05C0028F9D1A869E618C01AAC
:10049000A861286A184428622846AFF3008004E067
:1004A000D5E9012114F8010B9047B442F8D328464E
:1004B000AFF3008070BD00002DE9F0410646002436
:1004C00010687529314616A510D0AFF300800028BA
:1004D00002DA404213A507E031688A0701D512A568
:1004E00002E0490704D511A5012401E0AFF3008023
:1004F00000210A2206F1240709E0B0FBF2FCB0FB60
:10050000F2F302FB1C00303078541846491C0028D6
:10051000F3D123462A463046BDE8F04100F0C1B889
:10052000000000002D0000002B0000002000000053
:100530000B4910B5A1F17C020A4CC2E937123721F0
:1005400006E000EB104342F82130074B00FB03406C
:100550000B1EA1F10101F4DC10BD0120E8E7000051
:10056000FCAD0020E119D666CD0D010040EA010383
:1005700010B59B070FD1042A0DD310C808C9121F4C
:100580009C42F8D020BA19BA884201D9012010BD86
:100590004FF0FF3010BD1AB1D30703D0521C07E053
:1005A000002010BD10F8013B11F8014B1B1B07D1B7
:1005B00010F8013B11F8014B1B1B01D1921EF1D128
:1005C000184610BD032A40F2308010F0030C00F0F2
:1005D000158011F8013BBCF1020F624498BF11F87D
:1005E00001CB00F8013B38BF11F8013BA2F1040236
:1005F00098BF00F801CB38BF00F8013B11F00303AE
:1006000000F0D080083AC0F0088051F8043B083A66
:1006100051F804CBA0E80810F5E7121D5CBF51F8B3
:10062000043B40F8043BAFF30080D20724BF11F82D
:10063000013B11F801CB48BF11F8012B24BF00F892
:10064000013B00F801CB48BF00F8012B70474FF089
:10065000000200B5134694469646203922BFA0E812
:100660000C50A0E80C50B1F12001BFF4F7AF09071E
:1006700028BFA0E80C5048BF0CC05DF804EB89000F
:1006800028BF40F8042B08BF704748BF20F8022B52
:1006900011F0804F18BF00F8012B7047704770476A
:1006A00070472DE9F0470D4699469246044600F101
:1006B00024080168880604D5E06921F01001216052
:1006C00000E00120A84201DD471B00E00027A169EE
:1006D0007A1902EB0900081AA0612078C00602D43A
:1006E0002046AFF30080002608E0D4E901211AF883
:1006F00006009047206A401C761C20624E45F4DBC1
:100700002078C0060AD52046AFF3008006E0D4E981
:10071000012130209047206A401C2062381EA7F13A
:100720000107F4DC07E0D4E9012118F8050090473F
:10073000206A401C2062281EA5F10105F3DC20463A
:10074000AFF300802078000602D50220BDE8F087D4
:100750000120FBE710B5436913B1AFF3008001E05E
:10076000FFF780FE012010BD127800F124010A700D
:1007700000224A700122EDE711684FF0FF32E9E7ED
:10078000074B70B50D467B4400F047F804462846F9
:1007900000F056F810B14FF0FF3070BD204670BD2C
:1007A0000B5B000010B5203AC0F00B80B1E8185088
:1007B000203AA0E81850B1E81850A0E81850BFF44B
:1007C000F5AF5FEA027C24BFB1E81850A0E81850EA
:1007D00044BF18C918C0BDE810405FEA827C24BF3E
:1007E00051F8043B40F8043B08BF7047D20728BFCC
:1007F00031F8023B48BF11F8012B28BF20F8023B1B
:1008000048BF00F8012B70470048704764AE0020D5
:1008100001694A1C02610878704700B58FB0CDE9C4
:1008200001310021059105497944CDE903101146B4
:100830006846FFF7E3FD0FB000BD0000E5FFFFFFD6
:10084000007B00F0800070477546FFF7DDFFAE4685
:1008500005006946534620F00700854618B020B5CC
:10086000FFF734FDBDE820404FF000064FF00007D1
:100870004FF000084FF0000B21F00701AC46ACE848
:10088000C009ACE8C009ACE8C009ACE8C0098D46B5
:1008900070470446AFF300802046FFF7E8FC00BF36
:1008A000FEE7000010B5024800F0C0FC10BD0000DB
:1008B0007804002010B5024800F0B8FC10BD00001C
:1008C000B803002010B5024800F0B0FC10BD0000D5
:1008D0005803002010B5024800F0A8FC10BD00002D
:1008E0009805002010B5024800F0A0FC10BD0000E3
:1008F000F805002010B5024800F098FC10BD00007B
:100900001804002010B5024800F090FC10BD000053
:100910003805002010B5024800F088FC10BD00002A
:10092000D80400200146087810381823B0FBF3F2F1
:100930000848805CC865032A05D908686FF3090078
:10094000001D886503E008686FF309008865886DFD
:1009500070470000F21B0108014600208A6A8B697B
:10096000CBB932B1012A0DD0022A03D0032A10D10B
:100970000EE000BFCB6A03F08073B3F1807F00D13B
:10098000012007E0CB6AB3F1C07F00D1012001E074
:1009900000E000BF34E08B69B3F5005F1AD132B1DB
:1009A000012A07D0022A03D0032A11D10AE000BF8E
:1009B00001200EE0CB6A03F08073B3F1807F00D199
:1009C000012006E0CB6AB3F1C07F00D1012000E036
:1009D00000BF15E032B1012A05D0022A04D0032A53
:1009E0000CD103E000BF00BF012008E0CB6A03F098
:1009F0008073B3F1807F00D1012000E000BF00BF11
:100A0000704730B50468246824F4802405682C609D
:100A1000046863608468402C04D10468A2600468A0
:100A2000E16003E00468A1600468E26030BD7047E3
:100A300010B50146002227E002EB82040B6903EBAC
:100A4000C4000023036043608360C36003624362A9
:100A50004FF0004303604B6943F4804343604368B5
:100A600023F00043436001F1480343F82200032AC6
:100A700007D202EB82040B6903EBC4032833C36083
:100A800001E00B69C360521C042AD5D30024CC6555
:100A90000C668C66CC668C650B6803F580530C691C
:100AA000DC6010BD10B50146002222E002EB82049A
:100AB000CB6803EBC4000023036043608360C36022
:100AC00001F1180343F82200036843F48013036024
:100AD000032A07D202EB8204CB6803EBC40328335A
:100AE000C36001E0CB68C360036843F44003036064
:100AF000521C042ADAD300248C620B6803F580535D
:100B0000CC681C6110BD38B50446002000902068F8
:100B100000F58050806940F48011206800F5805015
:100B20008161206800F5805080690090012000F00C
:100B30005DFD0099206800F58050816138BD00009E
:100B400030B503461479557944EA0520084C0C4425
:100B50002064D4782406957844EA0544557844EA1C
:100B60000524157844EA0500014C0C44606430BD4E
:100B70000080024010B5A4B0044601208DF83C006E
:100B80008DF83D0000200D908DF84B0001208DF870
:100B90004A0000208DF8480001208DF83A008DF8B9
:100BA000300000208DF84C008DF83B0014908DF83B
:100BB00054001D908DF878001F908DF882008DF8FC
:100BC00080004FF480401090C010119000208DF8EC
:100BD00081000BA9204600F089F901208DF80C0056
:100BE0008DF80D008DF81D008DF80E000020059089
:100BF0008DF81C008DF81E00089001208DF824004F
:100C00008DF80400000402908001069040120490C8
:100C100001208DF8250000200A90009069462046AA
:100C200000F004F924B010BD0020704701F0CCB9E9
:100C300010B5024800F05CFF002010BD8C5F002062
:100C400010B513460A460146044800F0C6FE10B12E
:100C50004FF0FF3010BD002010BD00008C5F002061
:100C600010B513460A460146044801F066F810B173
:100C70004FF0FF3010BD002010BD00008C5F002041
:100C80002DE9F04F81460C46174609F11802136909
:100C9000D2F810C04FF0000A52F82310A568D346CE
:100CA000086800F00040B0F1004F04D002F11400D9
:100CB00050F8230010B10220BDE8F08F0AF1010ABC
:100CC0002868886048686FF30C00D5F804E040EAB3
:100CD0000E004860207800F0010038B1086820F468
:100CE0004000D4F814E040EA0E000860207800F0DC
:100CF000200038B1086820F04060D4F810E040EAE5
:100D00000E000860207800F0040018B1086840F078
:100D100080000860086840F08050086053E0086870
:100D200020F00050086027B1086840F0804008605B
:100D300003E0086820F08040086000BF5B1C042BC3
:100D400000D31B1F00BF52F82310086800F00040BA
:100D5000B0F1004F04D002F1140050F82300C8B1E4
:100D6000634652F823104FF000080FE0BFF35F8F87
:100D7000086820F00040086000BF5B1C042B00D313
:100D80001B1F00BF52F8231008F10108D045EDD316
:100D9000022091E7086820F0805008600AF1010AFB
:100DA000AD682868886048686FF30C00D5F804E0E7
:100DB00040EA0E0048600BF1010BBFF35F8F08683B
:100DC00040F000400860A8680028A8D127B1086852
:100DD00040F08040086003E0086820F08040086030
:100DE000086840F00050086052F82C10BFF35F8F85
:100DF000086840F00040086002F1140E506A4EF896
:100E00002300136100BFEFF31080064600BF0120EE
:100E100080F3108800BF0BF1010E906A704490625D
:100E200000BF86F3108800BF002045E770B5054677
:100E30000C46286800F5805086692B480640207BC8
:100E400008B9012000E000208006617B40EA416093
:100E5000617F09B9012100E0002140EA0150A17B36
:100E600040EA415061690843217F40EAC110A17FF7
:100E700040EA8110216A084394F8241040EA810076
:100E80000643286800F580508661286800F5805088
:100E90008669012000F0AAFB286800F58050866171
:100EA0002179A06840EA4160A169084321690843AB
:100EB00094F8251040EAC110A16A40EA8100216837
:100EC000084340F40001286800F58050016028685C
:100ED00000F580500668012000F088FB286800F5C6
:100EE0008050066070BD0000233FDEF870B50546F7
:100EF0000C46286806683B480640A07B4006217CDB
:100F000009B9012100E0002140EAC150617C09B922
:100F1000012100E0002140EA8150A1680843E17FFF
:100F200040EA014061690843A17F09B9012100E05D
:100F3000002140EA4130217F40EA0130A1690843A5
:100F4000217940EA812094F8201009B9012100E0BC
:100F5000002140EA4120E17B40EAC110616A084378
:100F600094F8281040EA01100643286806602868B3
:100F70000668012000F03AFB286806602868866948
:100F80004FF641700640A06C000494F84C1009B96B
:100F9000012100E0002140EAC110216D084394F8CE
:100FA0005510012900D100E0002140EAC10094F869
:100FB0005610012900D100E0002140EA810094F898
:100FC0005410012900D100E0002140EA410006430D
:100FD0002868866128688669012000F007FB286878
:100FE000866170BD0F8120FD2DE9F8430446002085
:100FF00000904FF00109A56E04F1480050F82560FB
:10100000E76E2CE0306A58B9684600F01BFD009886
:1010100010B94FF0000903E0009830620098B0600A
:10102000B9F1000F1BD0A06D30B9606940F00040ED
:1010300040F48040706003E0606940F4804070607C
:10104000306840F00040306000BF6D1C042D00D3BC
:101050002D1F00BF04F1480050F825607F1E17B116
:10106000B9F1000FCED1E06EB8420FD0E81C00F00D
:101070000308BFF35F8F08EB8801206900EBC10113
:10108000206800F580508160A566E766BDE8F883BA
:1010900072B600BFFEE7000070B5054600F094FF91
:1010A000064C2168401A642807D300F08DFF2060A9
:1010B0002846BDE8704004F0C1BF70BD800000202C
:1010C00001460846024B33F8100002B290B2704756
:1010D0003E0B002001460846024B33F8100002B2D6
:1010E00090B270477E0A002030B5A0F11002D417EC
:1010F00002EB5474E410094D2B5DD41702EB5474C9
:10110000E410A2EBC4050124AC401C4014B1012240
:101110000A7001E000220A7030BD0000680A002059
:1011200030B50246D41702EB5474E410094D2B5D20
:101130000246D41702EB5474E410A2EBC405012458
:10114000AC401C4014B101220A7001E000220A7078
:1011500030BD0000720A002070B50446A56D00F095
:1011600033FF064694F83500022808D080206065D9
:1011700000BF002084F8340000BF012070BD20684B
:10118000006820F01600216808602068406920F09F
:10119000800021684861206C08B9A06C28B12068E3
:1011A000006820F00800216808602068006820F0CE
:1011B00001002168086010E000F006FF801B052890
:1011C0000BD920206065032084F8350000BF002083
:1011D00084F8340000BF0320D0E72068006800F0E6
:1011E00001000028E8D194F85C103F208840A860F6
:1011F000012084F8350000BF002084F8340000BFCF
:1012000000BFBBE7014691F83500022803D08020DB
:10121000486501207047052081F83500086800689E
:1012200020F001000A6810600020F3E7F8B50446DA
:10123000002000908C4800684FF41651B0FBF1F785
:10124000A56D2E6894F85C1008208840304098B155
:101250002068006800F0040070B12068006820F089
:1012600004002168086094F85C1008208840A86099
:10127000606D40F00100606594F85C1001208840CA
:10128000304068B12068406900F0800040B194F8B7
:101290005C1001208840A860606D40F0020060652D
:1012A00094F85C1004208840304068B120680068E1
:1012B00000F0020040B194F85C1004208840A8605F
:1012C000606D40F00400606594F85C101020884068
:1012D000304078B32068006800F0080050B394F8FC
:1012E0005C1010208840A8602068006800F480200E
:1012F00080B12068006800F4002028B9206CC8B1D3
:101300002046216C884715E0A06C98B12046A16C5E
:1013100088470FE02068006800F4807028B92068D2
:10132000006820F0080021680860206C10B1204699
:10133000216C884794F85C102020884030400028B9
:1013400065D02068006800F0100000285FD094F895
:101350005C1020208840A86094F83500052828D12A
:101360002068006820F01600216808602068406945
:1013700020F0800021684861206C08B9A06C28B179
:101380002068006820F008002168086094F85C106C
:101390003F208840A860012084F8350000BF00206D
:1013A00084F8340000BF206D10B12046216D8847BD
:1013B000F8BD2068006800F4802080B120680068D3
:1013C00000F4002028B9606C10B12046616C884799
:1013D0001DE0E06BD8B12046E16B884717E020683C
:1013E000006800F4807068B92068006820F0100080
:1013F00021680860012084F8350000BF002084F8CF
:10140000340000BFE06B10B12046E16B8847606D8F
:1014100038B3606D00F00100F0B1052084F83500AC
:101420002068006820F001002168086000BF009873
:10143000401C0090B84200D905E02068006800F028
:1014400001000028F3D100BF012084F8350000BF5F
:10145000002084F8340000BFE06C10B12046E16C3D
:10146000884700BFA4E70000580000202DE9F041A4
:101470000446002500F0A8FD074614B90120BDE888
:10148000F081606A00B100BF022084F8350000BF1F
:10149000002084F8340000BF2068006820F00100BC
:1014A000216808600AE000F08FFDC01B052805D9FF
:1014B00020206065032084F83500E0E7206800689C
:1014C00000F001000028EED12068056821480540A1
:1014D000D4E901010843E1680843216908436169CF
:1014E0000843A1690843E1690843216A08430543A9
:1014F000606A042803D1D4E90B010843054320683E
:1015000005602068456925F00705606A0543606A43
:1015100004280DD1A06A0543E06A48B12046FFF7D0
:101520001BFA28B140206065012084F83500A6E749
:10153000206845612046FFF7F5F9064694F85C10EF
:101540003F208840B06000206065012084F83500AD
:10155000002094E73F8010F02DE9F04704460D4647
:1015600016461F464FF00008D4F8589000BF94F874
:101570003400012802D10220BDE8F087012084F860
:10158000340000BF94F83500012825D1022084F8EA
:101590003500002060653B46324629462046FFF76D
:1015A00030FA94F85C103F208840C9F808002068A1
:1015B000006840F0160021680860206C28B120689F
:1015C000006840F00800216808602068006840F06A
:1015D00001002168086006E000BF002084F83400A4
:1015E00000BF4FF002084046C6E7000070B5044651
:1015F00000F0EAFC06462546681C10B10448007855
:10160000054400BF00F0E0FC801BA842FAD370BD87
:1016100054000020024609B9012070471068006894
:10162000C0F3001081F828001068006800F0600026
:10163000486210680068C0F3402080F0010081F823
:10164000200010680068C0F30040C8771068006888
:10165000C0F3403080F00100887710680068C0F364
:10166000003008771068006800F400608861106836
:10167000006800F48040486110680068C0F3805042
:1016800080F00100487410680068C0F3C05080F01A
:101690000100087410680068C0F3C010C8731068B7
:1016A000006800F46020886010680068C0F3802043
:1016B000087110680068C0F3406088731068806922
:1016C000C0F3400081F8540010688069C0F3C01076
:1016D00080F0010081F84C001068806900F0300053
:1016E000086510688069000C886410688069C0F320
:1016F000800081F8560010688069C0F3C00081F84E
:101700005500002089E7000038B504460CB90120D7
:1017100038BDD4F8840028B92020C4F884002046BD
:1017200000F074F800BF002000903548006840F4D5
:101730008040334908600846006800F4804000900B
:1017400000BF00BF2F48006820F400002D4908604A
:1017500008460068A16808432A49086008460068EE
:10176000206800F58050006840F00101206800F515
:101770008050016000F028FC05460DE000F024FCDC
:10178000401BB0F5FA7F07D90420C4F88800E02098
:10179000C4F884000120BBE7206800F58050006891
:1017A00000F001000028E9D12046FFF7E3F92046C8
:1017B000FFF778F92046FFF73BF9002120466268E1
:1017C000FFF7BEF92068C06B40F402702168C8635F
:1017D0002068D0F80C010C4908432168C1F80C01BD
:1017E0002068D0F8100140F403102168C1F81001FE
:1017F0000020C4F888001020C4F88400002087E787
:10180000443802400438014060000200F0B587B05F
:101810000024029403940494059406940068A0F1B3
:101820008041B1F5203151D12948016841F0007162
:101830000160016801F000710191016841F080616F
:101840000160016801F080610191016841F000616F
:101850000160016801F000610191016841F004013B
:101860000160016801F004010191016841F001018A
:101870000160016801F001010191016841F002017C
:101880000160006800F002000190322002900227FF
:101890000397032505950B26069602A90D4800F02F
:1018A00081FA86200290039704940595069602A972
:1018B000094800F077FA4FF46050029003970494BF
:1018C0000595069602A9054800F06CFA07B0F0BD30
:1018D000303802400008024000000240000402408C
:1018E0002DE9F05F04460F464FF00008C34647B9A4
:1018F000D4F8880040F00100C4F888000120BDE859
:10190000F09FD4F88400402801D00120F7E7E66D6D
:1019100004F1480050F82650E06EC0F1040A3EE0A1
:10192000286800F4807018B1E969A167A969616746
:10193000286800F4007008B9E06F20B3286800F44C
:10194000007010B10021216661662868C0F30D495E
:10195000286800F4807018B1296821674FF0010BE6
:10196000A86828621FFA89F304F18001081F2A6A17
:1019700000F08EF8206E401C2066606E00EB0901BE
:1019800061660020286200BF761C042E00D3361F3B
:1019900000BF04F1480050F8265008F101082868FB
:1019A00000F0004020B9D04502D2BBF1000FB7D003
:1019B000E06E00EB0801E166E06E10B12046FFF733
:1019C00013FBE665BBF1010F05D1E06F3860002124
:1019D000E167002093E7012091E72DE9F0470546F4
:1019E0000E46174698462868046904F01C044FF414
:1019F000784000EAC62004434FF4F86000EA8710FC
:101A0000044324F0020444F001042868046100F057
:101A1000DBFA81460BE000F0D7FAA0EB0900B0F545
:101A2000803F02D30120BDE8F0872868046904F0F4
:101A300001000028EFD12868406980B2C8F8000092
:101A40000020F0E710B582B004460E4806F02EFCE8
:101A5000034683B103F1200020600B481861206821
:101A60004FF4C0610191009000214122084607F027
:101A7000F7FC02B010BD054901200870002020606D
:101A800002B010BD141C01080D9B0008640000206A
:101A9000203A4FF0000CC2F800C0A2F808C05381F1
:101AA000D0F800C0BCF1000F0ED0D1F800C0CCF8C7
:101AB00000200A600068002805D0018919440181CE
:101AC00000680028F9D170470260F2E770B504465B
:101AD0000D460DB9012070BDD4F88400102805D141
:101AE00029462046FFF702FA0020F4E70120F2E73A
:101AF00070B506463068046924F01C0400F006FC4A
:101B000005460D48854202D244F0080411E00B4816
:101B1000854202D244F00C040BE00948854200D211
:101B200007E00848854202D244F0040401E044F092
:101B300010043068046170BDC00E16020087930364
:101B400000E1F50580D1F00870B50446D4F88400B2
:101B500010283DD12020C4F884000421E1662046ED
:101B6000FFF742FA2068006840F00800216808602A
:101B7000206805680120FFF739FD206805602068AE
:101B8000006840F0040021680860206805680120B2
:101B9000FFF72CFD206805602046FEF7B4FF2068A3
:101BA00000F58050806940F40051206800F58050B5
:101BB0008161206800F58050806940F00201206852
:101BC00000F5805081614020C4F88400002070BD81
:101BD0000120FCE770B50446D4F88400402838D1D1
:101BE0002020C4F88400206800F58050806920F42B
:101BF0000051206800F580508161206800F5805018
:101C0000806920F00201206800F580508161206821
:101C1000006820F004002168086020680568012041
:101C2000FFF7E4FC206805602046FEF76CFF2068A3
:101C3000006820F00800216808602068056801201D
:101C4000FFF7D4FC206805601020C4F88400002051
:101C500070BD0120FCE72DE9F04104468846154699
:101C6000B8F1000F08D1D4F8880040F00100C4F8A2
:101C700088000120BDE8F081D4F8840040285AD1C2
:101C8000002241462046FEF7FBFF38B1D4F8880019
:101C900040F00200C4F888000120EBE7BFF34F8F4B
:101CA00004F11800A16A50F8217000BFA06A401C1E
:101CB000A062A06A042802D3A06A001FA06200BF2D
:101CC00004F11800A16A50F82110206800F5805036
:101CD000416000F079F9064627E0206800F5805061
:101CE000406900F4005068B1D4F8880040F0080062
:101CF000C4F88800206800F580504069C4F88C0062
:101D00000120B7E7681C80B100F05EF9801BA84293
:101D100000D855B9D4F8880040F00400C4F8880011
:101D20004FF0405038600120A4E7386800F00040D0
:101D30000028D2D19EE701209CE72DE9F047054617
:101D40000E46174698462868046904F01C044FF4B0
:101D5000784000EAC62004434FF4F86000EA871098
:101D6000044344F0020444F001041FFA88F0296897
:101D700048612868046100F027F981460BE000F013
:101D800023F9A0EB0900B0F5803F02D30120BDE8A4
:101D9000F0872868046904F001000028EFD100BF33
:101DA000F5E70000F8B502460B46002500240020A8
:101DB0000021D6E0012606FA01F51E6806EA0504B0
:101DC000AC4274D11E7906F00306012E04D01E79B0
:101DD00006F00306022E13D190684F000326BE4082
:101DE000B0434F00DE68BE4030439060506801262B
:101DF0008E40B0431E79C6F300168E4030435060CB
:101E00001E7906F00306032E09D0D0684F00032682
:101E1000BE40B0434F009E68BE403043D0601E7944
:101E200006F00306022E13D1CF0802F1200656F861
:101E300027004E07F70E0F26BE40B0434F07FF0E98
:101E40001E69BE403043CF0802F1200646F8270045
:101E500010684F000326BE40B0431E7906F003060B
:101E60004F00BE40304310605E6806F44036002EDE
:101E700076D000BF002600963C4E366846F4804679
:101E80003A4F3E603E46366806F48046009600BFF4
:101E900000BF374E8F0856F827008E07370F0F26E2
:101EA000BE40B043334EB24202D1002624E057E098
:101EB000314EB24201D101261EE0304EB24201D174
:101EC000022619E02E4EB24201D1032614E02D4E17
:101ED000B24201D104260FE02B4EB24201D10526B9
:101EE0000AE02A4EB24201D1062605E0284EB2424F
:101EF00001D1072600E008268F073F0FBE40304380
:101F00001B4E8F0846F82700224E3068A0435E68BB
:101F100006F4801606B120431E4E3060361D306830
:101F2000A0435E6806F4001606B12043194E361D24
:101F30003060184E361F3068A0435E6806F40036E5
:101F400006B12043134E361F3060361F3068A04361
:101F50005E6806F4803606B120430E4E083E3060BF
:101F6000491C1029FFF426AFF8BD00004438024098
:101F7000083801400000024000040240000802400E
:101F8000000C024000100240001402400018024001
:101F9000001C0240083C0140024613690B400BB193
:101FA000012000E00020704710B5426921EA0203D9
:101FB00002EA010443EA0443836110BD0AB181616E
:101FC00001E00B048361704701480068704700001E
:101FD0004C0000200348006803490978084401497F
:101FE000086070474C0000205400002010B50D48D8
:101FF000006840F400700B4908600846006840F42F
:10200000806008600846006840F480700860032023
:1020100000F0A6F80F2000F007F800F02BF80020E1
:1020200010BD0000003C024070B504460E48007828
:102030004FF47A71B1FBF0F00C490968B1FBF0F58F
:10204000284600F02FFC08B1012070BD102C07D2EB
:1020500000222146501E00F045F80548046001E0CA
:102060000120F2E70020F0E7540000205800002093
:102070005000002008B500BF002000900E48006806
:1020800040F480400C4908600846006800F4804035
:10209000009000BF00BF00BF00200090081F006834
:1020A00040F08050091F08600846006800F080502A
:1020B000009000BF00BF08BD4438024001460846FA
:1020C00000280DDB00BF00BF00F01F0301229A4073
:1020D00043099B0003F1E023C3F8002100BF00BFC8
:1020E00000BF70472DE9F05F80460D461646002779
:1020F00002F0FCFF074639462A46334601F0070046
:10210000C0F1070ABAF1040F02D94FF0040A01E046
:10211000C0F1070AD14600F1040ABAF1070F02D252
:102120004FF0000A01E0A0F1030AD4464FF0010A83
:102130000AFA09FAAAF1010A0AEA020A0AFA0CFAE8
:102140004FF0010B0BFA0CFBABF1010B0BEA030B8D
:102150004AEA0B042146404602F0D0FFBDE8F09F5A
:1021600000BF00F00702064B19684FF6FF03194045
:10217000044B0B4343EA0221014B196000BF704737
:102180000CED00E00000FA0570B504460D460CB9F0
:10219000012070BD5848006800F00700A84209D22D
:1021A00055490D700846006800F00700A84201D0AC
:1021B0000120EEE7207800F0020002281DD12078EF
:1021C00000F00400042805D14C48006840F4E050B9
:1021D0004A490860207800F00800082805D14748DF
:1021E000006840F46040454908604448006820F0B9
:1021F000F000A168084341490860207800F0010020
:10220000A8B36068012807D13C4808380068C0F3CB
:102210004040B8B90120BCE76068022802D060687D
:10222000032807D1354808380068C0F3406048B932
:102230000120AEE7314808380068C0F3400008B913
:102240000120A6E72D48006820F0030061680843DC
:102250002A490860FFF7B8FE064609E0FFF7B4FE1A
:10226000801B41F28831884202D9032091E707E0C0
:102270002248006800F00C006168B0EB810FEDD1DE
:102280001D48006800F00700A84209D91A490D70DE
:102290000846006800F00700A84201D0012078E756
:1022A000207800F00400042807D11448006820F4C6
:1022B000E050E168084311490860207800F0080008
:1022C000082808D10D48006820F46040216940EAE0
:1022D000C1000A49086000F03FF808490968C1F3E5
:1022E0000311074A515CC840064908600648006867
:1022F000FFF79AFE00204CE7003C024008380240FD
:10230000FA1B010858000020500000200148006816
:10231000704700005800002000B5FFF7F7FF0449A0
:102320000968C1F38221034A515CC84000BD000026
:10233000083802400A1C010800B5FFF7E7FF04490E
:102340000968C1F34231034A515CC84000BD000036
:10235000083802400A1C01082DE9F0470024002536
:102360000026A1462548006800F00C0020B1042892
:1023700005D008283AD105E0DFF8849039E0DFF88D
:10238000849036E01D48001F006800F03F041B48A1
:10239000001F006800F4800078B11A481749091F2F
:1023A0000968C1F38811A0FB017001462246002391
:1023B0003846FDF79FFF05460EE011480F49091FFB
:1023C0000968C1F38811A0FB017001462246002371
:1023D0003846FDF78FFF05460848001F0068C0F328
:1023E0000140401C4600B5FBF6F902E0DFF8109012
:1023F00000BF00BF4846BDE8F08700000838024033
:102400000024F40000C0A800F8B504460CB901206F
:10241000F8BD207800F00100002874D0F948006869
:1024200000F00C0004280DD0F648006800F00C0005
:10243000082813D1F348001F006800F48000B0F5AD
:10244000800F0BD1EF4808380068C0F340400028E7
:1024500059D06068002856D10120D9E700BF6068D4
:10246000B0F5803F08D1E7480838006840F4803074
:10247000E449083908601EE06068B0F5A02F0DD16E
:10248000E0480838006840F48020DE4908390860D8
:102490000846006840F4803008600CE0D9480838ED
:1024A000006820F48030D749083908600846006881
:1024B00020F48020086000BF606890B1FFF784FDC1
:1024C000054606E0FFF780FD401B642801D9032084
:1024D0009EE7CC4808380068C0F340400028F1D09F
:1024E00011E0FFF771FD054606E0FFF76DFD401BAB
:1024F000642801D903208BE7C24808380068C0F37C
:1025000040400028F1D1207800F0020002285FD17D
:10251000BC48006800F00C0058B1BA48006800F0F0
:102520000C0008281CD1B748001F006800F4800088
:10253000B0B9B44808380068C0F3400020B1E06882
:10254000012801D0012063E7AE480838006820F078
:10255000F800216940EAC100AA490839086037E05B
:10256000E06800B30120A8490860FFF72DFD05468B
:1025700006E0FFF729FD401B022801D9032047E7A9
:10258000A04808380068C0F340000028F1D09D48FA
:102590000838006820F0F800216940EAC100994934
:1025A0000839086014E0002097490860FFF70CFD27
:1025B000054606E0FFF708FD401B022801D903206D
:1025C00026E7904808380068C0F340000028F1D1A1
:1025D000207800F0080008282CD16069A8B10120FB
:1025E0008A490860FFF7F0FC054606E0FFF7ECFCBF
:1025F000401B022801D903200AE782486C3000689A
:10260000C0F340000028F1D014E000207F490860AA
:10261000FFF7DAFC054606E0FFF7D6FC401B022870
:1026200001D90320F4E677486C300068C0F340001D
:102630000028F1D1207800F00400042870D1002790
:1026400070483830006800F0805090B900BF00201A
:1026500000906C483830006840F08050694938314B
:1026600008600846006800F08050009000BF00BF7E
:1026700001276748006800F48070B0B964480068BA
:1026800040F4807062490860FFF79EFC054606E052
:10269000FFF79AFC401B022801D90320B8E65C48EA
:1026A000006800F480700028F2D000BFA068012804
:1026B00008D154486830006840F001005149683141
:1026C00008601DE0A06805280DD14E4868300068FC
:1026D00040F004004B49683108600846006840F04B
:1026E000010008600CE047486830006820F00100F5
:1026F0004449683108600846006820F0040008601A
:1027000000BFA068A8B1FFF75FFC054609E0FFF72E
:102710005BFC401B41F28831884202D9032077E6F6
:1027200026E0384868300068C0F340000028EED04A
:1027300013E0FFF749FC054608E0FFF745FC401BA6
:1027400041F28831884201D9032061E62D48683082
:102750000068C0F340000028EFD1012F07D12948BD
:102760003830006820F0805026493831086000BFBA
:10277000A069002845D02348006800F00C00082814
:102780005DD0A069022845D100201F490866FFF7E7
:102790001BFC054606E0FFF717FC401B022801D989
:1027A000032035E6174808380068C0F34060002869
:1027B000F1D1D4E907010843616A40EA811101229D
:1027C000A06AC2EB500041EA00412C20005D41EAC2
:1027D00000600C49091F086001200B490866FFF7DB
:1027E000F3FB054606E0FFF7EFFB401B022801D98B
:1027F00003200DE6034808380068C0F34060002855
:10280000F1D049E00838024000004742800E4742BC
:1028100000700040002021490866FFF7D5FB0546FF
:1028200006E0FFF7D1FB401B022801D90320EFE5AA
:102830001B480068C0F340600028F2D12CE0A0697A
:10284000012800D1E4E51648001D0668A0690128AA
:1028500020D006F48001E06981421BD106F03F01DF
:10286000206A814216D147F6C0703040616AB0EBF1
:10287000811F0FD106F440310122A06AC2EB500043
:10288000B1EB004F06D106F070612C20005DB1EB7A
:10289000006F01D00120BBE50020B9E500004742F0
:1028A0000038024070B504462546681EB0F1807FAE
:1028B00001D301200FE0681E4FF0E02148610F2195
:1028C0004FF0FF3002F01AFC00204FF0E021886149
:1028D00007200861002070BD7047704730B5024680
:1028E0000B4600BF92F83C00012801D1022030BD08
:1028F000012082F83C0000BF022082F83D001068F1
:1029000044681068816824F07004186804431068F3
:102910004460184D1068A8421BD01068B0F1804F79
:1029200017D0154D1068A84213D0144D1068A84256
:102930000FD0134D1068A8420BD0124D1068A8425A
:1029400007D0114D1068A84203D0104D1068A8425E
:1029500005D121F080015868014310688160012091
:1029600082F83D0000BF002082F83C0000BF00BF9D
:10297000BDE70000000001400004004000080040E6
:10298000000C0040000401400040014000180040DD
:1029900010B504460CB9012010BD94F83D0028B9CB
:1029A000002084F83C00204600F026F8022084F83D
:1029B0003D00211D206801F0C1FD012084F8460082
:1029C00000BF84F83E0001213F2001554020015501
:1029D0004120015500BF00BF012084F84200432080
:1029E0000155442001554520015500BF012084F8C0
:1029F0003D000020D0E7000038B504462849206893
:102A0000884218D100BF002000902648006840F09E
:102A10000100244908600846006800F001000090A9
:102A200000BF00BF00220A211920FFF75BFB19201D
:102A3000FFF744FB32E01C49206888421AD100BFEE
:102A4000002000901748001F006840F00200154960
:102A5000091F08600846006800F00200009000BFEF
:102A600000BF00220A211D20FFF73CFB1D20FFF7BD
:102A700025FB13E00D49206888420FD100BF0020DC
:102A800000900848006840F4803006490860084615
:102A9000006800F48030009000BF00BF38BD000027
:102AA0000000014044380240000400400040014062
:102AB000014691F83D00012801D001207047022015
:102AC00081F83D000868C06840F001000B68D860DC
:102AD0001A4B086898421BD00868B0F1804F17D095
:102AE000174B0868984213D0164B086898420FD0CD
:102AF000154B086898420BD0144B0868984207D0D1
:102B0000134B0868984203D0124B086898420CD1C6
:102B10000868806800F00702062A0CD00868006880
:102B200040F001000B68186005E00868006840F09C
:102B300001000B6818600020C0E7000000000140A1
:102B40000004004000080040000C00400004014068
:102B5000004001400018004001460868C06820F0AD
:102B600001000A68D06000BF0868006A41F21112D3
:102B7000104050B90868006A9210104028B90868DF
:102B8000006820F001000A68106000BF012081F891
:102B90003D00002070472DE9F04104460D46002716
:102BA00000BF94F83C00012802D10220BDE8F0816A
:102BB000012084F83C0000BF022084F83D0020681A
:102BC000866826F0770626F47F46206886602868A7
:102BD000502833D00CDC202850D004DC00284BD007
:102BE000102851D149E0302849D040284CD139E053
:102BF00060282DD0702807D0B0F5805F03D0B0F5E5
:102C0000005F41D10DE041E0D5E902136A68206818
:102C100001F015FD2068866846F07706206886601A
:102C200034E0D5E902136A68206801F008FD2068E5
:102C3000806840F480402168886027E0EA6869681D
:102C4000206801F0EDFD5021206801F003FD1DE03A
:102C5000EA686968206801F0F6FD6021206801F0EB
:102C6000F9FC13E0EA686968206801F0D9FD4021A9
:102C7000206801F0EFFC09E000BF00BF00BF296839
:102C8000206801F0E7FC01E0012700BF00BF012040
:102C900084F83D0000BF002084F83C0000BF3846A7
:102CA00084E7704770B504462068C56820680669E7
:102CB00006F00200022819D105F00200022815D101
:102CC000401F21680861012020772068806900F09A
:102CD000030018B12046FFF7E4FF05E0204600F0AE
:102CE000C7F8204600F07BF90020207706F00400AA
:102CF000042819D105F00400042815D1C043216827
:102D00000861022020772068806900F4407018B1C3
:102D10002046FFF7C6FF05E0204600F0A9F8204650
:102D200000F05DF90020207706F00800082819D18E
:102D300005F00800082815D1C04321680861042067
:102D400020772068C06900F0030018B12046FFF723
:102D5000A8FF05E0204600F08BF8204600F03FF980
:102D60000020207706F01000102819D105F010007F
:102D7000102815D1C04321680861082020772068F9
:102D8000C06900F4407018B12046FFF78AFF05E0E3
:102D9000204600F06DF8204600F021F90020207751
:102DA00006F0010048B105F0010030B16FF00100FC
:102DB00021680861204600F099F906F0800080281B
:102DC00009D105F08000802805D1C0432168086141
:102DD0002046FFF781FD06F04000402809D105F0AC
:102DE0004000402805D1C04321680861204600F01A
:102DF000C3F906F02000202809D105F02000202882
:102E000005D1C043216808612046FFF766FD70BD0B
:102E100010B586B00446142101A8FDF718FC11492D
:102E2000206888421CD100BF002000900E48006836
:102E300040F010000C4908600846006800F01000DF
:102E4000009000BF00BF40200190022002900020AF
:102E5000039004900320059001A90448FEF7A2FF07
:102E600006B010BD00400140303802400010024062
:102E700070472DE9F04104460D461646002700BF75
:102E800094F83C00012802D10220BDE8F081012025
:102E900084F83C0000BF36B1042E1BD0082E31D080
:102EA0000C2E5ED145E02946206801F0DDFB20684C
:102EB000806940F00800216888612068806920F0FE
:102EC00004002168886120688069296908432168B5
:102ED000886148E02946206801F0FEFB206880698F
:102EE00040F40060216888612068806920F4806077
:102EF0002168886120688069296940EA0120216889
:102F0000886130E02946206801F024FC2068C0690F
:102F100040F008002168C8612068C06920F0040002
:102F20002168C8612068C069296908432168C861AF
:102F300019E02946206801F049FC2068C06940F486
:102F400000602168C8612068C06920F48060216841
:102F5000C8612068C069296940EA01202168C86108
:102F600001E0012700BF00BF00BF002084F83C0043
:102F700000BF384689E710B504460CB9012010BDE2
:102F800094F83D0028B9002084F83C00204600F069
:102F900025F8022084F83D00211D206801F0CEFABA
:102FA000012084F8460000BF84F83E0001213F2044
:102FB0000155402001554120015500BF00BF0120AF
:102FC00084F8420043200155442001554520015515
:102FD00000BF012084F83D000020D0E77047704713
:102FE00070B504460D4615B994F83E000BE0042D6B
:102FF00002D13F20005D06E0082D02D14020005D97
:1030000001E04120005D012801D0012070BD1DB903
:10301000022084F83E000EE0042D03D102213F205F
:10302000015508E0082D03D102214020015502E09E
:1030300002214120015501222946206801F0EEFAC3
:1030400023492068884203D022492068884201D160
:10305000012000E0002028B12068406C40F40040CE
:10306000216848641A49206888421BD02068B0F162
:10307000804F17D018492068884213D0174920681C
:1030800088420FD01649206888420BD01149206829
:10309000884207D013492068884203D0124920682B
:1030A00088420CD12068806800F00706062E0CD0FC
:1030B0002068006840F001002168086005E0206891
:1030C000006840F001002168086000209EE70000D1
:1030D00000000140000401400004004000080040DE
:1030E000000C0040004001400018004010B50446AC
:1030F0001A4884421CD11A480068401C18490860CC
:1031000018480068401C1749086008460068B0F578
:103110007A7F0DDB01211448FEF746FF0221124899
:10312000FEF742FF01201149086000200D490860A8
:103130000F48844211D16FF001000D490968086100
:103140000B48FFF709FD0B4880880A49C88000201A
:10315000888005F065FA03F0ABF810BD600100202F
:103160002C00002028000020000C02402400002039
:10317000A8010020580600207047F8B504460D4607
:10318000164694F8420020282DD105B10EB9012031
:10319000F8BD0120206300206063324629462046A6
:1031A00001F050FE0746206B012819D100BF002016
:1031B000009020680068009020684068009000BF80
:1031C00000BF00BF00BF21680C3151E8001F41F073
:1031D000100021680C3141E80002002AF3D100E020
:1031E00001273846D4E70220D2E7000070B5044634
:1031F0000D462649206888420ED12548006840685F
:10320000C0F1FF00234908700123084602782249D3
:10321000224800680DF072FA2149206888420ED1D8
:10322000204800684068C0F1FF001F490870012372
:10323000084602781D491E4800680DF05FFA1D49D6
:10324000206888420ED11C4800684068C0F1FF0029
:103250001A4908700123084602781949194800687C
:103260000DF04CFA1849206888420ED117480068C2
:103270004068C0F1FF001649087001230846027833
:103280001449154800680DF039FA70BD004400403B
:1032900098050020310000206C0600203C01002031
:1032A000004C0040B8030020320000206B070020D3
:1032B000400100200050004078040020330000202E
:1032C0006A08002044010020001001403805002059
:1032D00034000020690900204801002070470000E8
:1032E0002DE9F84F0446206805682068C668206804
:1032F00047694FF00009CA4605F00F09B9F1000F00
:103300000AD105F0200038B106F0200020B1204697
:1033100001F003FCBDE8F88FB9F1000F7CD007F095
:10332000010018B906F49070002875D005F001006E
:1033300030B106F4807018B1606C40F00100606438
:1033400005F0040030B107F0010018B1606C40F0E6
:103350000200606405F0020030B107F0010018B10E
:10336000606C40F00400606405F0080048B106F0AD
:10337000200010B907F0010018B1606C40F008009F
:103380006064606C002846D005F0200028B106F08B
:10339000200010B1204601F0C0FB20684069C0F356
:1033A000801A606C00F0080010B9BAF1000F2DD03F
:1033B000204601F059FB2068406900F04000402899
:1033C00020D100BF00BF2168143151E8001F21F057
:1033D00040002168143141E80002002AF3D100BF07
:1033E000E06B50B17F48E16B0865E06BFDF70AFFC9
:1033F00088B1E06B016D88470DE02046FFF76EFF56
:1034000009E009E02046FFF769FF04E02046FFF7E6
:1034100065FF002060647DE7206B012878D105F00E
:103420001000002874D006F010000028FAD000BF69
:10343000002000902068006800902068406800909C
:1034400000BF00BF2068406900F04000402870D1F4
:10345000E06B006840681FFA80F8B8F1000F58D0A0
:10346000A08D404555DDA4F82E80E06BC069B0F515
:10347000807F43D000BF00BF21680C3151E8001F9E
:1034800021F4807021680C3141E80002002AF3D158
:1034900000BF00BF00BF2168143151E8001F21F0B8
:1034A00001002168143141E80002002AF3D100BF75
:1034B00000BF00BF2168143151E8001F21F0400017
:1034C0002168143141E80002002AF3D100BF202016
:1034D00084F842000020206300BF00BF21680C3147
:1034E00051E8001F21F0100021680C3141E8000272
:1034F000002AF3D100BFE06BFDF72EFE02206063CF
:10350000A08DE28D801A81B22046FFF76FFE0EE09B
:1035100052E0A08D40450AD1E06BC069B0F5807FD4
:1035200005D102206063A18D2046FFF75FFEF1E622
:10353000FFE7A08DE18D401A1FFA80F8E08DD0B32F
:10354000B8F1000F37D000BF00BF21680C3151E83F
:10355000001F21F4907021680C3141E80002002A1C
:10356000F3D100BF00BF00BF2168143151E8001F34
:1035700021F001002168143141E80002002AF3D152
:1035800000BF202084F842000020206300BF00BF5D
:1035900021680C3151E8001F21F0100021680C3126
:1035A00041E80002002AF3D100BF022060634146D7
:1035B0002046FFF71BFEADE605F0800030B106F0B7
:1035C000800018B1204601F0A9FCA3E605F04000F8
:1035D00030B106F0400018B1204601F07BFA99E6C0
:1035E00000BF97E6C948000810B504460CB9012091
:1035F00010BDA06900B100E000BF94F8410028B9F7
:10360000002084F84000204600F02AF8242084F8A6
:1036100041002068C06820F400502168C86020463E
:1036200001F0FAFA2068006920F4904021680861EE
:103630002068406920F02A00216848612068C0683D
:1036400040F400502168C86000206064202084F8A5
:10365000410084F842000020606300BFC8E700001A
:1036600010B586B00446142101A8FCF7F0FFFE490E
:103670002068884275D100BF00200090FB48006898
:1036800040F40020F94908600846006800F4002072
:10369000009000BF00BF00BF00200090F34810382A
:1036A000006840F00400F1491039086008460068DD
:1036B00000F00400009000BF00BF4FF44060019094
:1036C000022002900020039003200490082005901F
:1036D00001A9E748FEF766FBE648E74908604FF0B6
:1036E000006048604021E44881600021C1604FF4DF
:1036F00080610161002141618161C16101624162BA
:10370000FDF7B4FE08B1FDF7C3FC00BFDA48A063C3
:10371000846300BFD7483038D84908604005486006
:103720000021D6488160C1604FF4806101610021B1
:1037300041618161C16101624162FDF797FE08B19B
:10374000FDF7A6FC00BFCD48E063846300BF002204
:1037500011463420FEF7C6FC3420FEF7AFFCB2E180
:10376000FFE7C749206888427ED100BF0020009053
:10377000BE48006840F48010BC49086008460068F4
:1037800000F48010009000BF00BF00BF0020009038
:10379000B6481038006840F00400B4491039086099
:1037A0000846006800F00400009000BF00BF00BFA2
:1037B000002000900846006840F0080008600846B5
:1037C000006800F00800009000BF00BF881401905E
:1037D000022002900020039003200490082005900E
:1037E00001A9A348FEF7DEFA04200190022002900E
:1037F00000200390032004900820059001A9A1480F
:10380000FEF7D0FA9B4848309F4908604FF00060AF
:10381000486040219C4881600021C1604FF4806174
:103820000161002141618161C16101624162FDF775
:103830001DFE08B1FDF72CFC00BF9348A063846314
:1038400000BF8C48603891490860C005486000217D
:103850008E488160C1604FF4806101610021416147
:103860008161C161016200E013E04162FDF7FEFD8C
:1038700008B1FDF70DFC00BF8448E063846300BF1E
:10388000002211463520FEF72DFC3520FEF716FCF0
:1038900019E17F492068884277D100BF002000905D
:1038A0007248001D006840F010007049091D086052
:1038B0000846006800F01000009000BF00BF00BF85
:1038C0000020009069481038006840F00200674905
:1038D000103908600846006800F00200009000BF40
:1038E00000BFC0200190022002900020039003201E
:1038F00004900720059001A96648FEF753FA664830
:10390000664908604FF0006048604021634881606C
:103910000021C1604FF4806101610021416181613A
:10392000C16101624162FDF7A1FD08B1FDF7B0FB85
:1039300000BF5A48A063846300BF5748783858498D
:1039400008604FF000604860002155488160C16008
:103950004FF480610161002141618161C1610162B7
:103960004162FDF783FD08B1FDF792FB00BF4C48B3
:10397000E063846300BF002211462520FEF7B2FBFE
:103980002520FEF79BFB9EE0FFE746492068884222
:10399000F9D100BF002000903448006840F40030A6
:1039A000324908600846006800F40030009000BF0B
:1039B00000BF00BF002000902C481038006840F085
:1039C00008002A49103908600846006800F008001D
:1039D000009000BF00BF60200190022002900020F4
:1039E0000390032004900720059001A92548FEF7C5
:1039F000D9F9204818302C4908604FF00060486021
:103A0000002129488160C1604FF48061016100217B
:103A100041618161C16101624162FDF727FD08B129
:103A2000FDF736FB00BF2048E063846300BF114808
:103A300030301E4908604FF00060486040211B484C
:103A400081600021C1604FF480610161002141610A
:103A50008161C16101624162FDF708FD08B1FDF7B6
:103A600017FB00BF114823E0004C004040380240E3
:103A7000000802407060024058030020B803002094
:103A800000500040000C0240180400207804002080
:103A90000010014000040240B8640240D804002035
:103AA000380500200044004098050020F80500205B
:103AB000A063846300BF002211462620FEF712FB9C
:103AC0002620FEF7FBFA06B010BD704770472DE9BF
:103AD000F84F04460E46174699464FF0000A94F8F0
:103AE0004100202850D106B117B90120BDE8F88F58
:103AF00000206064212084F84100FEF765FA8246C8
:103B0000A784E784A068B0F5805F04D1206910B96C
:103B10000025B04602E035464FF000081EE053464F
:103B2000002280212046CDF8009001F027FA20B134
:103B3000202084F841000320D8E745B9B8F80000F8
:103B4000C0F308002168486008F1020803E0287803
:103B5000216848606D1CE08C401EE084E08C0028E9
:103B6000DDD15346002240212046CDF8009001F0DF
:103B700005FA20B1202084F841000320B6E7202078
:103B800084F841000020B1E70220AFE7F7B5044612
:103B9000154694F8410020283ED1019800B10DB996
:103BA0000120FEBD01982062A584E58400206064A8
:103BB000212084F841001948A16BC8631848A16B03
:103BC00008641848A16BC8640020A16B086501AEA9
:103BD00023681A1D31682B46A06BFDF7BDFC30B180
:103BE00010206064202084F841000120D9E76FF0A4
:103BF00040002168086000BF00BF2168143151E80F
:103C0000001F41F080002168143141E80002002AC1
:103C1000F3D100BF0020C4E70220C2E7034A000836
:103C20005B4A0008DB4800087047704700BFFEE7AA
:103C300038B504460020009063696A460121206877
:103C40009847002802DA6FF0040038BD63696A46BD
:103C5000012120689847002802DA6FF0040038BD7F
:103C6000009810F0040F09D063696A4600212068AB
:103C70009847002804DA6FF0040038BD012038BDF1
:103C8000009810F4805F09D063696A461F2120689C
:103C90009847002814DA6FF0040038BD4FF404513F
:103CA000814304D010F4005F03D0032038BD02200C
:103CB00038BD10F4807F01D0042038BD052038BD08
:103CC000009810F4805F09D000F01C00182807D07D
:103CD000082807D0142807D0052038BD062038BD95
:103CE000022038BD032038BD042038BDF8B5054694
:103CF00000200090002400266868002821D1A868D0
:103D000000B18047202028606B696A461221204656
:103D10009847002802DA6FF0040607E0009800F0E8
:103D20001F00A04202D12C60002602E0641C1F2C60
:103D3000EAD928681F2801D96FF002060EB90120C0
:103D400068603046F8BD002811D0CA687AB18A6828
:103D50006AB10A695AB10A6882604A68C260CA6870
:103D600042618A68026109698161002070474FF0F1
:103D7000FF30704708B500BF002000902E48006853
:103D800040F400102C4908600846006800F4001058
:103D9000009000BF00BF00BF0020009008460068F0
:103DA00040F4800008600846006800F4800000903D
:103DB00000BF00BF002211460B20FEF793F90B2035
:103DC000FEF77CF9002211460D20FEF78BF90D203D
:103DD000FEF774F900220A210F20FEF783F90F2065
:103DE000FEF76CF9002211461020FEF77BF9102037
:103DF000FEF764F9002211461120FEF773F9112035
:103E0000FEF75CF900220A212F20FEF76BF92F2024
:103E1000FEF754F9002211463A20FEF763F93A20E2
:103E2000FEF74CF9002211464620FEF75BF94620CA
:103E3000FEF744F908BD00003038024000B587B0F5
:103E4000142102A8FCF703FC00BF002001906C487D
:103E5000006840F010006A4908600846006800F0F9
:103E60001000019000BF00BF00BF00200190084675
:103E7000006840F0800008600846006800F080009C
:103E8000019000BF00BF00BF0020019008460068FD
:103E900040F0040008600846006800F0040001904B
:103EA00000BF00BF00BF002001900846006840F03E
:103EB000010008600846006800F00100019000BFA2
:103EC00000BF00BF002001900846006840F00200DB
:103ED00008600846006800F00200019000BF00BFC3
:103EE00000BF002001900846006840F0080008600C
:103EF0000846006800F00800019000BF00BF0122E2
:103F000041F21E113F48FEF759F8002221213D4899
:103F1000FEF754F8002201213B48FEF74FF800223B
:103F200010213A48FEF74AF8012211463848FEF7B8
:103F300045F8012211463748FEF740F800220221D9
:103F40003448FEF73BF800224FF400713048FEF78A
:103F500035F841F23F1002900120039000200490B8
:103F6000059002A92748FDF71DFF0120029003904C
:103F700000200490059002A92348FDF713FF482074
:103F8000029000200390049002A92048FDF70AFF48
:103F9000102002900120039000200490059002A9B7
:103FA0001A48FDF7FFFE40F2012002900120039025
:103FB00000200490059002A91548FDF7F3FE4FF488
:103FC0008270029000200390049002A91048FDF72F
:103FD000E9FE4FF48060029000200390049002A953
:103FE0000848FDF7DFFE0320029001200390002027
:103FF0000490059002A90748FDF7D4FE07B000BD64
:104000003038024000100240000802400000024028
:1040100000040240000C02402DE9F04184B0514CF4
:10402000C0212170A82262707223A370FF20251D79
:1040300028706870A8700027EF7004F108063170CE
:104040007270B370C820F070CD20E070DFF8188176
:10405000002201214046FDF7B1FF3C20FDF7C6FAE2
:10406000012211464046FDF7A9FF3C20FDF7BEFAAC
:1040700003F059FCE1782078A27841EA0063617886
:1040800000064FEA014C40EA01404CEA022C40EAAB
:10409000022143EA0C034FEA036C01F47F414CEA2E
:1040A000012100F47F0041EA1020A4F10C0140EA54
:1040B00013600860E9782878AA7841EA0063697893
:1040C00000064FEA014C40EA01404CEA022C40EA6B
:1040D000022143EA0C034FEA036C01F47F414CEAEE
:1040E000012100F47F0041EA1020A4F1080140EA18
:1040F00013600860F1783078B27841EA0063717833
:1041000000064FEA014C40EA01404CEA022C40EA2A
:10411000022143EA0C034FEA036C01F47F414CEAAD
:10412000012100F47F0041EA1020211F40EA1360C2
:1041300008600E480E49231F1A1F01910290009734
:10414000111F0C4804F0AAFA0A4804F0DFFD0948E0
:1041500004F026FF04B00849BDE8F041054804F02A
:104160004BBE000090000020000802408D5F000858
:10417000E161000894600020E960000810B505487E
:1041800002F076F806F01EFDBDE810400148FCF78D
:1041900083BF00009460002000B587B0002003902A
:1041A000049005900690019002901548154908600A
:1041B000002048600021134881604FF2FF21C16058
:1041C0000021016141618161FEF7E2FB08B1FCF76A
:1041D0005FFF4FF48050039003A90A48FEF7DBFC11
:1041E00008B1FCF755FF00200190029001A9054895
:1041F000FEF774FB08B1FCF74BFF07B000BD0000F1
:10420000000001406001002000B587B0002003904D
:10421000049005900690019002901448144908609B
:10422000002048600021124881604FF2FF21C160E8
:10423000002101618161FEF7ABFB08B1FCF728FFAB
:104240004FF48050039003A90948FEF7A4FC08B17D
:10425000FCF71EFF00200190029001A90448FEF720
:104260003DFB08B1FCF714FF07B000BD000400409F
:10427000A801002000B58BB000200790089009909D
:104280000A901C216846FCF7E2F91A481A490860AE
:10429000002048600021184881608621C16000210B
:1042A00001618161FEF774FB08B1FCF7F1FE4FF488
:1042B0008050079007A91048FEF76DFC08B1FCF785
:1042C000E7FE0D48FEF757FE08B1FCF7E1FE60205F
:1042D0000090002001900290049004226946064854
:1042E000FEF7C7FD08B1FCF7D3FE0348FEF790FDCB
:1042F0000BB000BD00400140F001002010B50D489A
:104300000D4908604FF4966048604FF480510A48A8
:1043100081600021C1604FF4C06101610C214161E5
:1043200000218161C161FFF75FF908B1FCF7B0FEC0
:1043300010BD0000004C00403802002010B50D48B0
:104340000D4908604FF4966048604FF480510A4868
:1043500081600021C1604FF4C06101610C214161A5
:1043600000218161C161FFF73FF908B1FCF790FEC0
:1043700010BD0000005000408002002010B50D4824
:104380000D4908604FF4966048604FF480510A4828
:1043900081600021C1604FF4C06101610C21416165
:1043A00000218161C161FFF71FF908B1FCF770FEC0
:1043B00010BD000000100140C802002010B50D48DB
:1043C0000D4908604FF4966048604FF480510A48E8
:1043D00081600021C1604FF4C06101610C21416125
:1043E00000218161C161FFF7FFF808B1FCF750FEC1
:1043F00010BD0000004400401003002000BFFEE795
:1044000030B502464FF6FF7012B10446A14200D10A
:1044100030BD11E012F8014B604000230AE000F0CB
:10442000010424B140104AF20104604000E0401051
:104430005C1CE3B2082BF2DB0C00A1F10105A9B270
:10444000E8D100BFE4E700BFFEE77047704710B552
:10445000FDF7C0FD10BD000000B593B0302107A8E6
:10446000FCF7F5F8142102A8FCF7F1F800BF0020D2
:1044700001902348006840F08050214908600846B8
:10448000006800F08050019000BF00BF00BF002016
:1044900001901C48006840F480401A4908600846B2
:1044A000006800F48040019000BF00BF0120079029
:1044B0000004089002200D9041050E9106210F91F5
:1044C00087211091022111910421129107A8FDF773
:1044D0009BFF08B1FCF7DCFD0F2002900220039047
:1044E000802004904001059000200690022102A83F
:1044F000FDF74AFE08B1FCF7CBFD13B000BD00008C
:1045000040380240007000400348006840F47000EA
:10451000014908607047000088ED00E010B50248CE
:10452000FEF7C0FB10BD00006001002010B502487E
:10453000FEF7B8FB10BD0000A801002010B502680E
:104540002B4B98420ED0B0F1804F0BD0294B9842A4
:1045500008D0294B984205D0284B984202D0284BCE
:10456000984203D122F070024B681A43204B9842C4
:1045700020D0B0F1804F1DD01E4B98421AD01E4B58
:10458000984217D01D4B984214D01D4B984211D021
:104590001C4B98420ED01C4B98420BD01B4B9842A0
:1045A00008D01B4B984205D01A4B984202D01A4BA8
:1045B000984203D122F44072CB681A4322F0800360
:1045C0004C6943EA04028B68C3620B688362084B40
:1045D000984202D00A4B984201D10B6903630368E9
:1045E00043F00403036001234361026010BD000037
:1045F000000001400004004000080040000C0040A2
:1046000000040140004001400044014000480140D6
:1046100000180040001C00400020004030B501F0B0
:104620001F05012404FA05F3046A9C430462046A2A
:1046300001F01F0502FA05F52C43046230BD30B5C8
:104640000C46816821F47F4142EA03252543294332
:10465000816030BD0A46816821F0700142F0070395
:10466000194381607047000030B5026A056A25F081
:10467000010505624368846924F0700424F0030492
:104680000D682C4322F002028D682A43104DA84287
:1046900000D103E00F4DA84206D100BF22F008026E
:1046A000CD682A4322F00402094DA84202D0094DE8
:1046B000A84207D123F4807323F400734D692B4380
:1046C0008D692B43436084614D684563026230BD50
:1046D000000001400004014030B5026A056A25F07F
:1046E000100505624368846924F4E04424F44074AE
:1046F0000D6844EA052422F020028D6842EA051282
:10470000124DA84200D103E0114DA84207D100BFCD
:1047100022F08002CD6842EA051222F040020B4DE1
:10472000A84202D00A4DA84209D123F4806323F4A1
:1047300000634D6943EA85038D6943EA850343605D
:1047400084614D688563026230BD00000000014055
:104750000004014030B5026A056A25F480750562DF
:104760004368C46924F0700424F003040D682C43EA
:1047700022F400728D6842EA0522124DA84200D14F
:1047800003E0114DA84207D100BF22F40062CD68BA
:1047900042EA052222F480620A4DA84202D00A4D64
:1047A000A84209D123F4805323F400534D6943EA0E
:1047B00005138D6943EA05134360C4614D68C56301
:1047C000026230BD000001400004014030B5036AC0
:1047D000056A25F4805505624468C26922F4E04206
:1047E00022F440720D6842EA052223F400538D68DA
:1047F00043EA0533084DA84202D0084DA84204D12F
:1048000024F480444D6944EA85144460C2614D68D3
:104810000564036230BD0000000001400004014057
:1048200030B50B461446026A056A25F0010505629B
:10483000816921F0F00141EA041122F00A021A43D1
:104840008161026230BD30B50B461446026A056ACA
:1048500025F010050562816921F4704141EA0431B7
:1048600022F0A00242EA03128161026230BD000020
:1048700010B5012210210648FDF7A0FB0548FEF700
:104880002FFDFF2204490348FEF777FC10BD00000E
:1048900000000240380200206B07002010B5012202
:1048A00011020648FDF78AFB0548FEF719FDFF22B5
:1048B00004490348FEF761FC10BD000000100240EF
:1048C000800200206A08002070B50446A56B002015
:1048D000E8852846FEF702FD70BD70B50646002546
:1048E000B46B20684069C0F3C01594F841002128DA
:1048F00005D125B10020E084204600F0FBF82068B7
:104900004069C0F3801594F84200222805D125B1F2
:104910000020E085204600F0A7F8606C40F0100011
:1049200060642046FEF7DAFC70BD70B50546AC6BDE
:104930002868006800F48070002842D1E08500BF3C
:1049400000BF21680C3151E8001F21F480702168FC
:104950000C3141E80002002AF3D100BF00BF00BFC4
:104960002168143151E8001F21F001002168143141
:1049700041E80002002AF3D100BF00BF00BF216858
:10498000143151E8001F21F040002168143141E842
:104990000002002AF3D100BF202084F84200206BDF
:1049A00001280ED100BF00BF21680C3151E8001F63
:1049B00021F0100021680C3141E80002002AF3D1F7
:1049C00000BF00206063206B012804D1A18D204628
:1049D000FEF70CFC02E02046FFF777F870BD70B5DB
:1049E0000546AC6B01206063206B012805D1A08DCA
:1049F00041082046FEF7FAFB02E02046FFF766F882
:104A000070BD70B50546AC6B2868006800F4807016
:104A1000F8B90020E08400BF00BF2168143151E8DC
:104A2000001F21F080002168143141E80002002AB3
:104A3000F3D100BF00BF00BF21680C3151E8001F57
:104A400041F0400021680C3141E80002002AF3D116
:104A500002E02046FFF7E8F870BD70B50446A56B8C
:104A60002846FFF7E2F870BD00BF00BF02680C32B5
:104A700052E8002F22F4907102680C3242E80013D1
:104A8000002BF3D100BF00BF00BF0268143252E810
:104A9000002F22F001010268143242E80013002BBB
:104AA000F3D100BF016B01290ED100BF00BF026826
:104AB0000C3252E8002F22F0100102680C3242E85A
:104AC0000013002BF3D100BF202180F842100021F9
:104AD0000163704710B504462068C06820F04000AC
:104AE0002168C860202084F841002046FFF79CF828
:104AF000002010BD00BF00BF02680C3252E8002F3A
:104B000022F0C00102680C3242E80013002BF3D1FE
:104B100000BF202180F841107047F8B504460025F9
:104B2000002694F84200222873D1A068B0F5805F77
:104B30000BD1206948B9A66A20684068C0F3080014
:104B40003080A06A801CA06214E0A56AA068B0F55D
:104B5000805F03D0A06828B9206918B92068406830
:104B6000287004E02068406800F07F002870A06A88
:104B7000401CA062E08D401E80B2E085002846D136
:104B80002068C06820F020002168C8602068C068E4
:104B900020F480702168C8602068406920F001001E
:104BA00021684861202084F8420000206063206B67
:104BB000012826D10020206300BF00BF21680C31EE
:104BC00051E8001F21F0100021680C3141E800027B
:104BD000002AF3D100BF2068006800F01000102800
:104BE0000AD100BF00200090206800680090206873
:104BF0004068009000BF00BFA18D2046FEF7F6FA86
:104C000002E02046FEF761FF0020F8BD01E0002031
:104C1000FBE70220F9E700002DE9F84F0446206881
:104C2000006920F44050E168084321680861216967
:104C3000A068084361690843E1690843009020685F
:104C4000C06849F20C618843009908432168C86034
:104C50002068406920F44070A169084321684861D8
:104C600076492068884203D075492068884203D17C
:104C7000FDF762FB814602E0FDF74EFB8146E069ED
:104C8000B0F5004F6CD102206168A0FB01500346D3
:104C90001920A9FB007001462A463846FBF72AFB7B
:104CA0006421B0FBF1F04FEA001A02206168A0FB1A
:104CB00001510B461920A9FB00712A463846FBF723
:104CC00019FB834602206168A0FB015003461920AE
:104CD000A9FB00712A463846FBF70CFB6421B0FBA8
:104CE000F1F000EBC00101EB0010ABEB80003221D2
:104CF00001EBC0006421B0FBF1F000F0F8000AEB1A
:104D0000400A02206168A0FB015003461920A9FB5C
:104D1000007001462A463846FBF7ECFA834602202B
:104D20006168A0FB015003461920A9FB00712A46C7
:104D30003846FBF7DFFA6421B0FBF1F000EBC0016D
:104D400001EB0010ABEB8000322101EBC0006421CD
:104D5000B0FBF1F000F007005044216888606AE081
:104D600004206168A0FB015003461920A9FB0070D4
:104D700001462A463846FBF7BDFA824604206168A0
:104D8000A0FB015003461920A9FB007001462A46EA
:104D90003846FBF7AFFA6421B0FBF1F000EBC0013D
:104DA00001EB0010AAEB8000322101EB001064211E
:104DB000B0FBF1F000F0F00A04206168A0FB017084
:104DC00003461920A9FB00513A462846FBF792FA00
:104DD0006421B0FBF1F00AEB001A04206168A0FB2B
:104DE00001510B461920A9FB00712A463846FBF7F2
:104DF00081FA834604206168A0FB01500346192014
:104E0000A9FB007001462A463846FBF773FA642175
:104E1000B0FBF1F000EBC00101EB0010ABEB800048
:104E2000322101EB00106421B0FBF1F000F00F0023
:104E3000504421688860BDE8F88F000000100140F0
:104E40000014014077B581B0044615460298A0626F
:104E5000A58500206064222084F842002C48E16B84
:104E6000C8632C48E16B08642B48E16BC8640020E0
:104E7000E16B086502AE32682368191D2B46E06BB2
:104E8000FCF76AFB38B110206064202084F84200EF
:104E9000012004B070BD00BF0020009020680068B1
:104EA000009020684068009000BF00BF206970B18A
:104EB00000BF00BF21680C3151E8001F41F4807031
:104EC00021680C3141E80002002AF3D100BF00BF85
:104ED00000BF2168143151E8001F41F00100216832
:104EE000143141E80002002AF3D100BF00BF00BF27
:104EF0002168143151E8001F41F04000216814314D
:104F000041E80002002AF3D100BF0020C1E7000001
:104F10002B490008DF490008DB480008014691F8EA
:104F20004100212828D18868B0F5805F0BD108693D
:104F300048B90A6A1088C0F308000B685860086A0C
:104F4000801C086205E00B6A581C086218780B6820
:104F50005860C88C401E80B2C88458B90868C068C0
:104F600020F080000B68D8600868C06840F04000FE
:104F70000B68D860002070470220FCE72DE9F84359
:104F800004460D4617469846089E31E0701C70B3E3
:104F9000FDF71AF8A0EB0800B04200D816B90320BC
:104FA000BDE8F8832068C06800F00400F8B1802DE7
:104FB0001ED0402D1CD020680068C0F3C000B0B1E6
:104FC00000BF0020009020680068009020684068C2
:104FD000009000BF00BF2046FFF746FD0820606438
:104FE00000BF002084F8400000BF0120D8E7FFE7A1
:104FF000206800682840A84201D1012000E000207C
:10500000B842C3D00020CBE710B5012211030648F7
:10501000FCF7D4FF0548FEF763F9FF220449034873
:10502000FEF7ABF810BD000000100240C8020020DF
:105030006909002010B5012211460648FCF7BEFFA1
:105040000548FEF74DF9FF2204490348FEF795F89D
:1050500010BD000000040240100300206C06002078
:1050600000BFFEE70246024B23F812107047000013
:105070003E0B002070B50A46B2F57F4F19D1A0F162
:105080001001CC1701EB5474E410174D2C5D0B4646
:10509000DD1703EB5575ED10A3EBC5060125B540F3
:1050A0002C43E5B2CC1701EB5474E4100E4E355589
:1050B00018E0BAB9A0F11001CC1701EB5474E41058
:1050C000094D2C5D0B46DD1703EB5575ED10A3EB79
:1050D000C5060125B540AC43CD1701EB5575ED1064
:1050E000014E745570BD0000680A00200248006837
:1050F000C0F30220704700000CED00E010B500285E
:1051000004DB0A07130E054A135406E00A07140EBF
:10511000034A00F00F031B1FD45410BD00E400E04D
:1051200018ED00E000BF704770B504460D4600263C
:1051300000BF04E014F8010B0CF082F8761CAE42BC
:10514000F8DB70BD10B5012400BF12E0E0B200F042
:1051500047F8012000F071F8E0B24FF6FF72062127
:1051600000F04DF8E0B240F20E72052100F047F871
:10517000641C052CEADB10BD30B52DED028B81B02F
:105180000546B0EE408A9FED150A28EE000AF3EEC0
:10519000080A80EE201ABCEEC10A10EE104A002068
:1051A000009004208DF80000200A8DF80100E0B284
:1051B0008DF80200284605F0A1FC142005F084FCBF
:1051C00003216846FFF7B0FF142005F07DFC05F0D1
:1051D0007DFC01B0BDEC028B30BD000000008047BB
:1051E00010B504464CF23C320821204600F007F886
:1051F0004CF23C320221204600F001F810BDF8B517
:1052000006460D461446002000908DF800502012EE
:105210008DF80100E0B28DF80200304605F06EFC1A
:10522000142005F051FC03216846FFF77DFF142090
:1052300005F04AFC05F04AFCF8BD01B50098FCF702
:10524000D5F908BD70B505460C4614F0030F06D01D
:1052500006A34FF4B67211A118A0FBF7C3F8A86813
:1052600000682060A868046070BD00002E2E2F4DDD
:105270006964646C6577617265732F5468697264E0
:105280005F50617274792F4C7749502F7372632F7E
:10529000636F72652F6D656D702E63006D656D7047
:1052A0005F667265653A206D656D2070726F70651E
:1052B000726C7920616C69676E6564004173736517
:1052C0007274696F6E2022257322206661696C6595
:1052D00064206174206C696E6520256420696E20ED
:1052E00025730A0010B580680468002C0DD0216871
:1052F000016014F0030F06D005A34FF48C7210A1C7
:1053000018A0FBF76FF8204610BD002010BD00006C
:105310002E2E2F4D6964646C6577617265732F540E
:10532000686972645F50617274792F4C7749502FAD
:105330007372632F636F72652F6D656D702E6300DE
:105340006D656D705F6D616C6C6F633A206D656D3E
:10535000702070726F7065726C7920616C69676E15
:1053600065640000417373657274696F6E20222555
:105370007322206661696C6564206174206C696EBB
:105380006520256420696E2025730A0070B50546E6
:105390000024084E04EB440006EBC000017D29B157
:1053A0008068A84202D1204600F046F9641C0A2C0D
:1053B000F0DB70BD909800202DE9F74F86B0804655
:1053C00091464FF00A0BDA460A2700240A2004907F
:1053D0000020039002900190584904EB440001EB37
:1053E000C0060590357D0A2F01D1002D1ED0002D5D
:1053F00028D0012D08D0022D06D251A340F223124D
:105400005DA16DA0FAF7EEFFB8F1000F10D0D8F84B
:105410000000716888420BD1B9F1000F02D0B0686A
:10542000484505D109B02046BDE8F08F274609E080
:10543000012D10D0022D05D3708A0199884201D325
:10544000A2460190601C04B20A2CC5DB079810F03C
:10545000020F1DD112E03948059950F8310030B1E2
:10546000708A03998842EDD304940390EAE7708A26
:1054700002998842E6D3A3460290E3E70A2F03D1BC
:10548000079810F0010F03D00A2F06DA3C462BE0F4
:1054900009B04FF0FF30BDE8F08FBAF10A0F0EDA15
:1054A0005446264804EB440150F8310080B124A34F
:1054B00040F26D124AA140A0FAF794FF08E0BBF158
:1054C0000A0F01DA5C4603E004980A2831DA049CEA
:1054D0000A2C06DB1AA340F27F1247A136A0FAF786
:1054E00081FF204600F0A8F80A2C06DB14A340F246
:1054F000831241A130A0FAF775FF104804EB440174
:1055000000EBC105287D30B10DA34FF4C2723FA15D
:1055100029A0FAF767FFB8F1000F02D0D8F8000011
:10552000686000206882C5F8089009B02046BDE890
:10553000F08F09B04FF0FF30BDE8F08F9098002059
:105540002E2E2F4D6964646C6577617265732F54DC
:10555000686972645F50617274792F4C7749502F7B
:105560007372632F636F72652F697076342F657461
:10557000686172702E6300007374617465203D3D34
:10558000204554484152505F53544154455F504563
:105590004E44494E47207C7C207374617465203EE4
:1055A0003D204554484152505F53544154455F5348
:1055B0005441424C45000000417373657274696F39
:1055C0006E2022257322206661696C6564206174F7
:1055D000206C696E6520256420696E2025730A00A1
:1055E0006172705F7461626C655B695D2E71203DF4
:1055F0003D204E554C4C000069203C204152505FEC
:105600005441424C455F53495A4500006172705FF6
:105610007461626C655B695D2E7374617465203DB5
:105620003D204554484152505F53544154455F45D5
:105630004D5054590000000070B5084D00EB400477
:10564000002655F83400002803D004F0AFF945F8DF
:10565000346005EBC400067570BD00009098002012
:10566000F0B587B007460D46002D05D07C68208830
:10567000B0F5807F12D108E023A340F28A2230A146
:1056800033A0FAF7AFFE07B0F0BD2079062805D1A8
:105690006079042802D16088082804D0384604F0D4
:1056A00085F907B0F0BDD4F80E000690A06905900A
:1056B000696819B1884203D1012602E0002600E0A2
:1056C00000260EB1012300E0022304F1080206A91E
:1056D000284600F0CDFBE088B0F5807F0ED16EB19A
:1056E0002B1D022006A9009304F1080202910390E9
:1056F000263301921946284600F0B0FA384604F0E5
:1057000055F907B0F0BD00002E2E2F4D6964646C72
:105710006577617265732F54686972645F50617256
:1057200074792F4C7749502F7372632F636F7265B2
:105730002F697076342F6574686172702E63000073
:105740006E6574696620213D204E554C4C0000006A
:10575000417373657274696F6E202225732220660F
:1057600061696C6564206174206C696E65202564D4
:1057700020696E2025730A0070B584B004460E4679
:105780001546002C06D14CA340F21E3258A15CA055
:10579000FAF728FE36B948A340F21F3262A158A09A
:1057A000FAF720FE280006D143A34FF4487261A106
:1057B00053A0FAF717FE2146286800F051FF08B100
:1057C000604B44E0286800F0F001E0292AD0A1688D
:1057D000636800EA010219408A4208D080B2A0F54D
:1057E0007E41A93903D0E068E0B304F10C05564BC3
:1057F00056491A7802EB420001EBC00090F814C041
:10580000BCF1020F33D3D0F808C0A4452FD1D5F88E
:1058100000C0406884452AD13146204600F098F8FF
:1058200004B070BD01208DF8080000208DF809003B
:105830005E208DF80A00687800F07F008DF80B007C
:10584000A8788DF80C00E8788DF80D0002AB4FF4C5
:105850000060009004F12A023146204600F046FC28
:1058600004B070BDFFE704B06FF0030070BD00220C
:1058700002EB420001EBC00090F814C0BCF1020F33
:105880000FD3D0F808C0A4450BD1D5F800C04068AC
:10589000844506D11A703146204600F059F804B00C
:1058A00070BD501CC2B20A2AE2D3324629462046B5
:1058B00000F0D0F804B070BD2E2E2F4D6964646CDA
:1058C0006577617265732F54686972645F506172A5
:1058D00074792F4C7749502F7372632F636F726501
:1058E0002F697076342F6574686172702E630000C2
:1058F0006E6574696620213D204E554C4C000000B9
:10590000417373657274696F6E202225732220665D
:1059100061696C6564206174206C696E6520256422
:1059200020696E2025730A007120213D204E554CC0
:105930004C00000069706164647220213D204E5566
:105940004C4C0000201C01082C01002090980020E5
:10595000F8B505460E461A4802EB420100EBC104B9
:10596000207D022806D217A340F2EE2223A12FA009
:10597000FAF738FD207D022816D1618A0327B1F598
:105980008E7F06D9211D284600F026FA60B92775BA
:105990000AE0B1F5877F07D304F10C02211D2846E8
:1059A00000F020FA00B927754FF40060009004F170
:1059B0000C0305F12A023146284600F097FBF8BD9A
:1059C000909800202E2E2F4D6964646C657761726B
:1059D00065732F54686972645F50617274792F4CDB
:1059E0007749502F7372632F636F72652F697076DA
:1059F000342F6574686172702E6300006172705F8D
:105A00007461626C655B6172705F6964785D2E734E
:105A100074617465203E3D204554484152505F53A7
:105A2000544154455F535441424C450041737365A2
:105A30007274696F6E2022257322206661696C651D
:105A400064206174206C696E6520256420696E2075
:105A500025730A002DE9F04F83B082460F461646A3
:105A60000AF12A0002904FF0FF344FF0000851462F
:105A7000386800F0F5FD90B9386800F0F001E029D1
:105A80000DD067B158B1524601213846FFF794FC5A
:105A90000546002D08DA03B068B2BDE8F08F03B008
:105AA0006FF00F00BDE8F08F7F2D06D33CA340F2CE
:105AB000C13249A14CA0FAF795FC05F0FF0B544800
:105AC0000BEB4B0900EBC905297D29B94FF0010803
:105AD00001212975C5F808A0287D012808D00228D1
:105AE00006D22FA340F2CD324AA13FA0FAF77AFCAA
:105AF000B8F1000F00D12EB93946504600F06CF9CC
:105B0000044696B1287D424F022812D34B4880F8B4
:105B100000B04FF40060009005F10C033146504690
:105B2000029A00F0E3FA044635E003B02046BDE8EF
:105B3000F08F01282FD100253446608921898842C1
:105B400008D1206830B116A340F2F1323CA126A062
:105B5000FAF748FC207B10F0400F01D0012502E04D
:105B60002468002CE9D13DB132464FF420710E205B
:105B700003F03EFD064602E0304604F0A9F846B1C7
:105B800057F8390008B103F011FF47F839600024D5
:105B900001E04FF0FF3403B02046BDE8F08F000075
:105BA0002E2E2F4D6964646C6577617265732F5476
:105BB000686972645F50617274792F4C7749502F15
:105BC0007372632F636F72652F697076342F6574FB
:105BD000686172702E63000074797065206F76655D
:105BE00072666C6F77000000417373657274696F41
:105BF0006E2022257322206661696C6564206174C1
:105C0000206C696E6520256420696E2025730A006A
:105C1000909800206172705F7461626C655B695D71
:105C20002E7374617465203D3D2050454E44494EAD
:105C300047206F7220535441424C45002C010020F4
:105C40006E6F207061636B65742071756575657327
:105C500020616C6C6F776564210000002DE9FF4FB7
:105C600081B00646DDF84090DDF83C800E9F9A46F4
:105C70004FF0000B002E06D12DA340F257423AA15F
:105C80003DA0FAF7AFFB4FF420721C210E2003F069
:105C90005DFA0546280045D068891C2806D224A351
:105CA00040F262423EA134A0FAF79CFB6C68119866
:105CB00001F034FEE08096F83000062806D01CA3E0
:105CC00040F2694243492CA0FAF78CFBDAF8000055
:105CD000A060BAF80400A081D8F80000C4F812004F
:105CE000B8F80400E0823868C4F80E00D9F8000063
:105CF000A0614FF480702080082060800620207111
:105D00000420607140F60600009029463046039B4F
:105D1000029A00F0EBF9284603F048FE05B0584619
:105D2000BDE8F08F05B04FF0FF30BDE8F08F000008
:105D30002E2E2F4D6964646C6577617265732F54E4
:105D4000686972645F50617274792F4C7749502F83
:105D50007372632F636F72652F697076342F657469
:105D6000686172702E6300006E6574696620213D63
:105D7000204E554C4C000000417373657274696F7E
:105D80006E2022257322206661696C65642061742F
:105D9000206C696E6520256420696E2025730A00D9
:105DA000636865636B2074686174206669727374DC
:105DB00020706275662063616E20686F6C6420736A
:105DC0007472756374206574686172705F68647260
:105DD00000000000EC1D0108014A00F003B80000BB
:105DE000201C010810B584B001230393DFF818C00C
:105DF000041D029100F12A03CDF804C00094194655
:105E0000FFF72CFF04B010BD261C01082DE9F0415E
:105E100000240426154D022704EB440005EBC002C4
:105E2000117DE9B1508A401C80B25082B0F5967F56
:105E300003D2012905D1052803D32046FFF7FCFB37
:105E40000EE0032904D0042904D0012904D007E07E
:105E5000167505E0177503E0111D9068FFF7BCFF8C
:105E6000641C0A2CD8DBBDE8F0810000909800206B
:105E7000F8B504460D4616461F4694F8300006282D
:105E800006D020A340F2A9122CA135A0FAF7AAFA55
:105E90009DB1286888B1214600F0E2FB68B92878F6
:105EA00000F0F000E02808D0224639462846FFF7E7
:105EB00083FA002804DA40B2F8BD6FF00F00F8BD95
:105EC000314A00EB400102EBC100022303758460FC
:105ED0003368C360B38803820023438252F8315091
:105EE00075B142F831304FF400600090334604F150
:105EF0002A022946204600F0F9F8284603F056FD0C
:105F00000020F8BD2E2E2F4D6964646C6577617298
:105F100065732F54686972645F50617274792F4C95
:105F20007749502F7372632F636F72652F69707694
:105F3000342F6574686172702E6300006E65746939
:105F4000662D3E6877616464725F6C656E203D3DCE
:105F5000204554485F4857414444525F4C454E00E9
:105F6000417373657274696F6E20222573222066F7
:105F700061696C6564206174206C696E65202564BC
:105F800020696E2025730A00909800202DE9F041C9
:105F900004460D460E2760890E2840D9E07B18B9CB
:105FA00095F83400401CE07360688689017811F030
:105FB000010F15D0012905D006221F49FAF7D6FA9C
:105FC00050B10DE0417859B980785E2808D1607BE6
:105FD00040F01000607303E0607B40F008006073E5
:105FE000082E03D0B6F5C16F19D10EE095F8310037
:105FF00010F0080F13D03946204603F0AFFE70B9F9
:106000002946204600F0A0FC13E095F8310010F07E
:10601000080F04D03946204603F0A0FE28B12046E0
:1060200003F0C4FC0020BDE8F08129462046FFF7BC
:1060300017FB0020BDE8F081201C0108F0B599B0E5
:10604000074664216846FAF702FB00240025002673
:106050002348FDF7EDFD97F8311011F0040F0CD037
:1060600001280ADC1F48FBF7B5FD384602F054FE54
:10607000384602F0C5FE19B0F0BD11F0040FFAD198
:106080000128F8DD022806D0032809D004280BD007
:1060900005280ED10CE04FF40066F500012408E05D
:1060A0004FF48045012404E04FF40066012400E031
:1060B0000124002CDFD069460A48FBF7ABFA0696AC
:1060C000059569460748FBF701FD0648FBF73CFDCF
:1060D000384602F065FF384602F0F8FE19B0F0BD10
:1060E000746000208C5F0020704700002DE9F041B3
:1060F00006460F4615461C46069801F00FFC8046E2
:106100000E21384602F0B6FF18B16FF00100BDE86D
:10611000F0817868A0F80C8021680160A1888180F6
:106120002968C0F80610A988418196F83000062831
:1061300006D006A34FF4997212A11FA0FAF752F9E4
:1061400039463046B269BDE8F04110472E2E2F4D3A
:106150006964646C6577617265732F5468697264F1
:106160005F50617274792F4C7749502F7372632F8F
:106170006E657469662F65746865726E65742E63EA
:10618000000000006E657469662D3E687761646486
:10619000725F6C656E206D757374206265203620A9
:1061A000666F722065746865726E65745F6F757472
:1061B0007075742100000000417373657274696F1B
:1061C0006E2022257322206661696C6564206174EB
:1061D000206C696E6520256420696E2025730A0095
:1061E00010B50446002C06D10AA340F26B1210A190
:1061F00013A0FAF7F7F8732084F83200742084F8BB
:106200003300194860611948A061204601F06CFA1A
:10621000002010BD2E2E2F4C5749502F546172670D
:1062200065742F65746865726E657469662E6300A7
:106230006E6574696620213D204E554C4C0000006F
:10624000417373657274696F6E2022257322206614
:1062500061696C6564206174206C696E65202564D9
:1062600020696E2025730A007957000825780008F8
:1062700070B50546284601F0C3FA04463CB12A69C8
:1062800029462046904710B1204603F08FFB002C92
:10629000F0D170BD13B50C464FF6FF73012269466D
:1062A0000248FDF714FC00981CBD0000C802002045
:1062B0007047000010B5002220211048FBF77EFE39
:1062C0006420FBF793F9012220210C48FBF776FEAE
:1062D000FF220B490B48FCF750FFFF220A490B48ED
:1062E000FCF74BFFFF220A490A48FCF746FFFF2252
:1062F00009490A48FCF741FF10BD000000100240A8
:106300006C060020100300206B07002038020020DC
:106310006A0800208002002069090020C8020020CD
:106320000A46032100F00EB92DE9F04784B0044677
:106330008846504FD7F808A09AF800000007850E4D
:10634000142DC0F0918060890428C0F08D806068B1
:106350000178002900F08280082940F07F8007F151
:106360001409786900F0F001E02954D0396800F090
:1063700077F900284FD120890828C0F0758005F1F1
:106380000E01204602F076FE002838D020894119FF
:1063900089B288423FD84FF420720E2002F0D6FE18
:1063A0000646002E37D0708905F10801884203D2D5
:1063B000304603F0FBFA2EE02A4651467068FAF7A1
:1063C00001F92946304603F0C9FC002809D02AA368
:1063D000B62237A144A0FAF705F8304603F0E6FAF2
:1063E00019E02146304603F053F918B1304603F066
:1063F000DDFA10E0204603F0D9FA344611E005F149
:106400000E01204603F0AAFC58B11BA3C72240A1ED
:1064100035A0F9F7E7FF04B02046BDE8F04703F0E8
:10642000C5BA66682946204602F024FEB0B9606805
:10643000D9F80010C16039690161002131707180A3
:10644000FF2202724181012000910190FF2300226E
:10645000CDF808804946204600F058FB04B020469D
:10646000BDE8F04703F0A2BA04B02046BDE8F0470B
:1064700003F09CBACC6000202E2E2F4D6964646C12
:106480006577617265732F54686972645F506172D9
:1064900074792F4C7749502F7372632F636F726535
:1064A0002F697076342F69636D702E6300000000D1
:1064B00069636D705F696E7075743A206D6F76698F
:1064C0006E6720722D3E7061796C6F616420746F0D
:1064D0002069636D7020686561646572206661691A
:1064E0006C65640A00000000417373657274696F23
:1064F0006E2022257322206661696C6564206174B8
:10650000206C696E6520256420696E2025730A0061
:1065100069636D705F696E7075743A20726573742B
:106520006F72696E67206F726967696E616C207047
:106530002D3E7061796C6F6164206661696C656481
:106540000A0000002DE9F04385B0064688469146D2
:106550004FF420722421222002F0F8FD0546280085
:1065600031D06889242806D218A34FF4B47225A12B
:106570002FA0F9F737FF77686C6884F8008084F8FB
:1065800001904FF00008A4F80480A4F80680686821
:10659000716808301C22FAF715F8F868049004A80E
:1065A00000F0C8FC60B1A4F80280012101910290C2
:1065B000FF2304AACDF800800021284600F0A6FAA7
:1065C000284603F0F3F905B0BDE8F0832E2E2F4DD9
:1065D0006964646C6577617265732F54686972646D
:1065E0005F50617274792F4C7749502F7372632F0B
:1065F000636F72652F697076342F69636D702E63D7
:1066000000000000636865636B2074686174206635
:106610006972737420706275662063616E20686FA2
:106620006C642069636D70206D65737361676500CC
:10663000417373657274696F6E2022257322206620
:1066400061696C6564206174206C696E65202564E5
:1066500020696E2025730A000A460B21FFF772BFDE
:1066600081B00090B0F1FF3F0CD002000AD091F849
:10667000312012F0020F08D04A68824208D100206F
:1066800001B07047012001B07047002001B0704791
:10669000896800EA01030A40934203D10843B0F13C
:1066A000FF3F02D0002001B07047012001B07047C9
:1066B0002DE9F74F8AB0044600270B98008D143857
:1066C000C11700EB5170C0F3CF000590142660682D
:1066D00007900798017801F00F01052903D00DB04C
:1066E000B81FBDE8F08F618914290BD269A34FF45C
:1066F0003F7277A17DA0F9F775FE0DB06FF0050030
:10670000BDE8F08FC08801F009F9C0F30C010491D5
:1067100000F400500390208914381FFA80F8B8F173
:10672000000F00F0B38005984FF6FF7101EAC0003A
:1067300009900998404501D9C24601E0DDF824A03E
:106740004FF4207214210E2002F000FD83465FEA10
:106750000B0000F06A80BBF80A00142806D24DA393
:106760004FF449726BA161A0F9F73CFE0798DBF882
:10677000041002680A6042684A6082688A60C268DF
:10678000CA6000690861DBF8040006905546002DD8
:1067900035D06089811B8FB2B04206D23DA340F252
:1067A0002D3264A151A0F9F71DFEBD4200D22F4643
:1067B00077B300F0FBFB81465FEA09002BD06068ED
:1067C0004B4630440090412239460197002002F0A8
:1067D00047FE0890089810B3204603F079FAC9F8EC
:1067E00014405848C9F810005846089902F05AFE5B
:1067F000E81B85B20DB100262468002DC9D1F0191F
:1068000086B20B98008D1438404513DB012112E04D
:1068100000262468F1E7584603F0C8F805E048462A
:1068200000F0C8FB584603F0C1F80DB04FF0FF3040
:10683000BDE8F08F00210498C0F30C0009B1039962
:1068400009B140F4005001F069F80699C8800AF1D6
:10685000140080B201F062F8069948800699002081
:1068600048810B9859460C9A43699847584603F05B
:106870009DF8A8EB0A001FFA80F8059904980844CF
:1068800080B20490B8F1000F7FF453AF0DB0002038
:10689000BDE8F08F2E2E2F4D6964646C65776172B0
:1068A00065732F54686972645F50617274792F4CFC
:1068B0007749502F7372632F636F72652F697076FB
:1068C000342F6970345F667261672E6300000000C8
:1068D0006970345F6672616728293A207062756654
:1068E00020746F6F2073686F72740000417373655A
:1068F0007274696F6E2022257322206661696C654F
:1069000064206174206C696E6520256420696E20A6
:1069100025730A0074686973206E6565647320616D
:10692000207062756620696E206F6E6520706965E3
:1069300063652100702D3E6C656E203E3D20706FBA
:1069400066660000517600082DE9F04707460E46BE
:106950007D6804212878B1EB101F05D0384603F07C
:1069600025F80020BDE8F08700074FEA90686888A6
:1069700000F0D4FF04463889A04203D921463846A6
:1069800003F00AF97889404505D33889A04202D33B
:10699000B8F1140F05D2384603F008F80020BDE81E
:1069A000F087DFF834912869C9F81400E968C9F85C
:1069B000101000F0F000E02805D0304600F090F80C
:1069C00060B134461BE096F8310010F0010F03D09F
:1069D000706808B1344612E0002410E0002499F8F1
:1069E00014007F280BD03D48046844B1B44203D062
:1069F000204600F075F810B92468002CF6D1314615
:106A0000D9F81000FFF72CFE58BB99F8100000F0E1
:106A1000F000E02825D054B3E88830F0C00005D05D
:106A2000384600F04DF907463FB37D68C9F800408D
:106A3000C9F80460C9F8085028780007800EA9F842
:106A40000C004146384603F089F9687A01281CD0C9
:106A5000062815D02146D9F81400FFF701FEC8B169
:106A600027E0384602F0A2FF0020BDE8F087384654
:106A700002F09CFF0020BDE8F0870020BDE8F08711
:106A80003146384605F0BAF916E031463846FFF788
:106A90004BFC11E099F8140000F0F000E02808D059
:106AA0000FFA88F1384603F055F802213846FFF70F
:106AB00037FC384602F07AFF0020C9F80000C9F818
:106AC0000400C9F80800A9F80C00C9F81000C9F8BA
:106AD0001400BDE8F0870000CC600020D00000204A
:106AE00010B5014691F8310010F0010F0AD04A6844
:106AF00042B105484069904202D0FFF7B1FD08B1AC
:106B0000012010BD002010BDCC60002070B584B005
:106B1000DDF828C0099D089C002A05D00E0001D090
:106B20000E680EB90CF10401CDF808C0019500946F
:106B300000F002F804B070BD2DE9F84FDDF82CA08C
:106B4000DDF828900C9F0546884616469B46A87B94
:106B5000012806D032A34FF455723EA140A0F9F7A8
:106B600041FC002E3ED01421284602F083FA18B1D1
:106B70006FF00100BDE8F88F6C686889142806D2B0
:106B800027A34FF4627240A135A0F9F72BFC84F8DB
:106B900008B084F809A0306820614520207084F88E
:106BA0000190288900F0BAFE60804FF0000AA4F836
:106BB00006A0DFF80491B9F8000000F0AFFEA08055
:106BC000B9F80000401CA9F80000B8F1000F05D08A
:106BD000D8F80000E060A4F80AA00EE0374800688A
:106BE000E060F8E76889142803D26FF00100BDE87F
:106BF000F88F6868006900906E46388D48B1298921
:106C0000814206D9324639462846FFF751FDBDE894
:106C1000F88F7B693246294638469847BDE8F88F99
:106C20002E2E2F4D6964646C6577617265732F54E5
:106C3000686972645F50617274792F4C7749502F84
:106C40007372632F636F72652F697076342F69706A
:106C5000342E6300702D3E726566203D3D2031006C
:106C6000417373657274696F6E20222573222066EA
:106C700061696C6564206174206C696E65202564AF
:106C800020696E2025730A00636865636B20746851
:106C90006174206669727374207062756620636126
:106CA0006E20686F6C6420737472756374206970F1
:106CB0005F686472000000002E010020181D0108AA
:106CC0002DE9F0478246DAF80450287800F00F00EA
:106CD000052840F0D780E88800F020FEC004060CAC
:106CE000688800F01BFE014628780007800E884265
:106CF00000F2C880081A1FFA80F9504602F06EFCB4
:106D00008046634F388840440A280BD941462846BC
:106D100000F048FC002800F0B580388840440A287C
:106D200000F2B0807C6874B1E8686169814207D183
:106D3000A1692A69914203D1A189AA88914202D00E
:106D40002468002CF1D134B1E88800F0E7FDC004DC
:106D5000C00C09D018E04146284600F01FFB04464D
:106D6000002C00F08F800FE0E08900F0D7FDC00418
:106D7000C00C09D02868A0606868E060A86820613D
:106D8000E86860612869A061E888012121EA50155E
:106D900045B106EB090080B2B04263D34FF6EB7108
:106DA00088425FD82A465146204600F04DF9B0F19E
:106DB000FF3F57D039884144398035B106EB09018E
:106DC000A183A17F41F00101A177012802D0002019
:106DD000BDE8F087A08B143080B261684E683568DA
:106DE000A1683160E16871602169B1606169F16039
:106DF000A169316100F092FD70800020F080708107
:106E0000D4F804805DB16E681421284602F0A6FF14
:106E10002946404602F046FB3568002DF3D17968DB
:106E20008C4201D1002106E029B10868A04202D0BD
:106E300001460029F9D1204600F052FA404602F0FE
:106E4000CDFB04463888A04206D212A340F29B2212
:106E50001FA126A0F9F7C6FA3888001B38804046E3
:106E6000BDE8F087606868B97868844206D009A3F5
:106E700040F2AB2227A11DA0F9F7B4FA0021204669
:106E800000F02EFA504602F091FD0020BDE8F08798
:106E9000300100202E2E2F4D6964646C657761727D
:106EA00065732F54686972645F50617274792F4CF6
:106EB0007749502F7372632F636F72652F697076F5
:106EC000342F6970345F667261672E6300000000C2
:106ED00069705F72656173735F70627566636F7509
:106EE0006E74203E3D20636C656E000041737365D7
:106EF0007274696F6E2022257322206661696C6549
:106F000064206174206C696E6520256420696E20A0
:106F100025730A006E6F74206669727374616C74F5
:106F2000686F756768206A75737420656E71756522
:106F30007565640030B404461A48006800281DD006
:106F400090F8311011F0010F15D011F0040F12D08C
:106F5000D0F804C0BCF1000F0DD02268836802EAAB
:106F600003050CEA03039D4219D011F0020F02D170
:106F7000C1688A4213D000680028E1D10A4800683D
:106F800060B190F8311011F0010F07D011F0040F2B
:106F900004D0416811B121787F2900D1002030BC94
:106FA00070470000D0000020D4000020042001F031
:106FB0002BB9000010B50446002C06D106A34FF4EF
:106FC000317214A116A0F9F70DFA2146BDE8104060
:106FD000042001F057B800002E2E2F4D6964646C18
:106FE0006577617265732F54686972645F5061726E
:106FF00074792F4C7749502F7372632F636F7265CA
:107000002F697076342F6970345F667261672E6302
:10701000000000007020213D204E554C4C00000027
:10702000417373657274696F6E2022257322206626
:1070300061696C6564206174206C696E65202564EB
:1070400020696E2025730A002DE9F047074688461F
:10705000914600250126D8F80440608800F05EFCC7
:10706000014620780007800E884202D9681EBDE8DC
:10707000F087A1EB000AE08800F050FCC004000C8F
:10708000D8F8044000212160A08000EB0A018AB2F8
:10709000E280824203D24FF0FF30BDE8F087D7F89C
:1070A00004C0BCF1000F3BD0DCF804309988884262
:1070B0001DD2C4F800C085B1E988884202D39888FF
:1070C000824203D94FF0FF30BDE8F087C5F8008059
:1070D000A088814224D0002622E09888824203D9E9
:1070E0004FF0FF30BDE8F087C7F8048018E003D107
:1070F0004FF0FF30BDE8F087B3F806C0604503D21B
:107100004FF0FF30BDE8F08725B1B5F806C08C45DB
:1071100000D00026D3F800C01D46BCF1000FC3D13B
:10712000BCF1000F1ED195B1E888A188884206D92C
:107130002FA34FF4DB723DA144A0F9F753F9C5F832
:107140000080E888A18888420CD000260AE0786890
:1071500030B127A34FF4DF7246A13CA0F9F742F902
:10716000C7F80480B9F1000F03D1B87F10F0010F08
:107170003BD0002E32D07A6812B15068808808B1B6
:1071800000262BE02168204651B14C68C088A188B8
:10719000884201D0002603E0216820460029F4D16E
:1071A000002E1BD032B912A340F2DF123FA127A05C
:1071B000F9F718F978684068A04206D10CA34FF49B
:1071C000F0723AA121A0F9F70DF9206830B108A3B7
:1071D0004FF4F17239A11DA0F9F704F916B101209D
:1071E000BDE8F0870020BDE8F0870020BDE8F0870B
:1071F0002E2E2F4D6964646C6577617265732F5410
:10720000686972645F50617274792F4C7749502FAE
:107210007372632F636F72652F697076342F697094
:10722000345F667261672E63000000006368656307
:107230006B20667261676D656E747320646F6E2774
:1072400074206F7665726C61700000004173736525
:107250007274696F6E2022257322206661696C65E5
:1072600064206174206C696E6520256420696E203D
:1072700025730A006E6F2070726576696F757320D2
:10728000667261676D656E742C2074686973206D19
:107290007573742062652074686520666972737402
:1072A00020667261676D656E7421000073616E699E
:1072B000747920636865636B0000000076616C6917
:1072C000646174655F646174616772616D3A6E6573
:1072D00078745F70627566213D4E554C4C0000001D
:1072E00070B504460D460C484168A14202D12168A0
:1072F00041600AE0002D06D108A340F2451216A114
:107300001CA0F9F76FF8206828602146BDE870409E
:10731000032000F0B7BE0000300100202E2E2F4DBC
:107320006964646C6577617265732F54686972640F
:107330005F50617274792F4C7749502F7372632FAD
:10734000636F72652F697076342F6970345F66726F
:1073500061672E630000000073616E6974792063B9
:107360006865636B206C696E6B6564206C6973740F
:1073700000000000417373657274696F6E202225EE
:107380007322206661696C6564206174206C696E8B
:107390006520256420696E2025730A0070B50546B6
:1073A0000E46032000F030FF044654B9314628460B
:1073B00000F0F8F8B04203DB032000F025FF04469C
:1073C000CCB100216160A160E16021616161A161D6
:1073D000E1610F20E0770948416821604460286836
:1073E000A0606868E060A8682061E868606128695A
:1073F000A061204670BD002070BD0000300100205B
:107400002DE9F04106460F460025B74205D132A3CB
:10741000AB2240A142A0F8F7E5FF002F08D0386862
:10742000B04205D02CA3AD2247A13DA0F8F7DAFF6A
:10743000746860688188002921D100687060606884
:10744000B1680160F1684160316981607169C16052
:10745000B169016101212046FFF7FEF8204602F0E4
:10746000BDF80546B5F5803F05D31BA3BC223BA163
:107470002BA0F8F7B7FFADB2204602F097FA746878
:10748000002C15D06068A0460468404602F0A6F8BB
:107490000544B5F5803F05D30FA3CC222FA120A032
:1074A000F8F7A0FFADB2404602F080FA002CE9D117
:1074B00039463046FFF714FF304C2088A84205D2E9
:1074C00005A3D2222EA116A0F8F78CFF2088401B1E
:1074D00020802846BDE8F0812E2E2F4D6964646C13
:1074E0006577617265732F54686972645F50617269
:1074F00074792F4C7749502F7372632F636F7265C5
:107500002F697076342F6970345F667261672E63FD
:10751000000000007072657620213D2069707200C5
:10752000417373657274696F6E2022257322206621
:1075300061696C6564206174206C696E65202564E6
:1075400020696E2025730A00707265762D3E6E6587
:107550007874203D3D20697072000000706275668D
:10756000735F6672656564202B20636C656E203CDA
:107570003D2030786666666600000000300100201D
:1075800069705F72656173735F70627566636F7552
:107590006E74203E3D2070627566735F667265652D
:1075A000640000002DE9F04705460F460026DFF88D
:1075B0006C800020002184460024D8F80420EAB121
:1075C000D5F80C9053694B4509D19369D5F810A0B3
:1075D000534504D19389B5F804A0534508D0641CE1
:1075E000C0B1D37F90F81FA0534501D810468C46F8
:1075F000136803B111461A46002AE3D118B1614657
:10760000FFF7FEFE0644BE4201DA012CD1DC304613
:10761000BDE8F08710468C46EAE700003001002004
:1076200070B5002509484468002C0DD0E07F20B1DA
:10763000401EE0772546246804E020462468294659
:10764000FFF7DEFE002CF1D170BD000030010020FC
:1076500010B50446002C06D107A340F2CE2215A196
:1076600017A0F8F7BFFE606908B102F09FF9204645
:10767000BDE81040FFF79EBC2E2E2F4D6964646C50
:107680006577617265732F54686972645F506172C7
:1076900074792F4C7749502F7372632F636F726523
:1076A0002F697076342F6970345F667261672E635C
:1076B0000000000070637220213D204E554C4C00AC
:1076C000417373657274696F6E2022257322206680
:1076D00061696C6564206174206C696E6520256445
:1076E00020696E2025730A00F0B583B00546414E2F
:1076F0003F48306000248DF8044080208DF805005C
:10770000E1208DF806008DF807408DF808408DF8CF
:10771000094001A870604FF40000B060A6F1A0001D
:10772000F060A03830614FF4C0607061CD208DF8FA
:1077300009003046F9F7E8FF0746A6F5A071C1F841
:10774000F441C1F8F841C1F8FC41C1F80042C1F868
:107750000842C1F80C42C1F81042C1F81442C1F805
:107760001842C1F81C42C1F82042C1F8244206F177
:10777000B000212101604FF4400141611E4800F03A
:107780002BFD062085F830007068007885F82A0007
:107790007068407885F82B007068807885F82C0038
:1077A0007068C07885F82D007068007985F82E0023
:1077B0007068407985F82F0040F2DC50288595F8F4
:1077C000310040F00A0085F831000C4906F1E8006C
:1077D000FCF7B9FA06F1E800FCF788FA1FB1F9F7EF
:1077E00057FC03B0F0BD2846FEF728FC03B0F0BDFF
:1077F000008002408C5F0020141C010868000020FB
:1078000008B50020009005480078002803D169469B
:107810000348FAF765F8009808BD000064000020EE
:107820008C5F002070B58CB0002300259C46CDF8FD
:1078300000C0CDF804C0CDF808C0CDF80CC0CDF81C
:1078400010C0CDF814C0CDF818C0CDF81CC0CDF8CC
:1078500020C0CDF824C0CDF828C0CDF82CC00A46F1
:1078600011006E461DD0042B03D30CB06FF00B003B
:1078700070BD03EB4304506846F8240006EB840413
:10788000508960602BB1581E00EB400006EB800071
:107890008460106808B9C4F808C05B1C1268002A2C
:1078A000E1D106480A89426086604163014614229C
:1078B000B038FAF7D0F90CB0284670BD3C60002013
:1078C00010B504466068804703F0A4F901460B4AEE
:1078D0002068526883185A1AB2F1004F06D3224624
:1078E0000844BDE81040064903F0F8B92246BDE857
:1078F00010400349184603F0F1B9000020010020B0
:10790000C1780008010600F47F4241EA022100F438
:107910007F0241EA122141EA106070470106090C1A
:1079200041EA1020704710B500F02EF900F046FC37
:1079300001F0D6F804F056FABDE8104003F04EBA54
:10794000FAF754FBFCF788FDFCF778FAFCF712FA1B
:10795000FCF790FCFCF7D2FCFCF7F0FCFCF70EFD0A
:10796000FCF71AFCFCF750FCFCF728FDFCF754FB75
:107970001D48FBF79DF81D48FBF7FDFA04211B4845
:10798000FBF72EFB4320194909688863FEF792FC38
:1079900008F0C8F8FDF7D6FB24E0FCF7EFFB14482D
:1079A0000068401E134931F8100000EE100AB8EECE
:1079B000400ADFED110A80EE201A104880ED001A0F
:1079C0000B4908780D4991ED000AFDF7D5FB0848F1
:1079D0000068401C0649086008460068042801DD6C
:1079E00001200860D9E7000060010020F0010020BC
:1079F000140000203E0B002000007A4410000020FC
:107A000070B5002842D010F0030F08D0BDE87040D8
:107A10001FA340F273222AA132A0F8F7E3BCA0F121
:107A200008043A4D29688C4203D369680C308842B7
:107A300008D9BDE8704016A340F27F2234A129A0E6
:107A4000F8F7D0BC207978B1204600F0B9F80028CA
:107A500013D000202071A868844200D2AC60204678
:107A6000BDE8704002F0EAB9BDE8704008A34FF4E9
:107A700023722EA11BA0F8F7B5BCBDE8704004A38B
:107A800040F2952233A117A0F8F7ACBC70BD0000FE
:107A90002E2E2F4D6964646C6577617265732F5467
:107AA000686972645F50617274792F4C7749502F06
:107AB0007372632F636F72652F6D656D2E630000A7
:107AC0006D656D5F667265653A2073616E69747984
:107AD00020636865636B20616C69676E6D656E74A9
:107AE00000000000417373657274696F6E20222577
:107AF0007322206661696C6564206174206C696E14
:107B00006520256420696E2025730A009C000020F2
:107B10006D656D5F667265653A20696C6C6567615D
:107B20006C206D656D6F7279000000006D656D5F92
:107B3000667265653A20696C6C6567616C206D657D
:107B40006D6F72793A20646F75626C65206672653C
:107B5000650000006D656D5F667265653A20696C51
:107B60006C6567616C206D656D6F72793A206E6F20
:107B70006E2D6C696E6B65643A20646F75626C651E
:107B8000206672656500000070B50B480B4C20F054
:107B9000030020604FF4C865058000214180017119
:107BA000284602F01DFA60600121017105804580C0
:107BB0002068A06070BD0000E76000209C000020ED
:107BC00070B50446204600F055F90546208802F0BD
:107BD00007FA0646608802F003FA01462088B0F5ED
:107BE000C86F0FD86088B0F5C86F0BD8A84202D014
:107BF0000888A84206D105484068864204D07088AB
:107C0000A84201D0002070BD012070BD9C00002062
:107C10002DE9F04700280FD0C11C21F0030525F401
:107C200080350C2D00D20C25B5F5C86F01D88542E2
:107C300005D20020BDE8F0870020BDE8F087DFF81E
:107C40002481D8F8080000F015F90646C5F5C86784
:107C5000B74240F28480304602F0C2F904462079EF
:107C6000002840F075802088801B0838A842C0F0AA
:107C70006F80208805F11401801B08384FF001093E
:107C800088421FD37019083087B2B7F5C86F06D184
:107C900035A340F2873240A144A0F8F7A3FB384651
:107CA00002F09EF900210171218801804680278021
:107CB00084F804900088B0F5C86F05D002F090F900
:107CC000478001E084F80490D8F80800844203D08B
:107CD00017E0008802F084F9017919B1D8F804108E
:107CE0008842F6D1C8F80800D8F80410884208D0B5
:107CF000007930B11CA340F2B53236A12BA0F8F7C1
:107D000071FB6019D8F804100830884206D916A310
:107D100040F2B93236A125A0F8F764FB04F108005F
:107D200010F0030F06D010A340F2BB323CA11FA0FD
:107D3000F8F758FB14F0030F06D00BA340F2BD3246
:107D400043A11AA0F8F74EFB04F10800BDE8F08744
:107D5000304602F045F90688B7423FF67CAF002076
:107D6000BDE8F0879C0000202E2E2F4D6964646CC6
:107D70006577617265732F54686972645F506172D0
:107D800074792F4C7749502F7372632F636F72652C
:107D90002F6D656D2E630000696E76616C696420DD
:107DA0006E65787420707472000000004173736512
:107DB0007274696F6E2022257322206661696C657A
:107DC00064206174206C696E6520256420696E20D2
:107DD00025730A006D656D5F6D616C6C6F633A2091
:107DE000216C667265652D3E757365640000000048
:107DF0006D656D5F6D616C6C6F633A20616C6C6F6B
:107E00006361746564206D656D6F7279206E6F7447
:107E10002061626F76652072616D5F656E642E0011
:107E20006D656D5F6D616C6C6F633A20616C6C6F3A
:107E30006361746564206D656D6F72792070726F17
:107E40007065726C7920616C69676E65642E0000E4
:107E50006D656D5F6D616C6C6F633A2073616E6907
:107E6000747920636865636B20616C69676E6D650A
:107E70006E74000002490988401A80B27047000001
:107E80009C0000202DE9F05F0646C81C20F003048A
:107E900024F480340C2C00D20C24B4F5C86F01D823
:107EA0008C4202D20020BDE8F09FDFF83091D9F873
:107EB0000000864203D3D9F80400864206D348A3C3
:107EC00040F2D12252A158A0F8F78CFAD9F800005C
:107ED000864203D3D9F80400864202D33046BDE877
:107EE000F09FA6F108052846FFF7C4FF074629883A
:107EF000C81B08381FFA80FB5C4506D938A34FF42D
:107F0000397253A148A0F8F76DFA5C4503D94FF0D8
:107F10000000BDE8F09F02D13046BDE8F09F288800
:107F200002F05EF880464FF0000A98F8040058B15D
:107F300004F1140058454ED83819083084B2288806
:107F4000B0F5C86F2AD030E02888B0F5C86F06D1E8
:107F500023A340F2F52246A133A0F8F743FAB8F87C
:107F600000B03819083084B2D9F80800404504D16F
:107F7000204602F035F8C9F80800204602F030F833
:107F800080F804A0A0F800B047802C800088B0F5ED
:107F9000C86F20D002F024F844801CE010A340F207
:107FA000163233A120A0F8F71DFA204602F018F887
:107FB000D9F80810884201D2C9F8080080F804A056
:107FC0002988018047802C800088B0F5C86F02D0D6
:107FD00002F006F844803046BDE8F09F9C00002087
:107FE0002E2E2F4D6964646C6577617265732F5412
:107FF000686972645F50617274792F4C7749502FB1
:108000007372632F636F72652F6D656D2E63000051
:108010006D656D5F7472696D3A206C6567616C2087
:108020006D656D6F72790000417373657274696F6D
:108030006E2022257322206661696C65642061745C
:10804000206C696E6520256420696E2025730A0006
:108050006D656D5F7472696D2063616E206F6E6C0B
:108060007920736872696E6B206D656D6F7279002F
:10807000696E76616C6964206E65787420707472C4
:1080800000000000082806D307A34FF4D57212A100
:1080900018A0F8F7A7B9002904D0204A52F8200008
:1080A000FDF7D0B8704700002E2E2F4D6964646C28
:1080B0006577617265732F54686972645F5061728D
:1080C00074792F4C7749502F7372632F636F7265E9
:1080D0002F6D656D702E63006D656D705F667265E6
:1080E000653A2074797065203C204D454D505F4DB8
:1080F00041580000417373657274696F6E202225C8
:108100007322206661696C6564206174206C696EFD
:108110006520256420696E2025730A008C1C0108E7
:1081200070B504460D46002C06D109A340F2951205
:1081300013A118A0F8F756F9002C07D0002D05D090
:1081400029462046BDE87040FDF77CB870BD0000B0
:108150002E2E2F4D6964646C6577617265732F54A0
:10816000686972645F50617274792F4C7749502F3F
:108170007372632F636F72652F6D656D702E630070
:10818000696E76616C696420706F6F6C20646573D2
:1081900063000000417373657274696F6E2022255D
:1081A0007322206661696C6564206174206C696E5D
:1081B0006520256420696E2025730A0030B50024EF
:1081C000044D55F8240000F007F8601C84B2082C18
:1081D000F7D330BD8C1C0108826800211160416812
:1081E000C91C21F0030100224388002B0ADD8368AB
:1081F0001B680B608368196003881944521C43880C
:108200009342F4DC7047000010B5082808D308A397
:1082100040F2571212A11AA0F8F7E4F8002010BD9E
:10822000214951F82000BDE81040FDF75BB800007F
:108230002E2E2F4D6964646C6577617265732F54BF
:10824000686972645F50617274792F4C7749502F5E
:108250007372632F636F72652F6D656D702E63008F
:108260006D656D705F6D616C6C6F633A20747970D1
:1082700065203C204D454D505F4D415800000000A9
:10828000417373657274696F6E20222573222066B4
:1082900061696C6564206174206C696E6520256479
:1082A00020696E2025730A008C1C010810B5044655
:1082B000002C06D107A34FF49E7212A116A0F8F766
:1082C00091F824B12046BDE81040FDF70BB800201E
:1082D00010BD00002E2E2F4D6964646C65776172AD
:1082E00065732F54686972645F50617274792F4CA2
:1082F0007749502F7372632F636F72652F6D656DB1
:10830000702E6300696E76616C696420706F6F6CAB
:108310002064657363000000417373657274696F54
:108320006E2022257322206661696C656420617469
:10833000206C696E6520256420696E2025730A0013
:108340002DE9F04104460D460CB1022D01DABDE8DD
:10835000F0812678677828480068864201D0002E90
:1083600048D1052F3AD008DC012F0DD0022F11D0B3
:10837000032F15D0042F37D118E0062F1CD00F2F54
:1083800020D0102F30D123E0A81E81B2A01C01F014
:108390002DFE2EE0A81E81B2A01C01F0AFFF28E048
:1083A000A81E81B2A01C02F027F922E0A81E81B20B
:1083B000A01C02F057FA1CE0A81E81B2A01C09F014
:1083C00031FB16E0A81E81B2A01C08F077FF10E078
:1083D000A81E81B2A01C09F001F90AE0A81E81B212
:1083E000A01C09F031FA04E06078012100F07EF869
:1083F00000BF00BF00BFAAE75C0000202DE9F041EC
:1084000004460D460CB1022D01DABDE8F0810020D2
:1084100003E0215C334A1154401C0428F9DBA6799F
:10842000E77931480068864201D0002E58D1052FE7
:1084300048D008DC012F0DD0022F13D0032F19D004
:10844000042F47D11EE0062F24D00F2F2AD0102F43
:1084500040D12FE0A5F1080081B204F1080001F03D
:108460007BFE3CE0A5F1080081B204F1080001F0B8
:10847000F7FF34E0A5F1080081B204F1080002F032
:1084800043F92CE0A5F1080081B204F1080002F0E4
:108490006FFA24E0A5F1080081B204F1080009F0A8
:1084A00023FB1CE0A5F1080081B204F1080008F0EC
:1084B000BDFF14E0A5F1080081B204F1080009F045
:1084C00017F90CE0A5F1080081B204F1080009F0E9
:1084D00023FA04E0E079012100F048F800BF00BF72
:1084E00000BF92E7600000205C000020F0B5ADF214
:1084F000044D05460E4600240027194802782146FF
:10850000641C01A8425445F080022146641C425478
:108510002146641C46542146FBF772FF074621465C
:10852000641C01A847543A122146641C42540D4869
:10853000008AA04201DB204601E00A48008A09497E
:1085400048824A8AC86801A9F8F73CF80548428A77
:10855000C168054808F06AFE0DF2044DF0BD000048
:108560005C00002058060020C802002070B5ADF560
:10857000806D05460E460024244802782146641C7E
:108580000DF8012042782146641C0DF80120827804
:108590002146641C0DF80120C2782146641C0DF8A8
:1085A000012000222146641C0DF8012003222146EF
:1085B000641C0DF80120164802782146641C0DF851
:1085C000012045F080022046611CCCB20DF800204D
:1085D0002046611CCCB20DF80060FF2C01DC204667
:1085E00000E0FF200B4908800846028869460A48D7
:1085F000F7F7E8FF012307480288074907480068A2
:1086000008F07CF80DF5806D70BD00006000002062
:108610005C0000205601002080A3002038010020CB
:108620002DE9F041002412480568C488022C01DAC3
:10863000BDE8F081002003E0295C0E4A1154401C83
:10864000A042F9DBA01E295C601E285C41EA0027DD
:10865000A01E81B22846FBF7D3FE0646B74200D0E3
:10866000E6E7034AD1881068FFF76AFE00BFDFE73C
:1086700058060020BE14002070B50024054D0648A1
:108680000488022C00DA70BD21462846FFF7B6FEAA
:1086900000BFF8E7809900204C0100202DE9F0414F
:1086A0000446DDF818C0079D0898002C04D0002D62
:1086B0000CD0002914D014E03EA340F227124AA1A6
:1086C00050A0F7F78FFE0020BDE8F08139A34FF4EA
:1086D000947256A14BA0F7F785FE0020BDE8F0810B
:1086E0005B4902B95A4A03B9594B4FF00008C4F824
:1086F0000480C4F80880C4F80C80564E6661A4F863
:10870000288084F83180C4F81C80C4F82080C4F824
:1087100024C0514F97F800C084F834C0206120462F
:1087200000F0A0FA2046A84710B10020BDE8F08173
:1087300094F83400FF2801D184F834800026BD6805
:10874000002D21D0A54206D11AA340F28B1243A1DD
:108750002CA0F7F747FE761CFF2E06DD15A340F28E
:108760008D1243A127A0F7F73DFE95F8340094F849
:108770003410884205D194F83400401C84F8340049
:1087800002E02D68002DDDD1002DD1D194F8340008
:10879000FE280CD0401C3870B8682060BC600022F5
:1087A0000121204600F09EF92046BDE8F08187F8BF
:1087B0000080F1E72E2E2F4D6964646C657761723D
:1087C00065732F54686972645F50617274792F4CBD
:1087D0007749502F7372632F636F72652F6E6574C4
:1087E00069662E63000000006E657469665F6164EF
:1087F000643A20696E76616C6964206E657469669E
:1088000000000000417373657274696F6E20222549
:108810007322206661696C6564206174206C696EE6
:108820006520256420696E2025730A006E657469D1
:10883000665F6164643A204E6F20696E69742066D9
:10884000756E6374696F6E20676976656E000000EF
:10885000181D01085D8C0008C80000206E65746951
:108860006620616C7265616479206164646564008E
:10887000746F6F206D616E79206E65746966732CFC
:10888000206D61782E20737570706F72746564202E
:108890006E756D6265722069732032353500000097
:1088A00004F070B970B504460D4616462868E168B4
:1088B000884210D036B909A34FF4147214A118A03D
:1088C000F7F790FDE06830601DB12868E060012096
:1088D00070BD0020FAE7002070BD00002E2E2F4D45
:1088E0006964646C6577617265732F54686972643A
:1088F0005F50617274792F4C7749502F7372632FD8
:10890000636F72652F6E657469662E6300000000E8
:10891000696E76616C696420706F696E746572004F
:10892000417373657274696F6E202225732220660D
:1089300061696C6564206174206C696E65202564D2
:1089400020696E2025730A00F8B505460C461646C8
:10895000002C06D114A340F2CB1220A123A0F7F7DC
:1089600041FD36B910A34FF4E6721CA11FA0F7F722
:1089700039FD20686968884214D0009031606946EA
:108980003046FFF78DFF5CB1206868600121284602
:1089900000F000F9E96909B1284688470120F8BDCF
:1089A0000020F2E70020F8BD2E2E2F4D6964646C84
:1089B0006577617265732F54686972645F50617284
:1089C00074792F4C7749502F7372632F636F7265E0
:1089D0002F6E657469662E6300000000696E766113
:1089E0006C696420706F696E7465720041737365A1
:1089F0007274696F6E2022257322206661696C652E
:108A000064206174206C696E6520256420696E2085
:108A100025730A0070B504460D4616462868A168FD
:108A2000884210D036B909A34FF4047214A118A0DB
:108A3000F7F7D8FCA06830601DB12868A06001205D
:108A400070BD0020FAE7002070BD00002E2E2F4DD3
:108A50006964646C6577617265732F5468697264C8
:108A60005F50617274792F4C7749502F7372632F66
:108A7000636F72652F6E657469662E630000000077
:108A8000696E76616C696420706F696E74657200DE
:108A9000417373657274696F6E202225732220669C
:108AA00061696C6564206174206C696E6520256461
:108AB00020696E2025730A00014600290BD0074863
:108AC000806840B190F83420521CD2B28A4203D060
:108AD00000680028F6D1002070470000C800002080
:108AE000704700002DE9F04105460E4617460B4839
:108AF0004468002D06D10AA340F2FC6215A11BA018
:108B0000F7F770FC002C07D023683A463146284618
:108B100098476468002CF7D1BDE8F081C8000020B8
:108B20002E2E2F4D6964646C6577617265732F54C6
:108B3000686972645F50617274792F4C7749502F65
:108B40007372632F636F72652F6E657469662E632F
:108B5000000000006E65746966206D757374206294
:108B60006520213D204E554C4C000000417373653B
:108B70007274696F6E2022257322206661696C65AC
:108B800064206174206C696E6520256420696E2004
:108B900025730A0070B504460D46002C06D10FA3BC
:108BA00040F26D321AA123A0F7F71CFC94F83100B3
:108BB00010F0040F11D010F0010F0ED015F0010FBE
:108BC0000BD06168002908D010F0080F05D0211DD6
:108BD0002046BDE87040FDF7FFB870BD2E2E2F4D2A
:108BE0006964646C6577617265732F546869726437
:108BF0005F50617274792F4C7749502F7372632FD5
:108C0000636F72652F6E657469662E6300000000E5
:108C10006E657469665F69737375655F7265706FA1
:108C20007274733A20696E76616C6964206E657443
:108C300069660000417373657274696F6E20222546
:108C40007322206661696C6564206174206C696EB2
:108C50006520256420696E2025730A006FF00B00E3
:108C6000704700002DE9FF4F87B00D461746984624
:108C700000240DF10C090DF1080A002D00D1224D40
:108C800007B9214FB8F1000F01D1DFF87C8025B37F
:108C9000286810B300260DF1040B46B101AA29463D
:108CA0000798FFF751FE10B11024CDF810B04A46D6
:108CB00039460798FFF7AEFE18B144F04004CDF8EE
:108CC0001490524641460798FFF7ECFD18B144F066
:108CD0002004CDF818A016B10BE00126DBE701AAAD
:108CE00029460798FFF730FE18B144F01004CDF87C
:108CF00010B0002C05D044F0800104AA0798FFF7BB
:108D0000F1FE0BB0BDE8F08F181D01080149C860E5
:108D100070470000C800002010B584B00446002C45
:108D200020D094F8310010F0010F25D000208DF8EC
:108D3000040001AA08212046FFF7D4FE94F8310070
:108D400000F0FE0084F8310010F0080F02D0204639
:108D5000FCF71CFBE16900290ED004B02046BDE8F9
:108D60001040084704B005A3BDE8104040F29B3214
:108D70000FA117A0F7F736BB04B010BD2E2E2F4D54
:108D80006964646C6577617265732F546869726495
:108D90005F50617274792F4C7749502F7372632F33
:108DA000636F72652F6E657469662E630000000044
:108DB0006E657469665F7365745F646F776E3A2081
:108DC000696E76616C6964206E6574696600000086
:108DD000417373657274696F6E2022257322206659
:108DE00061696C6564206174206C696E652025641E
:108DF00020696E2025730A00002800D001627047A8
:108E000010B584B00446002C16D094F8310010F050
:108E1000040F0FD000F0FB0084F83100216A09B183
:108E20002046884700208DF8040001AA042120462E
:108E3000FFF758FE04B010BD04B004A3BDE8104015
:108E400040F206420EA117A0F7F7CCBA2E2E2F4DF6
:108E50006964646C6577617265732F5468697264C4
:108E60005F50617274792F4C7749502F7372632F62
:108E7000636F72652F6E657469662E630000000073
:108E80006E657469665F7365745F6C696E6B5F6451
:108E90006F776E3A20696E76616C6964206E6574D6
:108EA00069660000417373657274696F6E202225D4
:108EB0007322206661696C6564206174206C696E40
:108EC0006520256420696E2025730A0010B584B0E2
:108ED0000446002C1AD094F8310010F0040F13D17E
:108EE00040F0040084F8310003212046FFF752FED1
:108EF000216A09B12046884701208DF8040001AAA3
:108F000004212046FFF7EEFD04B010BD04B004A319
:108F1000BDE810404FF478720EA117A0F7F762BABF
:108F20002E2E2F4D6964646C6577617265732F54C2
:108F3000686972645F50617274792F4C7749502F61
:108F40007372632F636F72652F6E657469662E632B
:108F5000000000006E657469665F7365745F6C691C
:108F60006E6B5F75703A20696E76616C6964206E15
:108F70006574696600000000417373657274696FFF
:108F80006E2022257322206661696C6564206174FD
:108F9000206C696E6520256420696E2025730A00A7
:108FA00010B584B00446002C1BD094F8310010F0AA
:108FB000010F20D140F0010084F83100E16909B1CE
:108FC0002046884701208DF8040001AA0821204688
:108FD000FFF788FD04B02046BDE810400321FFF7ED
:108FE000D9BD04B005A3BDE810404FF4547210A1E0
:108FF00016A0F7F7F7B904B010BD00002E2E2F4DC4
:109000006964646C6577617265732F546869726412
:109010005F50617274792F4C7749502F7372632FB0
:10902000636F72652F6E657469662E6300000000C1
:109030006E657469665F7365745F75703A20696EFA
:1090400076616C6964206E6574696600417373654E
:109050007274696F6E2022257322206661696C65C7
:1090600064206174206C696E6520256420696E201F
:1090700025730A00002200F001B8000070B5044614
:109080000D461646002C06D117A340F2DF1222A18E
:1090900024A0F7F7A7F914B1B5F5803F01D301205B
:1090A00070BD3DB1A8B2218901448BB2834203D285
:1090B000012070BD002070BD217B11F0800F07D012
:1090C0006168491B04F11002914204D2012070BD75
:1090D00046B16168491B61606189084460812381F0
:1090E000002070BD012070BD2E2E2F4D6964646C70
:1090F0006577617265732F54686972645F5061723D
:1091000074792F4C7749502F7372632F636F726598
:109110002F706275662E63007020213D204E554CE5
:109120004C000000417373657274696F6E202225D4
:109130007322206661696C6564206174206C696EBD
:109140006520256420696E2025730A002DE9F04F03
:1091500083B007460D469246BAF1010F15D0BAF119
:10916000410F12D00024BAF5C17F16D0BAF5207F86
:1091700000F05F804BA340F2271256A15CA0F7F7E6
:1091800031F903B00020BDE8F08F52462946002097
:1091900000F00AF9064600F07CB80026B146072028
:1091A000FFF732F80446200025D0F81C20F0030B0E
:1091B000CBF514701FFA80F8A84500D9A846002006
:1091C0000190E019133020F00301CDF800A04346D0
:1091D0002A46204600F0C8FC207910F0030F06D084
:1091E00030A34FF480724CA141A0F7F7FBF8BBF518
:1091F000147F0AD010E000F0C9FC16B1304600F030
:10920000D5FB03B00020BDE8F08F26A34FF4817298
:109210004DA137A0F7F7E6F84EB1C9F80040A146D6
:10922000A5EB080085B20027002DB8D131E0264615
:10923000F5E7F81CE91C20F0030021F003010844C5
:1092400080B200F1100292B2814201D8914203D95A
:1092500003B00020BDE8F08F1046FEF7D9FC0646AB
:1092600030001AD0F019133020F003012B462A46A3
:109270003046CDF800A0019400F076FC307910F073
:10928000030F06D007A34FF491723CA118A0F7F783
:10929000A9F803B03046BDE8F08F03B00020BDE868
:1092A000F08F00002E2E2F4D6964646C657761721B
:1092B00065732F54686972645F50617274792F4CC2
:1092C0007749502F7372632F636F72652F706275C9
:1092D000662E6300706275665F616C6C6F633A2026
:1092E0006572726F6E656F757320747970650000BA
:1092F000417373657274696F6E2022257322206634
:1093000061696C6564206174206C696E65202564F8
:1093100020696E2025730A00706275665F616C6C4F
:109320006F633A207062756620712D3E7061796CB2
:109330006F61642070726F7065726C7920616C6906
:10934000676E656400000000504255465F504F4F05
:109350004C5F42554653495A45206D7573742062DF
:109360006520626967676572207468616E204D458B
:109370004D5F414C49474E4D454E540070627566F5
:109380005F616C6C6F633A20706275662D3E706130
:10939000796C6F61642070726F7065726C79206196
:1093A0006C69676E65640000F0B583B006460D46D3
:1093B0001446412C08D0012C06D00EA34FF4A57200
:1093C00018A11DA0F7F70EF80620FEF71DFF0746AF
:1093D00038000BD0002001902B462A4631460094DD
:1093E000384600F0C1FB03B03846F0BD03B00020A2
:1093F000F0BD00002E2E2F4D6964646C657761729C
:1094000065732F54686972645F50617274792F4C70
:109410007749502F7372632F636F72652F70627577
:10942000662E6300696E76616C6964207062756691
:109430005F74797065000000417373657274696FC1
:109440006E2022257322206661696C656420617438
:10945000206C696E6520256420696E2025730A00E2
:1094600030B583B084461C46079B06980D460CF128
:10947000030121F0030101EB050C9C4502D903B067
:10948000002030BD08B1014400E00021022000921C
:1094900001902B462A46204600F066FB03B020468A
:1094A00030BD000070B50D46002826D0002D24D018
:1094B0000446206838B1208929890844208124681D
:1094C00020680028F7D120896189884206D00FA33F
:1094D00040F2623219A125A0F6F784FF206830B16E
:1094E0000AA340F263322BA120A0F6F77BFF20896C
:1094F000298908442081256070BDBDE8704003A320
:1095000040F2593227A119A0F6F76CBF2E2E2F4D2D
:109510006964646C6577617265732F5468697264FD
:109520005F50617274792F4C7749502F7372632F9B
:10953000636F72652F706275662E6300702D3E74C6
:109540006F745F6C656E203D3D20702D3E6C656EC6
:1095500020286F66206C61737420706275662069C4
:109560006E20636861696E290000000041737365B5
:109570007274696F6E2022257322206661696C65A2
:1095800064206174206C696E6520256420696E20FA
:1095900025730A00702D3E6E657874203D3D204E87
:1095A000554C4C00286820213D204E554C4C29201C
:1095B000262620287420213D204E554C4C29202859
:1095C00070726F6772616D6D65722076696F6C6124
:1095D00074657320415049290000000000210028D3
:1095E00004D0491C89B200680028FAD108467047A7
:1095F00070B50B4614461A462189FFF7A7FD0546AC
:1096000028000CD0214600F043F830B105A340F209
:10961000245210A114A0F6F7E5FE284670BD0020E4
:1096200070BD00002E2E2F4D6964646C65776172E9
:1096300065732F54686972645F50617274792F4C3E
:109640007749502F7372632F636F72652F70627545
:10965000662E6300706275665F636F707920666165
:10966000696C656400000000417373657274696F12
:109670006E2022257322206661696C656420617406
:10968000206C696E6520256420696E2025730A00B0
:109690002DE9F04105460C4600260027002D04D098
:1096A0001CB12889218988420AD238A340F2C932E4
:1096B00042A14EA0F6F796FE6FF00F00BDE8F081D4
:1096C00068896189801BA1EB0708404500D280466C
:1096D00060684246C11968683044F6F773FF464433
:1096E00047446889B04206D228A340F2D93249A142
:1096F0003EA0F6F777FE6089B84206D223A340F277
:10970000DA324AA139A0F6F76DFE6089B84201D875
:10971000002724686889B0420ED100262D685DB903
:1097200054B11AA34FF4797247A130A0F6F75AFE4C
:109730006FF00F00BDE8F081002C10D06089218906
:1097400088420CD1206850B110A340F2E93242A106
:1097500026A0F6F747FE6FF00500BDE8F08185B161
:109760006889298988420CD1286850B107A340F242
:10977000EE3239A11DA0F6F735FE6FF00500BDE809
:10978000F081002C9CD10020BDE8F0812E2E2F4DC1
:109790006964646C6577617265732F54686972647B
:1097A0005F50617274792F4C7749502F7372632F19
:1097B000636F72652F706275662E630070627566E6
:1097C0005F636F70793A20746172676574206E6FA1
:1097D000742062696720656E6F75676820746F20FA
:1097E000686F6C6420736F75726365004173736595
:1097F0007274696F6E2022257322206661696C6520
:1098000064206174206C696E6520256420696E2077
:1098100025730A006F66667365745F746F203C3D44
:1098200020705F746F2D3E6C656E00006F6666730E
:1098300065745F66726F6D203C3D20705F66726F6D
:109840006D2D3E6C656E0000705F746F20213D20B1
:109850004E554C4C00000000706275665F636F707F
:1098600079282920646F6573206E6F7420616C6C99
:109870006F77207061636B657420717565756573B2
:10988000210000002DE9F047894616460027B8461A
:10989000002804D0B9F1000F0BD0044631E01CA31E
:1098A00040F20A4226A12EA0F6F79CFD0020BDE85A
:1098B000F08717A340F20B4233A129A0F6F792FDDF
:1098C0000020BDE8F0872BB16089984202D8181AB1
:1098D00083B215E06089C01A85B2B54200D9354619
:1098E00060682A46C11809EB0700F6F76BFE08EB23
:1098F00005001FFA80F8781987B2701B86B2002322
:1099000024680EB1002CDED14046BDE8F08700008F
:109910002E2E2F4D6964646C6577617265732F54C8
:10992000686972645F50617274792F4C7749502F67
:109930007372632F636F72652F706275662E63009A
:10994000706275665F636F70795F70617274696170
:109950006C3A20696E76616C6964206275660000FD
:10996000417373657274696F6E20222573222066BD
:1099700061696C6564206174206C696E6520256482
:1099800020696E2025730A00706275665F636F70D0
:10999000795F7061727469616C3A20696E76616C8E
:1099A00069642064617461707472000070B504466B
:1099B000002C03D00025A07B48B10FE026A34FF474
:1099C000377231A133A0F6F70DFD002070BD22A340
:1099D00040F2F12239A12FA0F6F704FDA07B401E32
:1099E000C0B2A07320B10024002CE4D1284670BD81
:1099F0002668207B00F00F00617B11F0020F0CD075
:109A0000206930B914A340F2FF2232A121A0F6F759
:109A1000E9FC2169204688470BE002280DD0012887
:109A200010D0A0B10CA340F20F3233A119A0F6F769
:109A3000D9FC681CC5B23446D6E721460720FEF79C
:109A400021FBF6E721460620FEF71CFBF1E7204646
:109A5000FDF7D6FFEDE700002E2E2F4D6964646CF4
:109A60006577617265732F54686972645F506172C3
:109A700074792F4C7749502F7372632F636F72651F
:109A80002F706275662E63007020213D204E554C6C
:109A90004C000000417373657274696F6E2022255B
:109AA0007322206661696C6564206174206C696E44
:109AB0006520256420696E2025730A007062756632
:109AC0005F667265653A20702D3E726566203E20A5
:109AD0003000000070632D3E637573746F6D5F66B8
:109AE0007265655F66756E6374696F6E20213D20D7
:109AF0004E554C4C00000000696E76616C69642024
:109B000070627566207479706500000010B50146BA
:109B10000448FEF705FB04480178012901D1002122
:109B2000017010BD141C01086400002007490020CA
:109B3000087007480068002806D0416F09B102F09C
:109B40001DB9C0680028F8D170470000D800002077
:109B5000F40000200122AFF30080002902DA49421C
:109B600000F0FCB8FFF78ABA30B4DDF808C0039CF7
:109B70000025056041600281438180F80CC0447378
:109B800001218173C57330BC704700000149012079
:109B900008707047D800002070B504460D46002CB0
:109BA00006D122A34FF4CC722CA132A0F6F71AFCF6
:109BB0002089A84239D9401B86B26089A84211D2B7
:109BC0006089281A85B22089801B2081246834B9D5
:109BD00016A340F2AF1231A126A0F6F703FC60896C
:109BE000A842EDD3207B10F00F0F16D16089A84258
:109BF00013D0607B10F0020F0FD1A088001B284407
:109C000081B22046FEF73EF9044634B907A340F27C
:109C1000BD1228A117A0F6F7E5FB65812581206814
:109C200008B1FFF7C3FE0020206070BD2E2E2F4D1F
:109C30006964646C6577617265732F5468697264D6
:109C40005F50617274792F4C7749502F7372632F74
:109C5000636F72652F706275662E63007062756641
:109C60005F7265616C6C6F633A207020213D204EFD
:109C7000554C4C00417373657274696F6E202225D8
:109C80007322206661696C6564206174206C696E62
:109C90006520256420696E2025730A007062756650
:109CA0005F7265616C6C6F633A207120213D204EBC
:109CB000554C4C006D656D5F7472696D20726574F2
:109CC00075726E65642071203D3D204E554C4C00F0
:109CD00000280CD0817B491CC9B28173002906D1B0
:109CE00003A340F242320EA112A0F6F77BBB7047ED
:109CF0002E2E2F4D6964646C6577617265732F54E5
:109D0000686972645F50617274792F4C7749502F83
:109D10007372632F636F72652F706275662E6300B6
:109D20007062756620726566206F766572666C6F0C
:109D300077000000417373657274696F6E2022258D
:109D40007322206661696C6564206174206C696EA1
:109D50006520256420696E2025730A0070B50446CD
:109D60000D46002C06D114A340F24B221EA121A0C7
:109D7000F6F738FB14B1B5F5803F01D3012070BD73
:109D8000002D0CD0A8B2618981420AD20AA340F208
:109D9000552222A117A0F6F725FB012070BD002057
:109DA00070BD62682A446260091A61812189081ABB
:109DB0002081002070BD00002E2E2F4D6964646C40
:109DC0006577617265732F54686972645F50617260
:109DD00074792F4C7749502F7372632F636F7265BC
:109DE0002F706275662E63007020213D204E554C09
:109DF0004C000000417373657274696F6E202225F8
:109E00007322206661696C6564206174206C696EE0
:109E10006520256420696E2025730A00696E6372CF
:109E2000656D656E745F6D61676E697475646520DC
:109E30003C3D20702D3E6C656E0000002DE9F04128
:109E40000446314E3068844206D230A340F2DF121D
:109E50003AA140A0F6F7C6FA7068844206D32BA355
:109E60004FF4F07245A13BA0F6F7BCFA2079002828
:109E700006D026A340F2E11247A136A0F6F7B2FAC7
:109E80002088B0F5C86F06D920A34FF4F27249A11B
:109E900030A0F6F7A7FA208800F0A2F80546AC42F9
:109EA00016D02879A0B97068854211D0B068A84250
:109EB00000D1B460288820802888B0F5C86F07D00A
:109EC0002046FDF7D7FF0746288800F089F847802D
:109ED000608800F085F8A04213D00179002910D1E4
:109EE000B168A14200D1B060218801802188B1F51C
:109EF000C86F06D0FDF7BEFF0546208800F070F859
:109F00004580BDE8F08100009C0000202E2E2F4DE2
:109F10006964646C6577617265732F5468697264F3
:109F20005F50617274792F4C7749502F7372632F91
:109F3000636F72652F6D656D2E630000706C7567C1
:109F40005F686F6C65733A206D656D203E3D2072D1
:109F5000616D0000417373657274696F6E20222514
:109F60007322206661696C6564206174206C696E7F
:109F70006520256420696E2025730A00706C756762
:109F80005F686F6C65733A206D656D203C2072616F
:109F90006D5F656E64000000706C75675F686F6C64
:109FA00065733A206D656D2D3E75736564203D3D8A
:109FB00020300000706C75675F686F6C65733A20C5
:109FC0006D656D2D3E6E657874203C3D204D454D90
:109FD0005F53495A455F414C49474E454400000094
:109FE00001490968084470479C0000202DE9F04FA2
:109FF000ADF2144D054600240020CDF804044FF4C2
:10A00000806101A8F6F723FB6878297840EA0129E6
:10A01000E878A97840EA0126012E01DA502E72DC98
:10A02000B9F15F0F70DC06EB09006028FADCF01D67
:10A03000C11700EB5171C1F3C701CDF810144348AB
:10A0400002782146601CC4B201A842540122214674
:10A05000601CC4B201A842542046621CD4B201AABA
:10A06000DDF8101411540027BB462FE0002001A991
:10A07000085582461BE009EB070188B20DF20C413E
:10A08000F7F732F801A8005D9DF80C1401FA0AF107
:10A09000084301A90855781C87B2B74203DB0120A9
:10A0A000CDF8040406E00AF1010000F0FF0ABAF15D
:10A0B000080FE0DB00BF601CC4B2DDF80404012817
:10A0C00000D107E00BF1010000F0FF0BDDF81004F8
:10A0D0008345CBDB00BF214601A8FAF791F9804602
:10A0E0002046611CCCB201A901F800804FEA282269
:10A0F0002046611CCCB201A90A541548008AA0422E
:10A1000003DB204603E017E012E01148008A104903
:10A1100048824A8AC86801A9F6F754FA0C48428A6C
:10A12000C1680C4807F082F80DF2144DBDE8F08FBD
:10A130000220CDF8080402E00320CDF80804012035
:10A14000DDF80814FEF7D2F900BFEDE75C0000204F
:10A1500058060020C80200202DE9F04FADF20C4D4A
:10A16000054600240020CDF800044FF480616846C5
:10A17000F6F76DFA6878297840EA0129E878A97835
:10A1800040EA0126012E01DA502E7CDCB9F15F0F86
:10A190007ADC06EB09006028FADCF01DC11700EB41
:10A1A0005171C1F3C707504802782146601CC4B200
:10A1B0000DF801204C4842782146601CC4B20DF8CD
:10A1C0000120494882782046611CCCB20DF800205D
:10A1D0004548C2782046611CCCB20DF80020F81C1E
:10A1E00002122046611CCCB20DF80020F81CC2B24D
:10A1F0002046611CCCB20DF800203C480278204675
:10A20000611CCCB20DF8002001222046611CCCB2AA
:10A210000DF800202046611CCCB20DF800704FF004
:10A2200000084FF0000B34E000200DF804008246D7
:10A230001EE009EB080188B20DF58161F6F754FFC5
:10A240001DF804009DF8081401FA0AF10843C0B291
:10A250000DF8040008F101001FFA80F8B04503DB97
:10A260000120CDF8000406E00AF1010000F0FF0A29
:10A27000BAF1080FDDDB00BF601CC4B2DDF80004DA
:10A28000012802D107E024E01FE00BF1010000F0FB
:10A29000FF0BBB45C8DB00BFFF2C01DC204600E004
:10A2A000FF20134908800846028869461148F6F7DE
:10A2B00089F901230E4802880E490F48006806F00C
:10A2C0001DFA0DF20C4DBDE8F08F0220CDF804040C
:10A2D00002E00320CDF804040120DDF80414FEF7A9
:10A2E00045F900BFEDE70000600000205C000020A1
:10A2F0005601002080A30020380100202DE9F04FF6
:10A30000ADF2144D054600240020CDF80404687811
:10A31000297840EA0129E878A97840EA0126012E47
:10A3200001DA602E72DCB9F15F0F70DC06EB090018
:10A330006028FADCF01DC11700EB5171C1F3C701B1
:10A34000CDF81014434802782146601CC4B201A81D
:10A35000425402222146601CC4B201A84254204645
:10A36000621CD4B201AADDF8101411540027BB46B8
:10A370002FE0002001A9085582461BE009EB0701E8
:10A3800088B20DF20C41F6F7CBFE01A8005D9DF8F6
:10A390000C1401FA0AF1084301A90855781C87B288
:10A3A000B74203DB0120CDF8040406E00AF1010006
:10A3B00000F0FF0ABAF1080FE0DB00BF601CC4B276
:10A3C000DDF80404012800D107E00BF1010000F0E2
:10A3D000FF0BDDF810048345CBDB00BF214601A84D
:10A3E000FAF70EF880462046611CCCB201A901F8AC
:10A3F00000804FEA28222046611CCCB201A90A54F1
:10A400001548008AA04203DB204603E017E012E073
:10A410001148008A104948824A8AC86801A9F6F79B
:10A42000D1F80D48428AC1680C4806F0FFFE0DF2D3
:10A43000144DBDE8F08F0220CDF8080402E003209F
:10A44000CDF808040220DDF80814FEF74FF800BF2D
:10A45000EDE700005C00002058060020C802002044
:10A460002DE9F04FADF20C4D054600240020CDF84B
:10A4700000046878297840EA0129E878A97840EA58
:10A480000126012E01DA602E7CDCB9F15F0F7ADC47
:10A4900006EB09006028FADCF01DC11700EB5171D2
:10A4A000C1F3C7074F4802782146601CC4B20DF8BB
:10A4B00001204C4842782146601CC4B20DF80120AE
:10A4C000484882782046611CCCB20DF800204548EF
:10A4D000C2782046611CCCB20DF80020F81C021294
:10A4E0002046611CCCB20DF80020F81CC2B22046F8
:10A4F000611CCCB20DF800203B4802782046611C5C
:10A50000CCB20DF8002002222046611CCCB20DF81E
:10A5100000202046611CCCB20DF800704FF00008FE
:10A520004FF0000B34E000200DF8040082461EE0DE
:10A5300009EB080188B20DF58161F6F7F1FD1DF810
:10A5400004009DF8081401FA0AF10843C0B20DF89E
:10A55000040008F101001FFA80F8B04503DB012078
:10A56000CDF8000406E00AF1010000F0FF0ABAF19C
:10A57000080FDDDB00BF601CC4B2DDF80004012859
:10A5800002D107E024E01FE00BF1010000F0FF0B17
:10A59000BB45C8DB00BFFF2C01DC204600E0FF20EC
:10A5A000124908800846028869461148F6F70AF8F9
:10A5B00001230E4802880E490E48006806F09EF8F6
:10A5C0000DF20C4DBDE8F08F0220CDF8040402E03E
:10A5D0000320CDF804040220DDF80414FDF7C6FFC3
:10A5E00000BFEDE7600000205C0000205601002065
:10A5F00080A30020380100202DE9F04FADF2044D7A
:10A60000064600241EB90DF2044DBDE8F08F7078A7
:10A61000317840EA0127F078B17840EA0125012D30
:10A6200064DB602D62DC5F2F5DDC781900285ADB6B
:10A630007819602857DC314802782046611CCCB27A
:10A6400001A90A5403222046611CCCB201A90A5474
:10A650006806020E2046611CCCB201A90A544FF0D4
:10A66000000816E007EB080188B2F6F729FD8146DD
:10A670004FEA29222146601CC4B201A84254204658
:10A68000611CCCB201A901F8009008F101001FFA89
:10A6900080F8A845E6DB214601A8F9F7B1FE82461D
:10A6A0002046611CCCB201A901F800A04FEA2A2281
:10A6B0002046611CCCB201A90A541148008AA0426C
:10A6C00001DB204601E00E48008A0D4948824A8A93
:10A6D000C86801A9F5F776FF0948428AC1680948A8
:10A6E00006F0A4FD8FE74FF0020B01E04FF0030BE3
:10A6F00059460320FDF7FAFE00BF84E75C00002006
:10A7000058060020C80200202DE9F04FADF2044D9C
:10A7100006468A4600241EB90DF2044DBDE8F08FAE
:10A720007078317840EA0127F078B17840EA012565
:10A73000012D6EDB602D6CDC5F2F7EDC781900282C
:10A740007BDB7819602878DC414802782046611C60
:10A75000CCB201A90A543E4842782046611CCCB2D2
:10A7600001A90A543A4882782046611CCCB201A95A
:10A770000A543748C2782046611CCCB201A90A5459
:10A78000022000EB4500401CC0F307222046611C5C
:10A79000CCB201A90A54022000EB4500401CC2B211
:10A7A0002046611CCCB201A90A542A4802782046EE
:10A7B000611CCCB201A90A5403222046611CCCB210
:10A7C00001A90A546806020E2046611CCCB201A9F8
:10A7D0000A544FF0000816E007EB080188B2F6F7BC
:10A7E0006FFC81464FEA29222046611CCCB201A9A8
:10A7F0000A542046611CCCB201A901F8009008F16E
:10A8000001001FFA80F8A845E6DBFF2C03DC204698
:10A8100002E015E011E0FF200F4908800846028899
:10A8200001A90E48F5F7CEFE01230B4802880B491B
:10A830000B48006805F062FF6EE74FF0020B01E085
:10A840004FF0030B59460320FDF790FE00BF63E76E
:10A85000600000205C0000205601002080A3002042
:10A86000380100202DE9F04FADF2044D05460024DB
:10A870001DB90DF2044DBDE8F08F6878297840EAE3
:10A880000127E878A97840EA0126012E61DB602ED5
:10A890005FDC5F2F5ADCB819602857DC314802783A
:10A8A0002046611CCCB201A90A5404222046611C36
:10A8B000CCB201A90A547006020E2046611CCCB22B
:10A8C00001A90A544FF0000816E007EB080188B20E
:10A8D000F6F700FC81464FEA29222046611CCCB2E3
:10A8E00001A90A542046611CCCB201A901F80090CC
:10A8F00008F101001FFA80F8B045E6DB214601A807
:10A90000F9F77EFD82462046611CCCB201A901F810
:10A9100000A04FEA2A222046611CCCB201A90A54A9
:10A920001148008AA04201DB204601E00E48008A5F
:10A930000D4948824A8AC86801A9F5F743FE0A48CA
:10A94000428AC168094806F071FC92E74FF0020B99
:10A9500001E04FF0030B59460420FDF7C7FD00BF8F
:10A9600087E700005C00002058060020C802002095
:10A970002DE9F04FADF2044D06468A4600241EB97B
:10A980000DF2044DBDE8F08F7078317840EA012770
:10A99000F078B17840EA0125012D7DDB602D7BDC6C
:10A9A0005F2F7BDC7819602878DC424802782046EB
:10A9B000611CCCB201A90A543E4842782046611C71
:10A9C000CCB201A90A543B4882782046611CCCB223
:10A9D00001A90A543748C2782046611CCCB201A9AB
:10A9E0000A54022000EB4500401CC0F30722204619
:10A9F000611CCCB201A90A54022000EB4500401CA6
:10AA0000C2B22046611CCCB201A90A542A4802787D
:10AA10002046611CCCB201A90A5404222046611CC4
:10AA2000CCB201A90A546806020E2046611CCCB2C1
:10AA300001A90A544FF0000816E007EB080188B29C
:10AA4000F6F748FB81464FEA29222046611CCCB22A
:10AA500001A90A542046611CCCB201A901F800905A
:10AA600008F101001FFA80F8A845E6DBFF2C01DCA5
:10AA7000204600E0FF20114908800846028801A90D
:10AA80000F48F5F79FFD01230C4802880C490D483B
:10AA9000006805F033FE73E703E0FFE74FF0020BB9
:10AAA00001E04FF0030B59460420FDF75FFD00BFA6
:10AAB00066E70000600000205C00002056010020D6
:10AAC00080A30020380100207047000010B501224B
:10AAD00002210948F7F772FA012204210648F7F724
:10AAE0006DFA012208210448F7F768FA01221021C3
:10AAF0000148F7F763FA10BD0010024010B5044694
:10AB0000012C06D0022C19D0032C2CD0042C54D1AB
:10AB10003EE0002202212A48F7F750FA01220421E0
:10AB20002748F7F74BFA012208212548F7F746FA9C
:10AB3000012210212248F7F741FA3EE001220221CA
:10AB40001F48F7F73BFA002204211D48F7F736FAB1
:10AB5000012208211A48F7F731FA0122102118487A
:10AB6000F7F72CFA29E0012202211548F7F726FA17
:10AB7000012204211248F7F721FA00220821104887
:10AB8000F7F71CFA012210210D48F7F717FA14E025
:10AB9000012202210A48F7F711FA0122042108488C
:10ABA000F7F70CFA012208210548F7F707FA002207
:10ABB00010210348F7F702FA00BF00BF10BD0000E4
:10ABC000001002402DE9F04100F024F806460F4F36
:10ABD0000F4D387808B1FEF7A9FF2968002912D077
:10ABE0004A68B01AB0F1004F0DD2086828608C682E
:10ABF000D1F80C806A600520FDF744FA002CE8D0FB
:10AC00004046A047E5E7BDE8F0810000D8000020FD
:10AC100020010020F7F7D8B970B504460D46164656
:10AC2000B4F1804F06D308A340F2291213A121A04A
:10AC3000F5F7D8FBFFF7EEFF204432462946BDE882
:10AC4000704000F04BB800002E2E2F4D6964646CEC
:10AC50006577617265732F54686972645F506172C1
:10AC600074792F4C7749502F7372632F636F72651D
:10AC70002F74696D656F7574732E630054696D650B
:10AC80006F75742074696D6520746F6F206C6F6EC2
:10AC9000672C206D6178206973204C5749505F55AF
:10ACA000494E5433325F4D41582F34206D736563E4
:10ACB00073000000417373657274696F6E20222502
:10ACC0007322206661696C6564206174206C696E12
:10ACD0006520256420696E2025730A0070B504463E
:10ACE0000D4616460520FDF78FFA80B1002202605E
:10ACF0008560C6604460114A116800290FD04B6816
:10AD0000E31AB3F1004F0CD30160106070BDBDE8D1
:10AD100070400BA3BE2217A126A0F5F763BB1060FD
:10AD200070BD0A6822B15368E31AB3F1004F03D330
:10AD30000A680260086070BD1146F2E72001002039
:10AD40002E2E2F4D6964646C6577617265732F5484
:10AD5000686972645F50617274792F4C7749502F23
:10AD60007372632F636F72652F74696D656F75748D
:10AD7000732E63007379735F74696D656F75743AD0
:10AD80002074696D656F757420213D204E554C4CC3
:10AD90002C20706F6F6C204D454D505F5359535FA1
:10ADA00054494D454F555420697320656D70747931
:10ADB00000000000417373657274696F6E20222574
:10ADC0007322206661696C6564206174206C696E11
:10ADD0006520256420696E2025730A0070B5012462
:10ADE000054D064905EBC40255F83400FFF714FF82
:10ADF000641C032CF5D370BD001D0108C178000848
:10AE00002DE9F04F85B004468B46002C03D0207D01
:10AE100001280AD010E005B03AA3BDE8F04F40F297
:10AE20003D2244A14AA0F5F7DDBA36A34FF41072D3
:10AE300051A147A0F5F7D6FA207D0A283CD000257D
:10AE40000027216D0491D4F82480D4F89060D4F8C0
:10AE50001090DFF858A1002838D05D46E78A2146D7
:10AE60000AF1180002F06CFE01208AF80000206F41
:10AE700008B104F068FDE06E08B104F064FD606F95
:10AE800008B104F060FD55B1208B211D00910290A6
:10AE90002346424601972046049904F05FFC204671
:10AEA00000F034FE002E29D005B04846B446BDE877
:10AEB000F04F6FF00C01604721463D4802F040FE24
:10AEC00005B02046BDE8F04F00F020BEE08A002823
:10AED000CDD0DAF81000A04203D1C068CAF8100043
:10AEE00009E040B1C168A14202D1E168C16002E05D
:10AEF00008460028F6D10020E060B8E705B0BDE8BC
:10AF0000F08F00002E2E2F4D6964646C657761729E
:10AF100065732F54686972645F50617274792F4C45
:10AF20007749502F7372632F636F72652F7463704C
:10AF30002E6300007463705F6162616E646F6E3ACD
:10AF400020696E76616C69642070636200000000A5
:10AF5000417373657274696F6E20222573222066B7
:10AF600061696C6564206174206C696E652025647C
:10AF700020696E2025730A00646F6E277420636158
:10AF80006C6C207463705F61626F72742F74637095
:10AF90005F6162616E646F6E20666F72206C6973B0
:10AFA00074656E2D7063627300000000DC00002089
:10AFB000F80000200121FFF723BF002803D0027D05
:10AFC000012A00D18161704770B505460C461646CE
:10AFD0000C480068C08A41F29231884209D1094880
:10AFE0000068008B218B884203D006480068FFF779
:10AFF000E1FF044804600449204603F0E5FE002018
:10B0000070BD00003801002045F0000810B50C4666
:10B01000002C06D106A340F20F3211A118A0F5F7BB
:10B02000E1F92046FFF7C6FF6FF00C0010BD0000ED
:10B030002E2E2F4D6964646C6577617265732F5491
:10B04000686972645F50617274792F4C7749502F30
:10B050007372632F636F72652F7463702E630000C9
:10B060007463705F6163636570745F6E756C6C3A76
:10B0700020696E76616C6964207063620000000074
:10B08000417373657274696F6E2022257322206686
:10B0900061696C6564206174206C696E652025644B
:10B0A00020696E2025730A0070B505460020FDF763
:10B0B000ABF80446FCB900F07FFE01F04DFB002028
:10B0C000FDF7A2F80446B4B9092001F0E5FA002022
:10B0D000FDF79AF8044674B9082001F0DDFA002063
:10B0E000FDF792F8044634B9284601F0ADFA002085
:10B0F000FDF78AF804462CB39C212046F5F7A7FA01
:10B1000065754FF48661A4F8641048006085208559
:10B11000FF20E072481060860620A4F84000E08717
:10B12000C01F20860120A4F848000748C268226298
:10B130008078A077A4F84A100448C4F88400044832
:10B14000C4F89400204670BDDC00002099F000088F
:10B1500000DD6D002DE9F04105460C460426002C6B
:10B1600000D1284C002D0DD0287D002815D026A315
:10B1700040F2AB2230A13AA0F5F734F96FF00500A8
:10B18000BDE8F08120A340F2A9223FA134A0F5F749
:10B1900029F96FF00F00BDE8F081AAB14FF0000C63
:10B1A0003F4F57F82C000068C8B1C18A914213D1B3
:10B1B00030B1016821B11CB123680BB199420BD1A8
:10B1C0006FF00700BDE8F08101F06AFD0246100053
:10B1D00009D1801EBDE8F081C0680028E5D10CF1DE
:10B1E000010CB445DDDB14B1206800B12860EA82AF
:10B1F0002C480169E960056105F048F90020BDE8C7
:10B20000F0810000181D01082E2E2F4D6964646C1A
:10B210006577617265732F54686972645F506172FB
:10B2200074792F4C7749502F7372632F636F726557
:10B230002F7463702E6300007463705F62696E64C4
:10B240003A2063616E206F6E6C792062696E6420B3
:10B25000696E20737461746520434C4F53454400FC
:10B26000417373657274696F6E20222573222066A4
:10B2700061696C6564206174206C696E6520256469
:10B2800020696E2025730A007463705F62696E64C2
:10B290003A20696E76616C69642070636200000018
:10B2A000F01C0108DC00002010B500280BD0017D47
:10B2B000012903D0418B41F010014183BDE81040CA
:10B2C000012100F043B805A34FF4F4720FA115A0BB
:10B2D000F5F788F86FF00F0010BD00002E2E2F4DEF
:10B2E0006964646C6577617265732F546869726410
:10B2F0005F50617274792F4C7749502F7372632FAE
:10B30000636F72652F7463702E6300007463705FE7
:10B31000636C6F73653A20696E76616C6964207046
:10B3200063620000417373657274696F6E20222539
:10B330007322206661696C6564206174206C696E9B
:10B340006520256420696E2025730A002DE9F041EF
:10B3500084B004468846002C06D146A34FF4AF7251
:10B3600050A158A0F5F73EF8002501275F4EB8F12F
:10B37000000F44D0207D042801D007283FD1A06FC2
:10B3800018B9208DB0F5066F39D0A07E10F0100FDF
:10B3900006D138A34FF4B27255A14AA0F5F722F8AE
:10B3A000208BE18A221D02900092019123462046C3
:10B3B000626A216D04F0D2F9204602F059FBB069AF
:10B3C000A04202D1C068B06109E040B1C168A142A9
:10B3D00002D1E168C16002E008460028F6D1E560CC
:10B3E00037704A480068A04202D105F001F902E036
:10B3F000204600F08BFB04B00020BDE8F081207DEA
:10B4000048B101281ED0022827D004B02046BDE84C
:10B41000F04100F081B8E08A80B13069A04202D1E9
:10B42000C068306109E040B1C168A14202D1E16861
:10B43000C16002E008460028F6D1E560204600F031
:10B4400065FB12E0204601F0A1F92146304802F0E8
:10B4500077FB204600F046FC07E021462D4802F02D
:10B460006FFB3770204600F051FB04B00020BDE8B0
:10B47000F08100002E2E2F4D6964646C6577617237
:10B4800065732F54686972645F50617274792F4CD0
:10B490007749502F7372632F636F72652F746370D7
:10B4A0002E6300007463705F636C6F73655F736815
:10B4B0007574646F776E3A20696E76616C6964208A
:10B4C00070636200417373657274696F6E20222528
:10B4D0007322206661696C6564206174206C696EFA
:10B4E0006520256420696E2025730A00DC00002099
:10B4F0007063622D3E666C61677320262054465F40
:10B500005258434C4F534544000000001C0100209A
:10B51000F0000020F400002070B50446002C06D195
:10B520001AA34FF4CE7225A127A0F4F75BFF207D6C
:10B530000526032805D004280AD007280FD00020AC
:10B5400070BD204604F084FA05467DB926750DE0ED
:10B55000204604F07DFA054645B9267506E02046EA
:10B5600004F076FA05460DB9092020751DB1B5F134
:10B57000FF3F05D002E0204601F09CFC284670BD4C
:10B58000608B40F008006083002070BD2E2E2F4D90
:10B590006964646C6577617265732F54686972645D
:10B5A0005F50617274792F4C7749502F7372632FFB
:10B5B000636F72652F7463702E6300007063622086
:10B5C000213D204E554C4C00417373657274696F78
:10B5D0006E2022257322206661696C656420617487
:10B5E000206C696E6520256420696E2025730A0031
:10B5F0002DE9F047DDF8208007460D4691469A4632
:10B60000002F05D130A3A3223CA144A0F4F7EAFE09
:10B61000002D05D12CA3A4224AA140A0F4F7E2FEFC
:10B6200018F0010F01D0042600E000260220FCF7EC
:10B63000EBFD04001DD084F80A804FF00008C4F828
:10B64000008065602889B04205D21FA3B02246A1C0
:10B6500032A0F4F7C7FE2889801B208114212846D8
:10B66000FDF708FD58B1204604F05EF90020BDE862
:10B67000F0872846FEF79AF90020BDE8F087606859
:10B680004068E060F88AFCF749F9E1680880388B87
:10B69000FCF744F9E16848805046FCF733F9E1686B
:10B6A0004860052000EB96004FF6FF7101EA00307C
:10B6B00040EA0900FCF732F9E1688881E068A0F807
:10B6C00012802046BDE8F0872E2E2F4D6964646CF1
:10B6D0006577617265732F54686972645F50617237
:10B6E00074792F4C7749502F7372632F636F726593
:10B6F0002F7463705F6F75742E6300007463705FE6
:10B700006372656174655F7365676D656E743A2019
:10B71000696E76616C696420706362004173736561
:10B720007274696F6E2022257322206661696C65D0
:10B7300064206174206C696E6520256420696E2028
:10B7400025730A007463705F6372656174655F736B
:10B7500065676D656E743A20696E76616C69642008
:10B760007062756600000000702D3E746F745F6C2F
:10B77000656E203E3D206F70746C656E00000000A9
:10B7800070B504460D46002A06D10CA340F6C5024A
:10B7900016A120A0F4F726FE3DB1298D61B128291C
:10B7A00005D9A1F1280080B202E0204670BD00203A
:10B7B000844200D220460446204670BD2E2E2F4DD6
:10B7C0006964646C6577617265732F54686972642B
:10B7D0005F50617274792F4C7749502F7372632FC9
:10B7E000636F72652F7463702E6300007463705F03
:10B7F0006566665F73656E645F6D73735F6E6574B7
:10B8000069663A20696E76616C6964206473745F5E
:10B8100069700000417373657274696F6E20222530
:10B820007322206661696C6564206174206C696EA6
:10B830006520256420696E2025730A002DE9F843F0
:10B8400004460E46002516F0030F06D148A340F229
:10B850001142544954A0F4F7C5FD002C06D144A36D
:10B8600040F213425AA150A0F4F7BCFD16F0020FAB
:10B8700000D0012515F0010F01D0042700E00027BA
:10B880004FF4207239463620FDF760FC5FEA00086D
:10B8900000F02B80B8F80A00B84206D234A340F278
:10B8A000394253A140A0F4F79DFD00953246414630
:10B8B0002046E36DFFF79CFE05001ED0287B10F0AC
:10B8C000030F06D02AA340F2424258A136A0F4F753
:10B8D00089FD288930B126A340F2434259A132A004
:10B8E000F4F780FDE06E80B112E0608B40F08000E4
:10B8F00060834FF0FF30BDE8F883608B40F080003C
:10B9000060834FF0FF30BDE8F883E56604E0084649
:10B9100001680029FBD105600020A4F8680006F04A
:10B92000020006F00101084302D0E06D401CE06512
:10B9300016F0010F03D0608B40F020006083686830
:10B94000FDF74CFEB4F86610084480B2A4F8660017
:10B9500050B1206F40B9E06E30B905A340F26542A6
:10B9600043A111A0F4F73EFD0020BDE8F8830000DC
:10B970002E2E2F4D6964646C6577617265732F5448
:10B98000686972645F50617274792F4C7749502FE7
:10B990007372632F636F72652F7463705F6F75745A
:10B9A0002E630000941D0108417373657274696F02
:10B9B0006E2022257322206661696C6564206174A3
:10B9C000206C696E6520256420696E2025730A004D
:10B9D0007463705F656E71756575655F666C6167D0
:10B9E000733A20696E76616C69642070636200004E
:10B9F0007463705F656E71756575655F666C6167B0
:10BA0000733A20636865636B2074686174206669AB
:10BA100072737420706275662063616E20686F6C4B
:10BA200064206F70746C656E000000007365672D94
:10BA30003E746370686472206E6F7420616C696715
:10BA40006E6564007463705F656E71756575655FC2
:10BA5000666C6167733A20696E76616C6964207305
:10BA600065676D656E74206C656E677468000000B4
:10BA70007463705F656E71756575655F666C61672F
:10BA8000733A20696E76616C6964207175657565BD
:10BA9000206C656E677468002DE9F0411A4EB0782D
:10BAA000401CB0700027B469002C2BD0A17FB07867
:10BAB000814224D0A077608B10F0010F09D040F0B4
:10BAC00002006083204601F0F5F9608B20F003004E
:10BAD0006083608B10F0080F05D020F008006083B1
:10BAE0002046FFF719FDE568A06F30B1377020469A
:10BAF00002F0F2FB30780028D5D12C4600E0E46853
:10BB0000002CD3D1BDE8F081DC00002010B5044644
:10BB1000227D012A05D106A3D42211A115A0F4F794
:10BB200061FC2146BDE810400020FCF7ABBA0000E4
:10BB30002E2E2F4D6964646C6577617265732F5486
:10BB4000686972645F50617274792F4C7749502F25
:10BB50007372632F636F72652F7463702E630000BE
:10BB60007463705F667265653A204C495354454E64
:10BB700000000000417373657274696F6E202225A6
:10BB80007322206661696C6564206174206C696E43
:10BB90006520256420696E2025730A002DE9F04791
:10BBA00005460C469846DFF894902CE0264624681B
:10BBB0007068FDF713FD0746B5F86600B84206D277
:10BBC0001FA340F257422BA134A0F4F70BFCB5F8A9
:10BBD0006600C01BA5F866003089B9F80810084453
:10BBE000A9F80800304603F09FFEB5F8660000286B
:10BBF00009D054EA080006D111A340F2614231A1F4
:10BC000026A0F4F7EFFBB4B1E0684068FBF77AFEDA
:10BC10000646E0688089FBF781FE10F0030F01D033
:10BC2000012000E00020218930440844D9F8181090
:10BC3000401A0028BADD2046BDE8F087FC0000204D
:10BC40002E2E2F4D6964646C6577617265732F5475
:10BC5000686972645F50617274792F4C7749502F14
:10BC60007372632F636F72652F7463705F696E2EDA
:10BC7000630000007063622D3E736E645F717565D2
:10BC800075656C656E203E3D20706275665F636C05
:10BC9000656E286E6578742D3E702900417373655A
:10BCA0007274696F6E2022257322206661696C654B
:10BCB00064206174206C696E6520256420696E20A3
:10BCC00025730A007463705F726563656976653A0F
:10BCD0002076616C6964207175657565206C656E90
:10BCE0006774680010B50446227D012A05D106A3B9
:10BCF000DF2211A117A0F4F775FB2146BDE8104023
:10BD00000120FCF7BFB900002E2E2F4D6964646C32
:10BD10006577617265732F54686972645F506172F0
:10BD200074792F4C7749502F7372632F636F72654C
:10BD30002F7463702E6300007463705F66726565B4
:10BD40005F6C697374656E3A20214C495354454EBB
:10BD500000000000417373657274696F6E202225C4
:10BD60007322206661696C6564206174206C696E61
:10BD70006520256420696E2025730A0010B50446ED
:10BD8000606F002803D003F0DEFD0020606710BD67
:10BD9000084BD888411CD9801969002902D09A889B
:10BDA000904203D2D9681431085C7047801AC0B23F
:10BDB000085C7047FC00002010B509488069002825
:10BDC0000CD0C468418B11F0080F04D021F0080199
:10BDD0004183FFF7A1FB20460028F2D110BD0000EF
:10BDE000DC00002010B5F4F749FA0349C0F30D0058
:10BDF00000F54040888010BDDC0000202DE9F04FA8
:10BE000083B00546002D05D1DDA38322E9A1EFA073
:10BE1000F4F7E8FAF74F6868F86068891428C0F00A
:10BE20002B83DFF8D483D8F80010D8F81400FAF781
:10BE300017FC002840F0208398F8140000F0F00070
:10BE4000E02800F01983F8688089FBF767FD000B94
:10BE500081001429C0F0108328898842C0F00C8327
:10BE6000A1F1140080B278804FF00009C7F810905B
:10BE70006A898A4204D3B8802846FDF76FFF33E011
:10BE8000286828B9BEA3C222DCA1D0A0F4F7AAFA80
:10BE900014212846FDF762FF6989B9807888401A25
:10BEA00084B22846FDF75AFF28684189A142C0F0B4
:10BEB000E382416839612146FDF750FF2889001B64
:10BEC0002881688928B1AEA3DF22D0A1BFA0F4F7F2
:10BED00089FA286829890089814205D0A8A3E0222F
:10BEE000CDA1BAA0F4F77EFAF8680088FBF716FD3A
:10BEF0000146F86801804088FBF710FD0146F868AC
:10BF000041804068FBF7FEFC0146F86841607961BA
:10BF10008068FBF7F7FC0146F8688160B961C08969
:10BF2000FBF7FCFC0146F868C1818089FBF7F6FC51
:10BF300000F03F0139702889788111F0030F05D096
:10BF4000411C89B27981884200F296820026DFF88E
:10BF5000E8A2DAF80040002C00F05A80207D28B9D1
:10BF600087A3FB22B5A199A0F4F73CFA207D0A280B
:10BF700005D183A3FC22BBA194A0F4F733FA207D62
:10BF8000012805D17EA3FD22C1A190A0F4F72AFAD1
:10BF9000207A48B1D8F8041091F83410491CC9B27D
:10BFA000884201D0264630E0F868218B0288914211
:10BFB0002AD1E18A4088814226D16068D8F81010E1
:10BFC000884221D12068D8F8141088421CD1E0683A
:10BFD000A04206D16AA340F20D12B7A17BA0F4F7EC
:10BFE00001FA36B1E068F060DAF80000E060CAF803
:10BFF0000040E068A0420BD161A340F21512B9A144
:10C0000072A0F4F7EFF903E02646E468002CA5D10E
:10C01000002C6DD1BE480468002C32D0207D0A2847
:10C0200006D057A340F21F12BAA168A0F4F7DAF9BC
:10C03000207A38B1D8F8041091F83410491CC9B2EC
:10C0400088421BD1F868218B0288914216D1E18A7F
:10C050004088814212D16068D8F8101088420DD112
:10C060002068D8F81410884208D1204604F028FA35
:10C0700003B02846BDE8F04FFDF798BCE468002CFB
:10C08000CCD10021DFF8BCB2DBF800008246F8B169
:10C09000D8F80430D7F80CC0D8F81460027A4AB146
:10C0A00093F834E00EF1010E0EF0FF0E724501D050
:10C0B00001460AE0C28ABCF802E0724504D1026877
:10C0C000B24205D020B11AB10146C0680028E5D1BE
:10C0D00070B129B1C268CA60C0F80CA0CBF80000EA
:10C0E00000F0B6FB03B02846BDE8F04FFDF75EBC9C
:10C0F000002C42D0944EC6F800902889308175609B
:10C10000F868F060C7F81C9087F80190A7F80890CD
:10C11000387810F0080F03D0687B40F00100687396
:10C12000A06F80B1204602F0D7F810F10D0F03D0B8
:10C13000A06F40B1788930B1608D00281ED12046B3
:10C1400003F00CFC6DE13C62204601F0C3FD10F1F0
:10C150000D0F13D0787810F0080F10D0D4F890207D
:10C160001AB16FF00D01206990472146324801F065
:10C17000E7FC2046FFF7CAFC53E160E132E1E5E06D
:10C180002E2E2F4D6964646C6577617265732F5430
:10C19000686972645F50617274792F4C7749502FCF
:10C1A0007372632F636F72652F7463705F696E2E95
:10C1B000630000007463705F696E7075743A206983
:10C1C0006E76616C69642070627566004173736598
:10C1D0007274696F6E2022257322206661696C6516
:10C1E00064206174206C696E6520256420696E206E
:10C1F00025730A00FC000020CC600020702D3E6EEC
:10C2000065787420213D204E554C4C00702D3E6CBD
:10C21000656E203D3D203000702D3E746F745F6C64
:10C22000656E203D3D20702D3E6E6578742D3E7408
:10C230006F745F6C656E0000F40000207463705FC3
:10C24000696E7075743A20616374697665207063F5
:10C25000622D3E737461746520213D20434C4F5321
:10C26000454400007463705F696E7075743A2061B4
:10C270006374697665207063622D3E7374617465C2
:10C2800020213D2054494D452D574149540000007F
:10C290007463705F696E7075743A20616374697657
:10C2A00065207063622D3E737461746520213D20AA
:10C2B0004C495354454E00007463705F696E70754D
:10C2C000743A207063622D3E6E65787420213D20A3
:10C2D00070636220286265666F72652063616368BF
:10C2E000652900007463705F696E7075743A207020
:10C2F00063622D3E6E65787420213D20706362205C
:10C3000028616674657220636163686529000000B6
:10C31000F80000207463705F696E7075743A205481
:10C32000494D452D57414954207063622D3E737429
:10C33000617465203D3D2054494D452D5741495478
:10C3400000000000F00000208098002000203A89C2
:10C3500052B1D4F8803013B121462069984710F1CA
:10C360000D0F5ED0A7F80890204600F09BF8C8BBE0
:10C37000F86960B3A06F40B1AFF2FC134FF4F372F1
:10C3800040A1AFF2B810F4F72DF8A07E10F0100F16
:10C3900006D0F869FDF70AFB2046FEF70BFE40E0E9
:10C3A000D4F884C0BCF1000F05D0002320692146D9
:10C3B000FA69E04705E0002321461846FA6902F0D1
:10C3C0006BFE10F10D0F2CD008B1F869A0677878DA
:10C3D00010F0200F1CD0A06F28B1417B41F020014C
:10C3E000417315E01DE0208DB0F5066F01D0401CB3
:10C3F0002085D4F884C0BCF1000F05D000231A4674
:10C4000021462069E04700E0002010F10D0F08D020
:10C41000C7F82090204600F045F810B9204600F0FB
:10C4200049FDC7F82090C7F81C907068002803D019
:10C43000FDF7BCFAC6F8049003B0BDE8F08FF868C9
:10C440008089FBF76BFA10F0040F0FD1F868144ADB
:10C4500008F11403018840880092029101907989C3
:10C46000786942180020B96903F078F903B02846CA
:10C47000BDE8F04FFDF79ABA03B02846BDE8F04F8B
:10C48000FDF794BA7063622D3E72656675736564DC
:10C490005F64617461203D3D204E554C4C000000AE
:10C4A000DC60002010B50446002C06D110A340F239
:10C4B0005A221CA125A0F3F795FF2E48407810F0D2
:10C4C000100F13D0A07E10F0100F06D1D4F89020DA
:10C4D0001AB16FF00E01206990472146264801F0FD
:10C4E0002FFB2046FFF712FB012010BD002010BDDE
:10C4F0002E2E2F4D6964646C6577617265732F54BD
:10C50000686972645F50617274792F4C7749502F5B
:10C510007372632F636F72652F7463705F696E2E21
:10C52000630000007463705F696E7075745F6465AA
:10C530006C617965645F636C6F73653A20696E76D0
:10C54000616C696420706362000000004173736570
:10C550007274696F6E2022257322206661696C6592
:10C5600064206174206C696E6520256420696E20EA
:10C5700025730A00FC000020F400002070B504467A
:10C580000026002C06D112A340F624021DA124A0EF
:10C59000F3F728FF206D401EFBF7B4F90346002295
:10C5A0003146204600F00CFE05466DB133460022B0
:10C5B0002946204600F072FF231D224629462046C8
:10C5C000BDE8704000F0F6BE4FF0FF3070BD0000D7
:10C5D0002E2E2F4D6964646C6577617265732F54DC
:10C5E000686972645F50617274792F4C7749502F7B
:10C5F0007372632F636F72652F7463705F6F7574EE
:10C600002E6300007463705F6B656570616C6976A2
:10C61000653A20696E76616C69642070636200001F
:10C62000417373657274696F6E20222573222066D0
:10C6300061696C6564206174206C696E6520256495
:10C6400020696E2025730A0030B47F2800D97F202E
:10C6500000281DD0401E00F0FF0C002300200D4AD2
:10C66000916981B1D4684A7D624505D308D10D6ACC
:10C67000A4EB05059D4203D3086A231A0846944695
:10C68000C9680029EFD1002802D030BCFEF792BC67
:10C6900030BC7047DC00002010B50446082C08D0E0
:10C6A000092C06D011A340F2DD621CA11FA0F3F7F4
:10C6B00099FE002200232749886970B1D1F80CC087
:10C6C000017DA14206D1016AACEB0101914201D387
:10C6D0000A460346C0680028F2D1002B05D0BDE809
:10C6E000104000211846FEF78BBB10BD2E2E2F4D9B
:10C6F0006964646C6577617265732F5468697264EC
:10C700005F50617274792F4C7749502F7372632F89
:10C71000636F72652F7463702E630000696E7661BB
:10C720006C69642073746174650000004173736503
:10C730007274696F6E2022257322206661696C65B0
:10C7400064206174206C696E6520256420696E2008
:10C7500025730A00DC000020002300200A4AD1696A
:10C7600000290BD0D2F80CC00A6AACEB02029A4244
:10C7700001D313460846C9680029F5D1002801D025
:10C78000FEF718BC70470000DC00002070B50646BC
:10C79000002E06D10EA340F2111219A11BA0F3F72F
:10C7A00021FE307D012806D009A34FF4897221A112
:10C7B00016A0F3F717FE0124244D314655F8240046
:10C7C000006802F045FD641C042CF6D370BD000027
:10C7D0002E2E2F4D6964646C6577617265732F54DA
:10C7E000686972645F50617274792F4C7749502F79
:10C7F0007372632F636F72652F7463702E63000012
:10C8000070636220213D204E554C4C00417373658E
:10C810007274696F6E2022257322206661696C65CF
:10C8200064206174206C696E6520256420696E2027
:10C8300025730A007063622D3E7374617465203D38
:10C840003D204C495354454E00000000F01C0108A7
:10C85000F0B583B00546454E307810F0040F1ED178
:10C86000002D06D142A340F281224EA155A0F3F73C
:10C87000B9FD30785D4F10F0100F12D0F06807F15D
:10C88000100207F114030188408800920291019080
:10C890007189706942182846B16902F05FFF03B0E0
:10C8A000F0BD10F0020FFAD0687DFEF7FDFB0446E4
:10C8B000200049D07869206038696060E88AE082A9
:10C8C000F06800882083032020757069401C606236
:10C8D000E062204600F016FAA06520656064E0651D
:10C8E0007069401E606528692061E567687A00F01C
:10C8F0000C006072287A20723D480168E160046093
:10C9000003F0C4FD3B4901200870204600F086FF7B
:10C91000F068C089A4F86000A4F86200201DFAF74E
:10C9200009FB638E0146221D1846FEF729FF60862B
:10C9300012212046FEF782FF88B103B02046BDE8F1
:10C94000F0400021FEF75CBAAB69002BA7D0286944
:10C9500003B04FF0FF32BDE8F0400021184703B0AC
:10C960002046BDE8F04000F0A5BA0000FC00002021
:10C970002E2E2F4D6964646C6577617265732F5438
:10C98000686972645F50617274792F4C7749502FD7
:10C990007372632F636F72652F7463705F696E2E9D
:10C9A000630000007463705F6C697374656E5F6927
:10C9B0006E7075743A20696E76616C69642070637C
:10C9C00062000000417373657274696F6E202225E6
:10C9D0007322206661696C6564206174206C696EE5
:10C9E0006520256420696E2025730A00CC60002034
:10C9F000F4000020DC000020002200F001B800005C
:10CA000070B5044616460025002C0CD0207D002869
:10CA100013D029A340F25A3233A141A0F3F7E2FC2C
:10CA20006FF00E0044E024A340F2593246A13CA02E
:10CA3000F3F7D8FC6FF00F003AE00120FBF7E4FBBE
:10CA4000054628001AD020692861E08AE882012082
:10CA50002875607D6875607A687200222A72E07AB3
:10CA6000E872A07AA87220682860E08AA0B14249E2
:10CA70000869A04205D1C06808610CE04FF0FF30A2
:10CA800016E040B1C168A14202D1E168C16002E094
:10CA900008460028F6D1E2602046FFF737F837480D
:10CAA000A86137480168E960056003F0EFFC0020E9
:10CAB00006B13070284670BD2E2E2F4D6964646C0F
:10CAC0006577617265732F54686972645F50617233
:10CAD00074792F4C7749502F7372632F636F72658F
:10CAE0002F7463702E6300007463705F6C697374DD
:10CAF000656E5F776974685F6261636B6C6F675FB7
:10CB0000616E645F6572723A2070636220616C725C
:10CB10006561647920636F6E6E656374656400009F
:10CB2000417373657274696F6E20222573222066CB
:10CB300061696C6564206174206C696E6520256490
:10CB400020696E2025730A007463705F6C697374CA
:10CB5000656E5F776974685F6261636B6C6F675F56
:10CB6000616E645F6572723A20696E76616C6964A9
:10CB70002070636200000000DC0000200DB000089F
:10CB8000F000002070B504460D46002C1ED0206831
:10CB900000281BD00E4E2046B16900F01BF820463D
:10CBA000316900F017F8002D10D0286800280DD04A
:10CBB00006F114000268002A08D010682168884233
:10CBC00001D128681060D268002AF6D170BD00003B
:10CBD000DC00002070B506460C46002E06D10BA3E3
:10CBE0004FF4106215A122A0F3F7FCFB002C0CD02F
:10CBF00020683168884205D1E5682046FEF7DAF9F9
:10CC00002C4600E0E468002CF2D170BD2E2E2F4D92
:10CC10006964646C6577617265732F5468697264C6
:10CC20005F50617274792F4C7749502F7372632F64
:10CC3000636F72652F7463702E6300007463705F9E
:10CC40006E657469665F69705F616464725F636872
:10CC5000616E6765645F7063626C6973743A2069C2
:10CC60006E76616C6964206F6C645F6164647200ED
:10CC7000417373657274696F6E202225732220667A
:10CC800061696C6564206174206C696E652025643F
:10CC900020696E2025730A004020FEF705BA0000C7
:10CCA000F0B44FF0000C154C154D4FF6FF764FF4D5
:10CCB0004047A888401C80B2A880B04200D1AF8015
:10CCC0000021AA8854F82100006878B1C38A9342F1
:10CCD00009D10CF101001FFA80FCBCF5804FE8D3AC
:10CCE000F0BC00207047C0680028EFD1481CC1B2DA
:10CCF0000429E7D3A888F0BC70470000F01C0108A5
:10CD0000DC00002010B5002806D106A340F6AF02D3
:10CD100010A117A0F3F766FB1F49CA688868104482
:10CD2000886010BD2E2E2F4D6964646C657761722A
:10CD300065732F54686972645F50617274792F4C07
:10CD40007749502F7372632F636F72652F7463700E
:10CD50002E6300007463705F6E6578745F6973732F
:10CD60003A20696E76616C6964207063620000002D
:10CD7000417373657274696F6E2022257322206679
:10CD800061696C6564206174206C696E652025643E
:10CD900020696E2025730A00DC00002070B505466E
:10CDA0000C46002D06D121A340F21F422CA136A033
:10CDB000F3F718FBE8688089FAF7B0FD10F0010F6F
:10CDC00004D0204602F0BFFD00242CE0384E11E0D4
:10CDD0008089FAF7A3FD10F0010F07D00120FAF7C0
:10CDE0009DFD0146E86882891143818120462468BF
:10CDF00002F09AFD44B1E0682289736941681144E8
:10CE00002A891A44511AE3D56CB1288971694218EC
:10CE1000E0684068121A002A05DD401A81B22981B3
:10CE20006868FCF7B9FE2C6070BD00002E2E2F4DF7
:10CE30006964646C6577617265732F5468697264A4
:10CE40005F50617274792F4C7749502F7372632F42
:10CE5000636F72652F7463705F696E2E63000000EC
:10CE60007463705F6F6F735F696E736572745F7305
:10CE700065676D656E743A20696E76616C696420D1
:10CE80006373656700000000417373657274696FB6
:10CE90006E2022257322206661696C6564206174AE
:10CEA000206C696E6520256420696E2025730A0058
:10CEB000FC0000202DE9F05F0446002C06D192A36F
:10CEC00040F2E1429DA1A3A0F3F78CFA207D012856
:10CED00006D18DA340F2E342A8A19EA0F3F782FA07
:10CEE000B0480068A04202D10020BDE8F09FB4F82D
:10CEF0006080B4F84800804500D38046E56E65B197
:10CF0000221D2146204602F01FFC81465FEA0900EF
:10CF10000DD084B1206870B112E0A07E10F0020F35
:10CF200000F0EB802046BDE8F05F02F017BD6FF027
:10CF30000300BDE8F09F09F10400A0B10068206083
:10CF4000E8684068FAF7DEFC616C4FF0000A401AAE
:10CF50002989084440451ED9B4F86000404510D1E5
:10CF6000206F20B10DE06FF00300BDE8F09F94F852
:10CF7000990030B984F898A0012084F8990084F8C9
:10CF80009AA0A07E10F0020F00F0B7802046BDE806
:10CF9000F05F02F0E3BC84F899A0276F0FB99CE022
:10CFA000074638680028FBD197E0E8688089FAF7DF
:10CFB000B5FC10F0040F06D053A340F236527AA10C
:10CFC00064A0F3F70FFA206FA8B1618B11F0440F42
:10CFD00011D1E06E28B102686AB90089628E904270
:10CFE00009D2B4F8640030B1B4F86600092802D25E
:10CFF00011F0A00F7DD0207D022807D01020FAF775
:10D000008DFC0146E8688289114381814A462146A8
:10D01000284600F0B3FA28B1618B41F080016183AA
:10D02000BDE8F09F2868E066207D022803D0608B71
:10D0300020F003006083E8684068FAF763FC064666
:10D04000E8688089FAF76AFC10F0030F01D001202C
:10D0500000E00020298930440844216D091A00D5D8
:10D060002065E8688089FAF759FC10F0030F01D0B9
:10D07000012000E000202989C8422AD0C5F800A07C
:10D08000206F68B1E8684068FAF73CFC0646F8682B
:10D090004068FAF737FC301A18D504F1700603E03F
:10D0A00025672F4618E03668306858B1C068406878
:10D0B000FAF728FC8346E8684068FAF723FCBBEBE4
:10D0C0000000F0D430682860356005E03D602F46F0
:10D0D00002E0284602F028FCE56E55B1E868406899
:10D0E000FAF710FC616C401A2989084440457FF624
:10D0F0005CAFE06E08B9A4F868A0608B20F08000F7
:10D1000060830020BDE8F09F2E2E2F4D6964646C73
:10D110006577617265732F54686972645F506172DC
:10D1200074792F4C7749502F7372632F636F726538
:10D130002F7463705F6F75742E6300007463705F8B
:10D140006F75747075743A20696E76616C696420CD
:10D1500070636200417373657274696F6E2022257B
:10D160007322206661696C6564206174206C696E4D
:10D170006520256420696E2025730A00646F6E2780
:10D18000742063616C6C207463705F6F757470756C
:10D190007420666F72206C697374656E2D706362A3
:10D1A000730000001C010020525354206E6F742045
:10D1B0006578706563746564206865726521000038
:10D1C0002DE9F04184B004460E4617469846002CDF
:10D1D00006D110A340F242721BA125A0F3F702F979
:10D1E000608DB4F818C0E58A10210291CDF804C012
:10D1F0000095039043463A463146606A00F04CF889
:10D20000002803D0628D616A1144E16204B0BDE878
:10D21000F08100002E2E2F4D6964646C6577617279
:10D2200065732F54686972645F50617274792F4C12
:10D230007749502F7372632F636F72652F74637019
:10D240005F6F75742E6300007463705F6F75747028
:10D2500075745F616C6C6F635F6865616465723A79
:10D2600020696E76616C6964207063620000000062
:10D27000417373657274696F6E2022257322206674
:10D2800061696C6564206174206C696E6520256439
:10D2900020696E2025730A002DE9FF5FDDF844B098
:10D2A000DDF83CA0DDF83890109F0D469846A81890
:10D2B000143081B24FF420722220FBF747FF06465C
:10D2C00030002CD0708905F11401884206D216A3D3
:10D2D00040F2237221A12DA0F3F784F87468484628
:10D2E000FAF71CFB20805046FAF718FB6080C4F860
:10D2F00004800098FAF706FBA060052000EB95007B
:10D300004FF6FF7101EA00303843FAF707FBA081BE
:10D310005846FAF703FBE08100202082608204B0C7
:10D320003046BDE8F09F00002E2E2F4D6964646CDE
:10D330006577617265732F54686972645F506172BA
:10D3400074792F4C7749502F7372632F636F726516
:10D350002F7463705F6F75742E630000636865637C
:10D360006B207468617420666972737420706275D2
:10D37000662063616E20686F6C64207374727563DD
:10D3800074207463705F6864720000004173736599
:10D390007274696F6E2022257322206661696C6544
:10D3A00064206174206C696E6520256420696E209C
:10D3B00025730A00F0B583B004460D4616461F4695
:10D3C000002D06D113A340F287721FA129A0F3F705
:10D3D00009F83A463146204602F0B6F9014619B13D
:10D3E0002CB1E37AA07A04E06FF003040BE0FF2392
:10D3F000002006220192029100903A4631462846CA
:10D40000F9F784FB04462846FCF7D0FA03B020461F
:10D41000F0BD00002E2E2F4D6964646C657761723B
:10D4200065732F54686972645F50617274792F4C10
:10D430007749502F7372632F636F72652F74637017
:10D440005F6F75742E6300007463705F6F75747026
:10D4500075745F636F6E74726F6C5F7365676D6513
:10D460006E743A20696E76616C69642070627566CC
:10D4700000000000417373657274696F6E2022258D
:10D480007322206661696C6564206174206C696E2A
:10D490006520256420696E2025730A0070B50C464E
:10D4A0001546002C06D10FA340F256721AA124A0F3
:10D4B000F2F798FF606800F1140315F0010F01D036
:10D4C000042100E0002108441430984208D0BDE84F
:10D4D000704004A340F2757223A119A0F2F782BF35
:10D4E00070BD00002E2E2F4D6964646C65776172EB
:10D4F00065732F54686972645F50617274792F4C40
:10D500007749502F7372632F636F72652F74637046
:10D510005F6F75742E6300007463705F6F75747055
:10D5200075745F66696C6C5F6F7074696F6E733A67
:10D5300020696E76616C6964207062756600000017
:10D54000417373657274696F6E20222573222066A1
:10D5500061696C6564206174206C696E6520256466
:10D5600020696E2025730A006F7074696F6E7320D6
:10D570006E6F742066696C6C656400002DE9F04183
:10D5800084B004460D461746002C06D142A34FF442
:10D59000B7624EA155A0F2F725FF002D06D13EA39C
:10D5A00040F2B9525BA151A0F2F71CFF002F06D147
:10D5B00039A340F2BA525FA14CA0F2F713FF204604
:10D5C00000F0D6F818B104B00020BDE8F081686A18
:10D5D000FAF798F9E1688860688DFAF79FF9E168D1
:10D5E000C881698D686A0844E862E06800F1140641
:10D5F000A07A10F0010F0BD02A1D39464FF40670A7
:10D60000FEF7BEF840F00170FAF77CF93060361D85
:10D61000B5F930004FF00008002801DAA5F8308095
:10D62000686B38B94C4800686863E0684068FAF78E
:10D6300069F9A8636168A0898A88801A4A89121AE0
:10D640004A8161680A89101A08816168E068486047
:10D65000E068A0F81080A07AE16810F0010F01D016
:10D66000042000E0002014300844B04206D00AA391
:10D6700040F21C6239A11DA0F2F7B4FEA87A06217F
:10D68000019102970090EB7A2A1D29466068F9F70C
:10D690003DFA04B0BDE8F0812E2E2F4D6964646C14
:10D6A0006577617265732F54686972645F50617247
:10D6B00074792F4C7749502F7372632F636F7265A3
:10D6C0002F7463705F6F75742E6300007463705FF6
:10D6D0006F75747075745F7365676D656E743A20ED
:10D6E000696E76616C696420736567004173736568
:10D6F0007274696F6E2022257322206661696C65E1
:10D7000064206174206C696E6520256420696E2038
:10D7100025730A007463705F6F75747075745F733E
:10D7200065676D656E743A20696E76616C69642018
:10D73000706362007463705F6F75747075745F738B
:10D7400065676D656E743A20696E76616C696420F8
:10D750006E65746966000000E80000206F707469EF
:10D760006F6E73206E6F742066696C6C6564000068
:10D7700010B50446002C06D107A340F29A5213A11B
:10D780001CA0F2F72FFE6068807B012801D00120E9
:10D7900010BD002010BD00002E2E2F4D6964646C5A
:10D7A0006577617265732F54686972645F50617246
:10D7B00074792F4C7749502F7372632F636F7265A2
:10D7C0002F7463705F6F75742E6300007463705FF5
:10D7D0006F75747075745F7365676D656E745F6285
:10D7E0007573793A20696E76616C69642073656738
:10D7F00000000000417373657274696F6E2022250A
:10D800007322206661696C6564206174206C696EA6
:10D810006520256420696E2025730A0070B50646D0
:10D82000002E06D11DA340F27D7229A12FA0F2F790
:10D83000D9FD384D6888002817D04FF00000E880E7
:10D8400013D9FEF7A5FA00280FD0012809D0022825
:10D850000CD0FEF79DFA022807D3E9880844801E01
:10D86000E880E88869888842EBD370BDFEF790FABB
:10D870000428FAD1E8886988801C8842F5D8FEF728
:10D8800087FA0402FEF784FA2043B0F5067F00D839
:10D8900008B94FF406707086E3E700002E2E2F4D76
:10D8A0006964646C6577617265732F54686972642A
:10D8B0005F50617274792F4C7749502F7372632FC8
:10D8C000636F72652F7463705F696E2E6300000072
:10D8D0007463705F70617273656F70743A20696E03
:10D8E00076616C6964207063620000004173736547
:10D8F0007274696F6E2022257322206661696C65DF
:10D9000064206174206C696E6520256420696E2036
:10D9100025730A00FC0000202DE9F05FDDF830B02F
:10D92000DDF82CA00A9D81460C4616461F46A046EF
:10D93000002F05D121A3E8222DA136A0F2F752FD38
:10D94000002D05D11DA3E9223CA132A0F2F74AFD2A
:10D95000B44216D21AF0020F0AD1A87E10F0400F7E
:10D960000FD1BBF1000F03D0E86E08B9286F40B1AA
:10D9700004F21B2020F00301B14200D80E461FFA2A
:10D9800086F84FF4207241464846FBF7DFFB054618
:10D99000002D10D0286830B108A340F20B122FA13F
:10D9A0001CA0F2F71FFD6889001B38802C816C8158
:10D9B0002846BDE8F09F0020BDE8F09F2E2E2F4D99
:10D9C0006964646C6577617265732F546869726409
:10D9D0005F50617274792F4C7749502F7372632FA7
:10D9E000636F72652F7463705F6F75742E630000D0
:10D9F0007463705F706275665F707265616C6C6F86
:10DA0000633A20696E76616C6964206F7665727323
:10DA1000697A6500417373657274696F6E2022259F
:10DA20007322206661696C6564206174206C696E84
:10DA30006520256420696E2025730A007463705F79
:10DA4000706275665F707265616C6C6F633A2069B5
:10DA50006E76616C69642070636200006E65656457
:10DA600020756E636861696E65642070627566001A
:10DA700070B50446002C1FD0207D00281BD00A283A
:10DA800019D0012817D0A06F002510B1FBF78EFF29
:10DA9000A567606F10B12046FEF770F94FF0FF30B8
:10DAA0002086E06E01F04FFF206F01F04CFFE5662D
:10DAB0002567A4F8685070BDBDE8704003A340F628
:10DAC00051020EA114A0F2F78DBC00002E2E2F4D96
:10DAD0006964646C6577617265732F5468697264F8
:10DAE0005F50617274792F4C7749502F7372632F96
:10DAF000636F72652F7463702E6300007463705FD0
:10DB00007063625F70757267653A20696E76616CEA
:10DB10006964207063620000417373657274696F99
:10DB20006E2022257322206661696C656420617411
:10DB3000206C696E6520256420696E2025730A00BB
:10DB400070B505460C46002C06D12AA340F6830288
:10DB500034A13BA0F2F746FC002D06D125A340F6E8
:10DB6000840241A136A0F2F73DFC2868A04202D110
:10DB7000C068286009E040B1C168A14202D1E168F3
:10DB8000C16002E008460028F6D10025E560204685
:10DB9000FFF76EFF207D0A280BD0012809D0608B8B
:10DBA00010F0010F05D040F0020060832046FFF71F
:10DBB00081F9207D01281AD0E06E30B10DA340F626
:10DBC000930231A11EA0F2F70DFC206F30B109A322
:10DBD00040F6940232A11AA0F2F704FC606F30B153
:10DBE00004A340F6960235A115A0F2F7FBFB2575BC
:10DBF000E58270BD2E2E2F4D6964646C657761726D
:10DC000065732F54686972645F50617274792F4C28
:10DC10007749502F7372632F636F72652F7463702F
:10DC20002E6300007463705F7063625F72656D6F76
:10DC300076653A20696E76616C6964207063620073
:10DC4000417373657274696F6E202225732220669A
:10DC500061696C6564206174206C696E652025645F
:10DC600020696E2025730A007463705F7063625FC1
:10DC700072656D6F76653A20696E76616C696420B5
:10DC80007063626C69737400756E73656E74207373
:10DC900065676D656E7473206C65616B696E670096
:10DCA000756E61636B6564207365676D656E747313
:10DCB000206C65616B696E67000000006F6F7365B3
:10DCC00071207365676D656E7473206C65616B6937
:10DCD0006E6700002DE9F04F83B004460025A94689
:10DCE000002C06D1EBA34FF44772F7A1FDA0F2F789
:10DCF00079FBDFF818B49BF8000010F0040F38D05F
:10DD0000227D022A06D0606ADBF81410884208D10E
:10DD1000012511E0206DDBF8181088420CD1012597
:10DD20000AE00B1A08D4238D1844081A002803DCD3
:10DD3000608B40F002006083002D16D032B9D5A36D
:10DD40004FF44E72F2A1E7A0F2F74CFB9BF80100F2
:10DD500040F008008BF80100608B20F00100608328
:10DD600003B06FF00D00BDE8F08F03B00020BDE8F8
:10DD7000F08F10F0020F0CD0207D022809D003286C
:10DD800007D0608B40F00200608303B00020BDE844
:10DD9000F08FA07E10F0100F02D1E54800682062DD
:10DDA0004FF0000A84F89BA084F89AA02046FFF761
:10DDB00035FD207DDF4B811E01270422DFF87883AB
:10DDC000DE4EDF4D03F11000082980F08182DFE88C
:10DDD00001F004ABFBFAF9FBF8F79BF8001011F027
:10DDE000100F7FD011F0020F7CD0D4F844C00CF19A
:10DDF0000105DBF818C0654574D1DBF81400411C3F
:10DE00006162E162C4F844C0DBF80C10C989A4F86F
:10DE10006010A4F86210401E60652275201DF9F79D
:10DE200089F8638E0146221D1846FDF7A9FC60861D
:10DE300041F21C12B2EB400F01D2410001E041F26D
:10DE40001C11B1EB800F01D9800006E0B2EB400F4E
:10DE500001D2400001E041F21C10A4F84800B4F8DF
:10DE6000660030B98BA34FF45B72B6A19DA0F2F7A8
:10DE7000B9FAB4F86600401EA4F86600256FDDB15B
:10DE800028682067284601F04FFD206F08B3A4F8EA
:10DE900030A084F842A0D4F8883023B10022214673
:10DEA00020699847814619F10D0F16D0608B40F01C
:10DEB0000200608300F00CBAE56E35B975A34FF42B
:10DEC0005D72A6A187A0F2F78DFA2868E066D9E70F
:10DED00008E04FF0FF302086DDE703B06FF00C0064
:10DEE000BDE8F08F11F0100F00F0F281DBF80C109C
:10DEF00014330A884988029201910090BBF80A10F5
:10DF0000DBF8140042182046DBF8181001F026FC5C
:10DF100094F84200062880F0DB81A4F830A0204667
:10DF200001F0DEFA00F0D4B99BF8001011F0100FE8
:10DF30007BD0D4F844C0DBF81810A1EB0C0CBCF17A
:10DF4000010F5ED4D4F850C0A1EB0C0CBCF1000F53
:10DF500057DC2275E06F10B1806918B109E06FF0ED
:10DF6000050010E04BA34FF46A7281A15DA0F2F7A7
:10DF700039FAE06F836923B100222146206998476E
:10DF800001E06FF00F0050B110F10D0F02D02046EC
:10DF9000FDF710F803B06FF00C00BDE8F08F2046DD
:10DFA00000F024FABBF8080010B1401EABF80800DE
:10DFB000608E41F21C12B2EB400F06D2410006E027
:10DFC00071E144E11AE14CE03CE041F21C11B1EB9B
:10DFD000800F01D9800006E0B2EB400F01D2400073
:10DFE00001E041F21C10A4F848009BF8010010F079
:10DFF000200F4CD0608B40F002006083072020751A
:10E0000066E1DBF80C201433B2F800C05288CDF87A
:10E0100008C001920090BBF80A20DBF8140002440B
:10E02000204601F09BFB53E1FFE711F0020F2ED0D9
:10E03000606ADBF81410401E884228D1204601F0A7
:10E040005DF945E1204600F0D1F99BF8010010F0A0
:10E05000200F1CD0608B40F00200608307202075E9
:10E0600036E1204600F0C2F99BF8010010F0200FC5
:10E070000FD09BF8000010F0100F06D0206DDBF8D9
:10E080001810884201D1E06E10B1608B80E0DDE0B5
:10E0900084E0A4E02E2E2F4D6964646C6577617274
:10E0A00065732F54686972645F50617274792F4C84
:10E0B0007749502F7372632F636F72652F7463708B
:10E0C0005F696E2E630000007463705F70726F632F
:10E0D0006573733A20696E76616C6964207063625F
:10E0E00000000000417373657274696F6E20222511
:10E0F0007322206661696C6564206174206C696EAE
:10E100006520256420696E2025730A00FC0000202C
:10E110007463705F696E7075743A207063622D3E2F
:10E12000737461746520213D20434C4F5345440076
:10E13000E8000020CC600020DC000020F800002077
:10E14000F40000207063622D3E736E645F7175652C
:10E1500075656C656E203E20300000006E6F207388
:10E1600065676D656E7420746F206672656500006A
:10E170007063622D3E6C697374656E65722D3E61CD
:10E18000636365707420213D204E554C4C000000A7
:10E1900040F0020060830820207599E0608B40F019
:10E1A000020060832046FFF763FC2868A04202D18A
:10E1B000C068286009E040B1C168A14202D1E168AD
:10E1C000C16002E008460028F6D188F800700A20F5
:10E1D00020753068E060346002F058F978E09BF810
:10E1E000000010F0100F73D0206DDBF8181088427B
:10E1F0006ED1E06E50BB0620207569E0204600F02D
:10E20000F5F89BF8010010F0200F61D0608B40F012
:10E21000020060832046FFF72BFC2868A04202D151
:10E22000C068286009E040B1C168A14202D1E1683C
:10E23000C16002E008460028F6D188F800700A2084
:10E2400020753068E060346002F020F940E020463C
:10E2500000F0CCF89BF8000010F0100F38D0206DC3
:10E26000DBF81810884233D1E06E88BB2046FFF7F8
:10E27000FFFB2868A04202D1C068286009E040B1D5
:10E28000C168A14202D1E168C16002E008460028ED
:10E29000F6D188F800700A2020753068E06034609C
:10E2A00002F0F4F814E0204600F0A0F89BF800001B
:10E2B00010F0100F0CD0206DDBF81810884207D139
:10E2C000E06E28B99BF8010040F010008BF80100C7
:10E2D00003B00020BDE8F08F70B50446002C0ED0CE
:10E2E000A56F6E7B0020A067D4F884C0BCF1000F3E
:10E2F0000FD000232A4621462069E0470FE01BA3E8
:10E3000040F2096225A12FA0F2F76CF86FF00F0020
:10E3100070BD00232A462146184600F0BDFE30B1EC
:10E3200010F10D0F1ED0A5676FF0040070BD16F040
:10E33000200F12D0218DB1F5066F01D0491C218527
:10E34000D4F884C0BCF1000F04D000231A46214643
:10E350002069E04710F10D0F01D0002070BD6FF073
:10E360000C0070BD6FF00C0070BD00002E2E2F4D04
:10E370006964646C6577617265732F54686972644F
:10E380005F50617274792F4C7749502F7372632FED
:10E39000636F72652F7463702E6300007463705F27
:10E3A00070726F636573735F726566757365645FC2
:10E3B000646174613A20696E76616C69642070638F
:10E3C00062000000417373657274696F6E202225CC
:10E3D0007322206661696C6564206174206C696ECB
:10E3E0006520256420696E2025730A002DE9F04719
:10E3F00004460025002C06D1E1A340F27B42EDA1AA
:10E40000F3A0F1F7EFFF207D042806D2DCA340F251
:10E410007C42F9A1EEA0F1F7E5FFFE4F4FF6FF7A3F
:10E420004FF00006387810F0100F00F01D81B4F89E
:10E430006020A06D1318D4F854C07969BCEB0108B2
:10E440000ED48C4504D1D7F818C0B0EB0C0C07D40F
:10E45000D7F818C0604510D1F868C08990420CD92F
:10E46000F868C089A4F86000B4F86220824201D242
:10E47000A4F862006165B869A065626CB869811A28
:10E48000002930DC798949BBB4F860C0A16D6144D2
:10E49000994223D1B4F9301000291FDB82421DD1EB
:10E4A000012594F84310481CC0B2884201D984F871
:10E4B000430094F8431003290BD9B4F84800628E46
:10E4C000024492B2824202D3A4F8482001E0A4F8A8
:10E4D00048A0032902D3204600F08AFF002D72D104
:10E4E00084F84360A0E001296ED4226D821A002ACC
:10E4F0006ADC628B12F0040F08D022F004026283FF
:10E50000B4F84A20A4F84820A4F86A6084F842606D
:10E51000E28FB4F93C3002EBE302A4F8402089B268
:10E5200084F843606064207D042838D3B4F8480040
:10E53000B4F84A20904216D2628B12F4006F01D0D8
:10E54000012200E00222638E5A4392B28A4200D82E
:10E550001146014489B2814202D3A4F848101EE05A
:10E56000A4F848A01BE0B4F86A20114489B2914293
:10E5700002D3A4F86A1001E0A4F86AA0B4F86A1003
:10E5800081420CD3091AA4F86A10618E014489B241
:10E59000814202D3A4F8481001E0A4F848A09EA24A
:10E5A0002046E36E216FFDF7F9FA206703469CA22F
:10E5B0002046E16EFDF7F2FAE066216F29B126866A
:10E5C000267730B107E02FE02BE04FF0FF322286B4
:10E5D000F6E7A4F86860B4F864203B891A44A4F80C
:10E5E0006420628B12F4006F1ED061B1C86840686D
:10E5F000F9F788F9E16C081A002815DC608B20F423
:10E600000060608310E038B1C0684068F9F77AF9BB
:10E61000E16C081A002807DC608B20F4006060833E
:10E6200002E0204601F09AF9606BE8B1A16BBA698B
:10E63000891A19D57C490988081AB4F93C10A0EB4D
:10E64000E10000B2014409B2A187002801DA40428A
:10E6500000B2B4F93E20A0EBA2001044E08700EB2A
:10E66000E100A4F8400066637A89002A00F09B83E9
:10E67000207D072880F09783606A7969DFF8AC8194
:10E68000A0EB0109B9F1010F49D40A44821A521CC6
:10E69000002A44DCD8F8045035B939A340F294522A
:10E6A00063A14BA0F1F79EFED14506D334A340F2FF
:10E6B000955263A146A0F1F795FE1FFA89F9D8F8A3
:10E6C00004000089484506D22DA340F2975260A16C
:10E6D0003FA0F1F787FEB8F80800A0EB0900A8F802
:10E6E0000800D8F804000089A0EB090080B269890D
:10E6F00049450AD26989A9EB01011FFA81F92881EC
:10E700006E812D6869894945F4D349462846FBF74F
:10E7100025FB606A7861D8F80C10486005E0081A9B
:10E7200003D5608B40F002006083616A7869421A09
:10E7300000F13483228D0A44821A521C002A00F30D
:10E740002D83814240F0FE81D8F80C008089F9F7D2
:10E75000E5F810F0030F01D0012000E00020B8F828
:10E760000810084480B27881218D814278D2D8F88F
:10E770000C008089F9F7D2F810F0010F71D071E028
:10E780002E2E2F4D6964646C6577617265732F540A
:10E79000686972645F50617274792F4C7749502FA9
:10E7A0007372632F636F72652F7463705F696E2E6F
:10E7B000630000007463705F726563656976653A33
:10E7C00020696E76616C69642070636200000000ED
:10E7D000417373657274696F6E20222573222066FF
:10E7E00061696C6564206174206C696E65202564C4
:10E7F00020696E2025730A007463705F726563651B
:10E800006976653A2077726F6E67207374617465FC
:10E8100000000000FC000020756E61636B65640001
:10E82000756E73656E740000E8000020809800200B
:10E83000696E7365672E7020213D204E554C4C004B
:10E84000696E73616E65206F666673657421000082
:10E850007062756620746F6F2073686F7274210028
:10E8600048E011E0D8F80C008089F9F757F8C0F3B8
:10E8700044004000F9F752F80146D8F80C008289AC
:10E8800022F47C5211438181208DA8F80800D8F829
:10E890000C008089F9F742F810F0020F04D0B8F8A4
:10E8A0000800401EA8F80800B8F80810D8F80400BE
:10E8B000FBF772F9D8F80C008089F9F72FF810F0FF
:10E8C000030F01D0012000E00020B8F80810084430
:10E8D00080B27881228D616A11447A69104488423D
:10E8E00008D0AFF2641340F2CB52F7A1AFF2201080
:10E8F000F1F778FD606F002870D0D8F80C0080899F
:10E90000F9F70CF810F0010F0BD0606F00287DD0E4
:10E91000606F0168616701F007F8606F0028F7D148
:10E9200074E0656F27E08089F8F7F8FF10F0010FB9
:10E930001DD0D8F80C008089F8F7F0FF10F0020F16
:10E9400015D10120F8F7EAFF0146D8F80C008289BA
:10E95000114381810846F8F7E1FF10F0030F01D061
:10E96000012000E00020B8F808100844788128460B
:10E970002D6800F0D9FF45B1E8682A897B89416894
:10E9800011447A691A44511ACDD545B37989786909
:10E990004218E9684968521A002A36DD081AA8F8B0
:10E9A0000800D8F80C008089F8F7B8FF10F0020FC3
:10E9B00004D0B8F80800401EA8F80800B8F80810FD
:10E9C000D8F80400FBF7E8F8D8F80C008089F8F7CD
:10E9D000A5FF10F0030F03D0012002E016E014E0C1
:10E9E0000020B8F80810084480B27881796908449A
:10E9F000E9684968884208D0AFF27C2340F2FC52B3
:10EA0000BFA1AFF23420F1F7EDFC65677889796931
:10EA100001446162218D814208D2AFF29C2340F211
:10EA20000762C6A1AFF25820F1F7DCFC218D78898E
:10EA3000081A2085204601F0E3FDD8F8040001897A
:10EA400011B1F861C8F80460D8F80C008089F8F7B3
:10EA500065FF10F0010F03D0787840F02000787047
:10EA60004FF0070857E079618089F8F757FF10F0F9
:10EA7000030F01D0012000E000202A89616A1144BF
:10EA800008446062E8688089F8F748FF10F0030FD7
:10EA900001D0012000E0002029890844218D88420E
:10EAA00008D9AFF2243340F22B62ACA1AFF2E020E0
:10EAB000F1F798FCE8688089F8F730FF10F0030F51
:10EAC00001D0012000E0002029890844218D081A86
:10EAD0002085204601F094FD6968088930B1F86905
:10EAE00010B1FAF7DFFC00E0F9616E60E868808938
:10EAF000F8F714FF10F0010F08D0787840F02000EC
:10EB00007870207D042801D184F81480286860671B
:10EB1000284600F009FF656F25B1E868626A416820
:10EB20009142A0D0608B10F0010F06D020F00100C0
:10EB300040F002006083BDE8F08740F00100608390
:10EB4000BDE8F087656F8DB10026E96849688142AC
:10EB500016D1B8F80800298988427BD9894800F085
:10EB60008BFE002876D036B1306005E0854800F095
:10EB700083FE60670DE160672946FEF70FF908E143
:10EB800026B3F2685268821A012A2AD4421A521C09
:10EB9000002A26DC7B4800F06FFE80465FEA080012
:10EBA00058D0F0683189406842187969521A002AB1
:10EBB00005DD081A81B231817068FAF7EDFFC6F8F9
:10EBC000008029464046FEF7E9F8E2E0421A08D5FF
:10EBD0006C4800F051FEE8B360672946FEF7DEF8A6
:10EBE000D7E02E462A68B2BB411A002933DDE86817
:10EBF0008089F8F793FE10F0010F2BD1614800F0E7
:10EC00003BFE286030B3E868416828890A187869B3
:10EC1000121A002A05DD401A81B229816868FAF7C4
:10EC2000BBFF218D606A7A69084479891144081A0A
:10EC300000280FDD2868C0688089F8F76FFE10F0A3
:10EC4000010F14D02868C0688089F8F767FEC0F308
:10EC5000440001E098E098E04000F8F75FFE0146CC
:10EC60002868C068828922F47C5211438181A08C7B
:10EC7000218D0844B98A401A81B228680181286828
:10EC80004068FAF789FF2868C0688089F8F746FE6F
:10EC900010F0030F01D0012000E00020296809894D
:10ECA000084480B27881228D616A11447A691044E7
:10ECB00088426ED0AFF238534FF4DF6202A1AFF258
:10ECC000F040F1F78FFB64E07463705F7265636519
:10ECD0006976653A207365676D656E74206E6F7432
:10ECE000207472696D6D656420636F727265637400
:10ECF0006C7920746F207263765F776E640A00000F
:10ED00007463705F726563656976653A20736567E1
:10ED10006D656E74206E6F74207472696D6D6564BC
:10ED200020636F72726563746C7920746F206F6FEB
:10ED30007365712071756575650A00007463705F95
:10ED4000726563656976653A207463706C656E20E0
:10ED50003E207263765F776E640A00007463705FB2
:10ED6000726563656976653A206F6F7365712074AB
:10ED700063706C656E203E207263765F776E640A06
:10ED8000000000008098002003E015462A007FF470
:10ED9000DCAE2046BDE8F04700F0E0BD2046BDE80F
:10EDA000F04700F0DBBD606A79690A1A06D4228D4B
:10EDB0001044081A401C00287FF7C2AE608B40F058
:10EDC00002006083BDE8F08770B504460D46002C54
:10EDD0000BD0207D012806D104A340F2DF720FA1E1
:10EDE00018A0F1F7FFFAC4F8845070BD2E2E2F4DF5
:10EDF0006964646C6577617265732F5468697264C5
:10EE00005F50617274792F4C7749502F7372632F62
:10EE1000636F72652F7463702E630000696E766194
:10EE20006C696420736F636B6574207374617465BF
:10EE300020666F7220726563762063616C6C62611C
:10EE4000636B0000417373657274696F6E202225D5
:10EE50007322206661696C6564206174206C696E40
:10EE60006520256420696E2025730A002DE9F04194
:10EE700007460D4614461E46E4B12189284600F097
:10EE800065F912480560228911486168F1F79AFB1B
:10EE9000208910490880002201210F48F3F78EF8DD
:10EEA0000C4802880A490D4802F0C0F92046FAF7DA
:10EEB0007DFD09E024B92846FCF7F6F9BDE8F081AC
:10EEC00016B12046FAF772FD0020F7E73C0100205A
:10EED000809B00204E01002000040240100300200F
:10EEE0002DE9F04107460D4614461E46E4B121893E
:10EEF000284600F02BF91248056022891148616804
:10EF0000F1F760FB208910490880002210210F488A
:10EF1000F3F754F80C4802880A490D4802F086F9C4
:10EF20002046FAF743FD09E024B92846FCF7BCF96E
:10EF3000BDE8F08116B12046FAF738FD0020F7E76A
:10EF400040010020809D0020500100200000024070
:10EF5000380200202DE9F04107460D4614461E46B2
:10EF6000ECB12189284600F0F1F8134805602289A8
:10EF700012486168F1F726FB2089114908800022B8
:10EF80004FF480710F48F3F719F80D4802880B49C8
:10EF90000D4802F04BF92046FAF708FD09E024B9C4
:10EFA0002846FCF781F9BDE8F08116B12046FAF752
:10EFB000FDFC0020F7E7000044010020809F0020B6
:10EFC0005201002000100240800200202DE9F04193
:10EFD00007460D4614461E46ECB12189284600F02E
:10EFE000B5F813480560228912486168F1F7EAFA1A
:10EFF00020891149088000224FF480510F48F2F710
:10F00000DDFF0D4802880B490D4802F00FF920463C
:10F01000FAF7CCFC09E024B92846FCF745F9BDE82D
:10F02000F08116B12046FAF7C1FC0020F7E7000096
:10F030004801002080A1002054010020001002405F
:10F04000C80200202DE9F04107460D4614461E4631
:10F050009CB12189284600F079F80C480560228986
:10F060000B486168F1F7AEFA20890A490880F9F780
:10F0700003FB2046FAF79AFC05E026B92846FCF780
:10F0800013F9BDE8F0810020FBE700003801002003
:10F09000809900204C01002010B508461446002835
:10F0A00008D0002C10D0218900F050F82046FAF743
:10F0B0007DFC0AE008A34FF4D36213A119A0F1F775
:10F0C00091F96FF00F0010BD0BB1002010BDBDE82D
:10F0D0001040FCF7E9B800002E2E2F4D6964646CD7
:10F0E0006577617265732F54686972645F506172ED
:10F0F00074792F4C7749502F7372632F636F726549
:10F100002F7463702E6300007463705F72656376A2
:10F110005F6E756C6C3A20696E76616C6964207004
:10F1200063620000417373657274696F6E202225FB
:10F130007322206661696C6564206174206C696E5D
:10F140006520256420696E2025730A0070B5044689
:10F150000D46002C03D0207D012809D00FE0BDE82A
:10F16000704015A340F2CF321FA125A0F1F73AB9A4
:10F1700011A340F2D2322CA121A0F1F733F9228D54
:10F18000501980B2B0F5066F01D8824203D94FF40E
:10F190000660208500E02085204601F031FAB0F5B8
:10F1A000067F08D3608B40F0020060832046BDE8F4
:10F1B0007040FDF77FBE70BD2E2E2F4D6964646CCC
:10F1C0006577617265732F54686972645F5061720C
:10F1D00074792F4C7749502F7372632F636F726568
:10F1E0002F7463702E6300007463705F72656376C2
:10F1F00065643A20696E76616C69642070636200B0
:10F20000417373657274696F6E20222573222066C4
:10F2100061696C6564206174206C696E6520256489
:10F2200020696E2025730A00646F6E277420636165
:10F230006C6C207463705F72656376656420666FC2
:10F2400072206C697374656E2D70636273000000C8
:10F2500070B504460D46002D05D108A3FF2213A169
:10F260001CA0F1F7BFF8002C07D00020E16FA942E5
:10F2700000D1E067E468002CF8D170BD2E2E2F4D30
:10F280006964646C6577617265732F546869726430
:10F290005F50617274792F4C7749502F7372632FCE
:10F2A000636F72652F7463702E6300007463705F08
:10F2B00072656D6F76655F6C697374656E65723AC1
:10F2C00020696E76616C6964206C697374656E6523
:10F2D00072000000417373657274696F6E2022259D
:10F2E0007322206661696C6564206174206C696EAC
:10F2F0006520256420696E2025730A002DE9F04100
:10F300000546002D06D11DA340F2C16228A12EA002
:10F31000F1F768F82E6F3EB13046FEF729FA38B1A2
:10F320006FF00500BDE8F0816FF00500BDE8F081E9
:10F330003068286705F16C0400E02468206850B14B
:10F34000C0684068F8F7DEFA0746F0684068F8F7EA
:10F35000D9FA381AF1D4206830602660306800216C
:10F3600008B9A5F8681095F84200FF2802D2401CA1
:10F3700085F8420069630020BDE8F0812E2E2F4DF4
:10F380006964646C6577617265732F54686972642F
:10F390005F50617274792F4C7749502F7372632FCD
:10F3A000636F72652F7463705F6F75742E630000F6
:10F3B0007463705F7265786D69743A20696E766106
:10F3C0006C69642070636200417373657274696F65
:10F3D0006E2022257322206661696C656420617449
:10F3E000206C696E6520256420696E2025730A00F3
:10F3F00010B50446002C06D11AA340F2F96226A1EA
:10F400002DA0F0F7EFFF206F002829D0A07E10F08C
:10F41000040F25D12046FFF771FF002820D1B4F852
:10F420004810B4F86000814200D208464108A4F8B0
:10F430004A10608EB1EB400F05D24FF6FF7101EA22
:10F440004001A4F84A10B4F84A1000EB4000084408
:10F45000A4F84800608B40F0040060830020208600
:10F4600010BD00002E2E2F4D6964646C65776172AB
:10F4700065732F54686972645F50617274792F4CA0
:10F480007749502F7372632F636F72652F746370A7
:10F490005F6F75742E6300007463705F7265786DC2
:10F4A00069745F666173743A20696E76616C696431
:10F4B0002070636200000000417373657274696FAD
:10F4C0006E2022257322206661696C656420617458
:10F4D000206C696E6520256420696E2025730A0002
:10F4E00010B50446002C06D108A340F2AD6214A169
:10F4F0001AA0F0F777FF204600F09CF8002804D10E
:10F500002046BDE8104000F03DB810BD2E2E2F4D16
:10F510006964646C6577617265732F54686972649D
:10F520005F50617274792F4C7749502F7372632F3B
:10F53000636F72652F7463705F6F75742E63000064
:10F540007463705F7265786D69745F72746F3A206E
:10F55000696E76616C6964207063620041737365E3
:10F560007274696F6E2022257322206661696C6552
:10F5700064206174206C696E6520256420696E20AA
:10F5800025730A0010B50446002C06D109A34FF4D8
:10F59000D36215A11DA0F0F725FF94F84200FF28C3
:10F5A00002D2401C84F842002046BDE81040FDF71E
:10F5B00081BC00002E2E2F4D6964646C65776172EA
:10F5C00065732F54686972645F50617274792F4C4F
:10F5D0007749502F7372632F636F72652F74637056
:10F5E0005F6F75742E6300007463705F7265786D71
:10F5F00069745F72746F5F636F6D6D69743A2069CF
:10F600006E76616C6964207063620000417373659B
:10F610007274696F6E2022257322206661696C65A1
:10F6200064206174206C696E6520256420696E20F9
:10F6300025730A002DE9F0410546002D06D122A3CD
:10F6400040F263622DA136A0F0F7CCFE2C6F4CB1D6
:10F65000206878B12046FEF78BF838B16FF00500CE
:10F66000BDE8F0816FF00500BDE8F08124682068F6
:10F670000028EFD12046FEF77BF818B16FF00500A7
:10F68000BDE8F081E86E2060286FE86600272F67EC
:10F69000688B40F400606883E0684068F8F732F9EE
:10F6A0000646E0688089F8F739F910F0030F01D0B9
:10F6B000012000E00020218930440844E8646F63A1
:10F6C0000020BDE8F08100002E2E2F4D6964646C8F
:10F6D0006577617265732F54686972645F506172F7
:10F6E00074792F4C7749502F7372632F636F726553
:10F6F0002F7463705F6F75742E6300007463705FA6
:10F700007265786D69745F72746F5F707265706135
:10F7100072653A20696E76616C696420706362007C
:10F72000417373657274696F6E202225732220669F
:10F7300061696C6564206174206C696E6520256464
:10F7400020696E2025730A00002803D0007A08B1D2
:10F75000F9F7B2B91046F7F7EDBB00002DE9FF4FFE
:10F7600085B08B46149F139E129D92469846B8F121
:10F77000000F06D11BA340F2C47227A12DA0F0F701
:10F7800031FE002D06D117A340F2C57233A129A086
:10F79000F0F728FE4FF0000946F208045846F8F743
:10F7A000B1F81421034602910022019700960394B8
:10F7B00049465046FDF770FD0446002C0ED04B46DE
:10F7C000002221460598FDF769FE059809B02B46F1
:10F7D00042462146BDE8F04FFDF7ECBD09B0BDE85B
:10F7E000F08F00002E2E2F4D6964646C6577617276
:10F7F00065732F54686972645F50617274792F4C1D
:10F800007749502F7372632F636F72652F74637023
:10F810005F6F75742E6300007463705F7273743A67
:10F8200020696E76616C6964206C6F63616C5F69DE
:10F8300070000000417373657274696F6E20222539
:10F840007322206661696C6564206174206C696E46
:10F850006520256420696E2025730A007463705F3B
:10F860007273743A20696E76616C69642072656D9A
:10F870006F74655F6970000070B50546002D06D194
:10F880000CA340F2826217A11DA0F0F7ABFD02208D
:10F89000F8F7BAFC04465CB1EB682A68A9686868A6
:10F8A000E3602260A1606060FAF712FA204670BD42
:10F8B000002070BD2E2E2F4D6964646C65776172D7
:10F8C00065732F54686972645F50617274792F4C4C
:10F8D0007749502F7372632F636F72652F74637053
:10F8E0002E6300007463705F7365675F636F707988
:10F8F0003A20696E76616C69642073656700000068
:10F90000417373657274696F6E20222573222066BD
:10F9100061696C6564206174206C696E6520256482
:10F9200020696E2025730A0010B50446002C09D00A
:10F93000606808B1FAF73AF82146BDE810400220A5
:10F94000F8F7A0BB10BD10B5002805D00468FFF77C
:10F95000EBFF20460028F9D110BD00002DE9F04151
:10F96000044600260027002C06D11AA340F2EA72B2
:10F9700025A12DA0F0F736FD0025206DF7F7C2FF79
:10F980000346002229462046FDF71AFC054695B19C
:10F990003B46324629462046FDF780FD231D224680
:10F9A00029462046FDF706FD68B1618B41F0030151
:10F9B0006183BDE8F081608B40F0030060836FF0ED
:10F9C0000100BDE8F081618B21F003016183BDE896
:10F9D000F08100002E2E2F4D6964646C6577617292
:10F9E00065732F54686972645F50617274792F4C2B
:10F9F0007749502F7372632F636F72652F74637032
:10FA00005F6F75742E6300007463705F73656E645E
:10FA10005F656D7074795F61636B3A20696E7661C2
:10FA20006C69642070636200417373657274696FFE
:10FA30006E2022257322206661696C6564206174E2
:10FA4000206C696E6520256420696E2025730A008C
:10FA500070B50546002D06D114A340F2EB3220A16B
:10FA600026A0F0F7BFFCEC6E0CB90AE00C4621684A
:10FA70000029FBD1E0688089F7F750FF10F0070FED
:10FA800005D02846BDE870400121FBF7D7BE012014
:10FA9000F7F744FF0146E068828911438181688B52
:10FAA00040F020006883002070BD00002E2E2F4DF6
:10FAB0006964646C6577617265732F5468697264F8
:10FAC0005F50617274792F4C7749502F7372632F96
:10FAD000636F72652F7463705F6F75742E630000BF
:10FAE0007463705F73656E645F66696E3A20696EF9
:10FAF00076616C6964207063620000004173736515
:10FB00007274696F6E2022257322206661696C65AC
:10FB100064206174206C696E6520256420696E2004
:10FB200025730A002DE9F041002400250026002756
:10FB3000A046FDF7B1F8044641F292322B49204627
:10FB4000FBF708FBFF212046FCF756FF0446284937
:10FB50002046FBF732FAFDF79FF8054641F29C324A
:10FB600022492846FBF7F6FAFF212846FCF744FF16
:10FB7000054620492846FBF720FAFDF78DF8064692
:10FB800041F2A63219493046FBF7E4FAFF2130462C
:10FB9000FCF732FF064618493046FBF70EFAFDF730
:10FBA0007BF8074641F2B03210493846FBF7D2FAEB
:10FBB000FF213846FCF720FF074610493846FBF77F
:10FBC000FCF9FDF769F8804641F2BA320749404630
:10FBD000FBF7C0FAFF214046FCF70EFF80460849BC
:10FBE0004046FBF7EAF9BDE8F0810000181D010866
:10FBF000C9AF0008E5100108291101086D110108BD
:10FC0000B11101082DE9F04F83B0DFF88083D8F8F7
:10FC10000C00401CC8F80C0098F80200401C88F842
:10FC20000200DFF86CB34FF0000A0026D8F8184045
:10FC3000002C00F09C81207D002806D1D5A340F245
:10FC4000BE42E0A1EAA0F0F7CDFB207D012806D15D
:10FC5000D0A340F2BF42F0A1E5A0F0F7C3FB207DA6
:10FC60000A2806D1CBA34FF49862F6A1E0A0F0F7E2
:10FC7000B9FBA17F98F80200814203D12646E468CF
:10FC800000F072B9A0770025A946207D022806D190
:10FC900094F84200062802D3012500F09DB894F89C
:10FCA00042000C2802D3012500F096B894F8990080
:10FCB000002845D0206F30B1B6A340F2D442EDA168
:10FCC000CBA0F0F78FFBE06E30B9B2A340F2D54283
:10FCD000F5A1C7A0F0F786FB94F89A000C2801D391
:10FCE000012579E094F8990010F80B0094F8981029
:10FCF000814202D2491C84F8981094F898108142ED
:10FD00006AD30127B4F8601021B1204600F098FAB8
:10FD100030B10AE0204601F03FF930B1002704E09D
:10FD20002046FDF7C7F800B90027E7B384F898A08C
:10FD300094F8990007284FD2401C84F899004BE0B2
:10FD4000B4F9300047F6FF77B84201D2401C208654
:10FD5000B4F93000B4F9401088423DDB2046FFF78B
:10FD600069FC18B1206FF0B9E06EE0B1207D022887
:10FD700014D094F842000C2800D30C20B4F93E10A3
:10FD8000B4F93C2001EBE202D549085C02FA00F02C
:10FD9000B84201DB47F6FF70A4F84000A4F830A099
:10FDA000B4F8480000E017E0B4F86010884200D3CF
:10FDB00008464108A4F84A10608E4FF6FF7202EA26
:10FDC0004002914201D2A4F84A20A4F84800A4F8C5
:10FDD0006AA02046FFF7D6FB207D06280BD1A17E26
:10FDE00011F0100F07D0216AD8F80C20511A2829D9
:10FDF00001D9691CCDB2617A11F0080F2CD004280A
:10FE000001D0072828D1B748D4F894104FF4FA73DA
:10FE10000844B0FBF3F2206AD8F80CC0ACEB000049
:10FE2000824204D2681CC5B24FF0010914E094F874
:10FE30009B2042F29F4C12FB0CF201EBC201B1FB82
:10FE4000F3F1814208D22046FCF798FB20B994F8E0
:10FE50009B00401C84F89B00606F68B1206AD8F852
:10FE60000C10091AB4F9400000EB4000B1EB400F50
:10FE700002D32046FBF782FF207D032807D1216AA9
:10FE8000D8F80C20511A282901D9691CCDB20928AB
:10FE900007D1206AD8F80C10081AF02801D9681C7C
:10FEA000C5B2002D42D0D4F890502046FDF7E0FDB9
:10FEB0006EB1D8F81800844206D136A340F26D52D4
:10FEC00089A14BA0F0F78EFAE068F0600DE0D8F859
:10FED0001800A04206D02FA340F271528DA144A079
:10FEE000F0F780FAE068C8F81800B9F1000F0BD0FD
:10FEF000208BE18A221D0290009201912346204628
:10FF0000626A216DFFF72AFC27692046E468FBF747
:10FF1000FDFD88F800A01DB16FF00C013846A84720
:10FF200098F8000000287FF480AE1DE02646E468C3
:10FF3000307F401CC0B23077717F884214D386F87E
:10FF40001CA088F800A0D6F88C201AB13146306980
:10FF5000904700E0002098F8001000297FF465AE7B
:10FF600010B93046FCF7A6FF002C7FF464AE0025E4
:10FF7000D8F81C40002C06D0207D0A2804D005A308
:10FF800040F2A152DCE017E1DFE00000DC000020DD
:10FF9000AB1C01082E2E2F4D6964646C657761726D
:10FFA00065732F54686972645F50617274792F4C65
:10FFB0007749502F7372632F636F72652F7463706C
:10FFC0002E6300007463705F736C6F77746D723AA8
:10FFD00020616374697665207063622D3E7374617D
:10FFE000746520213D20434C4F5345440A000000D6
:10FFF000417373657274696F6E20222573222066C7
:020000040801F1
:1000000061696C6564206174206C696E652025648B
:1000100020696E2025730A007463705F736C6F77BC
:10002000746D723A20616374697665207063622D25
:100030003E737461746520213D204C495354454EF4
:100040000A0000007463705F736C6F77746D723AAE
:1000500020616374697665207063622D3E737461FC
:10006000746520213D2054494D452D574149540A7E
:10007000000000007463705F736C6F7774696D7259
:100080003A2070657273697374207469636B696E6A
:1000900067207769746820696E2D666C696768747B
:1000A00020646174610000007463705F736C6F772B
:1000B00074696D723A207065727369737420746923
:1000C000636B696E67207769746820656D707479F9
:1000D0002073656E642062756666657200000000BC
:1000E000E01C0108B84C0A007463705F736C6F7792
:1000F000746D723A206D6964646C6520746370205D
:10010000213D207463705F6163746976655F70631D
:10011000627300007463705F736C6F77746D723A12
:1001200020666972737420706362203D3D207463A1
:10013000705F6163746976655F706362730000006D
:100140001FA1AFF25410F0F74DF90020216AD8F842
:100150000C20511AF02900D9012040B32046FDF7A8
:1001600087FC7DB1D8F81C00844208D1AFF2DC13C3
:1001700040F2AF521EA1AFF28810F0F733F9E068F9
:10018000E8600FE0D8F81C00A04208D0AFF2FC13E2
:1001900040F2B35220A1AFF2A810F0F723F9E068C3
:1001A000C8F81C002046E468FBF7B0FC01E02546D7
:1001B000E468002C7FF4E0AE03B0BDE8F08F0000EF
:1001C0007463705F736C6F77746D723A2054494D2D
:1001D000452D57414954207063622D3E73746174FC
:1001E00065203D3D2054494D452D5741495400005F
:1001F0007463705F736C6F77746D723A206D6964AD
:10020000646C652074637020213D207463705F749A
:10021000775F7063627300007463705F736C6F77F5
:10022000746D723A20666972737420706362203D47
:100230003D207463705F74775F70636273000000C9
:100240002DE9F84F05460F46002D06D15EA340F27A
:100250004B326AA172A0F0F7C5F8EC6E34B14FB121
:100260002089B84211D80020BDE8F88F4FF0FF3048
:10027000BDE8F88F54A340F2533273A168A0F0F7A1
:10028000B1F86FF00500BDE8F88F688EB84206D26D
:100290004DA340F25B3275A161A0F0F7A3F820896D
:1002A00030B949A34FF4577274A15DA0F0F79AF8E2
:1002B00094F80AB01BF0010F01D0042600E00026DC
:1002C0002089C01B1FFA80F808EB060081B24FF4AA
:1002D00020723620F8F73AFF82465FEA0A0068D0BB
:1002E000606822890189891A39448BB2DAF80410CE
:1002F00042463144F9F7C6FA40455AD1E068808950
:10030000F7F70CFB00F03F064FF0000916F0080F5E
:1003100003D026F008064FF0080916F0010F03D0AD
:1003200026F0010649F00109E0684068F7F7EAFAAB
:10033000C3194A4651462846CDF800B0FBF758F994
:100340000746380035D06068F9F748F9B5F8661007
:10035000081AA5F8660060680189A1EB080189B256
:10036000F9F71AFC2089A0EB080020813046F7F746
:10037000D5FA0146E0688289114381816068F9F706
:100380002DF9B5F866100844A5F866007868F9F705
:1003900025F9B5F866100844A5F8660020683860AD
:1003A0002760386810B90020A5F868000020BDE873
:1003B000F88FBAF1000F02D05046F9F7F7FA4FF074
:1003C000FF30BDE8F88F00002E2E2F4D6964646C5D
:1003D0006577617265732F54686972645F506172EA
:1003E00074792F4C7749502F7372632F636F726546
:1003F0002F7463705F6F75742E6300007463705F99
:1004000073706C69745F756E73656E745F73656726
:100410003A20696E76616C69642070636200000046
:10042000417373657274696F6E2022257322206692
:1004300061696C6564206174206C696E6520256457
:1004400020696E2025730A0043616E277420737043
:100450006C6974207365676D656E7420696E746F66
:10046000206C656E677468203000000073706C69E2
:1004700074203C3D206D7373000000007573656748
:100480002D3E6C656E203E203000000008488168DB
:1004900000290CD10749084A09681268114306D09F
:1004A0000121816000220549FA20FAF7B5BB7047A7
:1004B00020010020F4000020F8000020F5110108C0
:1004C00030B583B004461F4D287810F0040F23D1B7
:1004D000002C06D11CA340F2EE2228A12FA0EFF79A
:1004E00081FF287810F0020F18D0616A6869421AFB
:1004F0001AD4228D1144411A002915DCE968314BC8
:100500000A88498800930292019169891B1D42184B
:100510002046A969FFF722F903B030BD10F0010FA2
:1005200002D029480068206268890028F4D0608BD6
:1005300040F00200608303B02046BDE83040FCF785
:10054000B9BC0000FC0000202E2E2F4D6964646CA5
:100550006577617265732F54686972645F50617268
:1005600074792F4C7749502F7372632F636F7265C4
:100570002F7463705F696E2E630000007463705F98
:1005800074696D65776169745F696E7075743A201E
:10059000696E76616C696420706362004173736593
:1005A0007274696F6E2022257322206661696C6502
:1005B00064206174206C696E6520256420696E205A
:1005C00025730A00DC600020E800002010B5FBF76E
:1005D00063FA06494878401C487010F0010F03D0B8
:1005E000BDE81040FFF70EBB10BD0000DC0000208E
:1005F0000248417841F0100141707047FC00002032
:1006000070B50446002C06D116A340F2A63221A1F3
:1006100029A0EFF7E7FEB4F828C0626A02EB0C01EC
:10062000638EE06AB3F5866F01D94FF486630344A5
:10063000CB1A03D4A4F82AC0081A70BD111A0029D5
:1006400002DD002060850BE0851AB5F5803F06D3FA
:1006500004A340F2B63222A117A0EFF7C3FE6585CE
:10066000002070BD2E2E2F4D6964646C6577617219
:1006700065732F54686972645F50617274792F4C8E
:100680007749502F7372632F636F72652F74637095
:100690002E6300007463705F7570646174655F72CF
:1006A00063765F616E6E5F776E643A20696E766125
:1006B0006C69642070636200417373657274696F62
:1006C0006E2022257322206661696C656420617446
:1006D000206C696E6520256420696E2025730A00F0
:1006E0006E65775F7263765F616E6E5F776E6420B2
:1006F0003C3D203078666666660000002DE9FF4FBD
:100700008FB00546174600200D90002480460C90BF
:10071000834600260A90099082460890002D07D053
:10072000688EB5F86210B0EB510F0DD201460CE0A7
:10073000DBA34FF4CF72E7A1ECA0EFF753FE6FF00D
:100740000F0013B0BDE8F08F490801B901460791C9
:10075000109870B13946284600F05AFB0028F0D1B5
:10076000B5F866900B90E86E002800F0CA80044649
:100770000CE0CBA340F2AD12E6A1DCA0EFF732FE15
:1007800013B06FF00F00BDE8F08F0446206800281A
:10079000FBD1A07A10F0010F01D0042000E000206E
:1007A00005902189059801440798814206D9BCA388
:1007B0004FF4F372E4A1CDA0EFF714FE2189059860
:1007C00001440798401A80B20690B5F86800099075
:1007D000002827D00699884206D9B1A34FF4FC72AD
:1007E000DFA1C2A0EFF7FEFDA046BDF82400B8428D
:1007F00001D2014600E03946069A914202D9DDF85D
:1008000018A004E0B84201D2824600E0BA4606EBE6
:100810000A018EB2A0EB0A0009900698A0EB0A002C
:1008200080B20690BDF8240040B1BE4206D09CA321
:100830004FF40072D2A1ADA0EFF7D4FDBE426AD250
:100840000698002867D02089002864D00699B81B34
:10085000884200DD069880B20490A046129810F0FD
:10086000010F1CD0129801210190029109AB009553
:100870000020069A0499FDF74FF80D90002800F02B
:100880005B821098049A81190D984068EFF79AFEE0
:100890000D98F8F7A3FE48441FFA80F92DE0606830
:1008A00000E0084601680029FBD1017B11F0C00F70
:1008B00010D1416840890144109881420AD136B173
:1008C00077A340F23122B6A188A0EFF78BFD049800
:1008D000089012E0012200200499F8F737FC0D90EF
:1008E000002800F02982109881190D9841600D9818
:1008F000F8F774FE48441FFA80F90498304486B231
:1009000009E0B5F8680030B165A340F24A22AFA112
:1009100076A0EFF767FDBE4280F09B8007990B98A9
:10092000081A0E90B81B80B20E9989B2884200D383
:1009300008460690129810F0010F2CD0BBF1000F62
:1009400027D000201299019102900B9906980095EA
:10095000084481B209AB3620079AFCF7DDFF5FEA55
:10096000000800F0E981B8F80A100698814206D222
:100970004BA340F26622A1A15CA0EFF733FD1098D3
:10098000D8F8042081190B981044069AEFF71AFE44
:1009900025E00120D6E7BDF8240030B140A340F2A5
:1009A0007122A6A151A0EFF71DFD01223620069964
:1009B000F8F7CCFB0590002800F0BE811098811953
:1009C000059841604FF4207236200B99F8F7BEFB72
:1009D0005FEA000811D040460599F8F763FD4046EC
:1009E000F8F7FCFD48441FFA80F9B9F1090F09D95D
:1009F0004046F8F7DBFF00F09FB90598F8F7D6FFFF
:100A000000F09AB90A980090E86D002283194146D7
:100A10002846FAF7EDFD5FEA000800F08D81BBF192
:100A2000000F02D00C9810B108E0C34609E01CA3E7
:100A300040F2AB2285A12DA0EFF7D4FC0C98C0F8B2
:100A40000080CDF830800698304486B2BE42FFF474
:100A500069AFBAF1000F16D066688EB13089504484
:100A60003081306848B971897068524608441099DD
:100A7000EFF7A8FD7089504470813668002EEDD1E3
:100A8000208950442081BDF82400A5F868000D9805
:100A900020B124B902A34FF43872E1E0EFE0E4E0C2
:100AA0002E2E2F4D6964646C6577617265732F54C7
:100AB000686972645F50617274792F4C7749502F66
:100AC0007372632F636F72652F7463705F6F7574D9
:100AD0002E6300007463705F77726974653A2069F1
:100AE0006E76616C696420706362000041737365A7
:100AF0007274696F6E2022257322206661696C65AD
:100B000064206174206C696E6520256420696E2004
:100B100025730A007463705F77726974653A2061A7
:100B20007267203D3D204E554C4C202870726F67F7
:100B300072616D6D65722076696F6C61746573208A
:100B400041504929000000006D73735F6C6F636151
:100B50006C20697320746F6F20736D616C6C000082
:100B6000696E636F6E73697374656E74206F7665FA
:100B70007273697A652076732E20737061636500E5
:100B8000696E636F6E73697374656E74206F7665DA
:100B90007273697A652076732E206C656E00000092
:100BA0007463705F77726974653A20524F4D20709C
:100BB000627566732063616E6E6F74206265206F6C
:100BC00076657273697A656400000000756E7365FE
:100BD0006E745F6F76657273697A65206D69736D87
:100BE0006174636820287063622D3E756E73656E54
:100BF00074206973204E554C4C2900007463705F5B
:100C000077726974653A20636865636B2074686104
:100C10007420666972737420706275662063616EF9
:100C200020686F6C642074686520636F6D706C65FC
:100C30007465207365676C656E0000006F76657281
:100C400073697A65203D3D20300000007072657642
:100C50005F73656720213D204E554C4C000000001D
:100C600047A1AFF27810EFF7BDFB60680D99F8F778
:100C700019FC0D98218900890844208124E00898F6
:100C800010B30CB1606840B9AFF2EC1340F2E62249
:100C900049A1AFF2A810EFF7A5FB6068016839B170
:100CA0000289089911440181006801680029F7D17F
:100CB00002890899114401814289089911444181AE
:100CC00021890898084420818CB1C4F800B0E86DEF
:100CD0003844E865B5F86400C01BA5F86400A5F8C1
:100CE0006690B9F1000F10D0286F18B10DE0C5F86B
:100CF0006CB0ECE7E86E40B9AFF25C2340F2123220
:100D00003BA1AFF21820EFF76DFBB8F1000F0FD049
:100D1000D8F80C0060B1129810F0020F08D108202A
:100D2000F6F7FCFD0146D8F80C0082891143818159
:100D300013B00020BDE8F08F688B40F0800068831E
:100D40000D9810B10D98F8F731FEBBF1000F02D0ED
:100D50005846FEF7F8FDB5F8660060B1286F50B947
:100D6000E86E40B9AFF2C82340F2273220A1AFF2BB
:100D70008420EFF737FB13B04FF0FF30BDE8F08F62
:100D80007463705F77726974653A2063616E6E6F29
:100D90007420636F6E636174656E6174652077683B
:100DA000656E207063622D3E756E73656E7420698A
:100DB0007320656D707479007463705F7772697405
:100DC000653A20657874656E73696F6E206F662072
:100DD0007265666572656E636520726571756972AC
:100DE0006573207265666572656E6365000000005C
:100DF0007463705F77726974653A2076616C6964B8
:100E0000207175657565206C656E677468000000FB
:100E100070B504460D46002C06D124A340F23312CF
:100E20002FA137A0EFF7DEFA207D042808D007288D
:100E300006D0022804D0032802D06FF00A0070BD4B
:100E400055B1B4F86400A84208D2608B40F080002D
:100E500060834FF0FF3070BD002070BDB4F86600B5
:100E6000092806D3608B40F0800060834FF0FF308C
:100E700070BD00280DD0206F002815D1E06E00282D
:100E800012D10AA340F2551227A11DA0EFF7AAFA2A
:100E90000AE0206F08B9E06E30B104A34FF4AC72E1
:100EA00030A117A0EFF79EFA002070BD2E2E2F4D17
:100EB0006964646C6577617265732F5468697264E4
:100EC0005F50617274792F4C7749502F7372632F82
:100ED000636F72652F7463705F6F75742E630000AB
:100EE0007463705F77726974655F636865636B7361
:100EF0003A20696E76616C6964207063620000005C
:100F0000417373657274696F6E20222573222066A7
:100F100061696C6564206174206C696E652025646C
:100F200020696E2025730A007463705F777269749C
:100F3000653A207062756673206F6E2071756575F5
:100F400065203D3E206174206C65617374206F6E76
:100F500065207175657565206E6F6E2D656D707499
:100F6000790000007463705F77726974653A206E6F
:100F70006F207062756673206F6E20717565756580
:100F8000203D3E20626F7468207175657565732021
:100F9000656D7074790000002DE9F04705464FF04B
:100FA0000009002D06D12FA340F64F023AA143A01D
:100FB000EFF718FAEC6E44B395F89A00FF2802D2C6
:100FC000401C85F89A00E0688089F6F7A7FC10F0CD
:100FD000010F01D02089D8B10027DFB10022E068DD
:100FE000494643682846FCF7EBF880465FEA08006C
:100FF00012D0D8F804609FB11120F6F78FFCB189A8
:1010000021F47C510843B08114E00020BDE8F08752
:101010000127E2E70122E2E74FF0FF30BDE8F08769
:1010200006F11401606823890289D21A93B2012261
:10103000F8F728FCE0684068F6F764FC401C296D6E
:10104000091A00D528654B46002241462846FCF780
:1010500025FA2B1D2A4641462846BDE8F047FCF7F5
:10106000A9B900002E2E2F4D6964646C65776172FA
:1010700065732F54686972645F50617274792F4C84
:101080007749502F7372632F636F72652F7463708B
:101090005F6F75742E6300007463705F7A65726FA2
:1010A0005F77696E646F775F70726F62653A20690F
:1010B0006E76616C696420706362000041737365D1
:1010C0007274696F6E2022257322206661696C65D7
:1010D00064206174206C696E6520256420696E202F
:1010E00025730A0070B505460C4616460C48006884
:1010F000C08A41F29C31884209D109480068008BBE
:10110000218B884203D006480068F9F753FF044852
:10111000046004492046FDF757FE002070BD000022
:101120003C0100206DEE000870B505460C461646E1
:101130000C480068C08A41F2A631884209D10948AA
:101140000068008B218B884203D006480068F9F7BD
:1011500031FF0448046004492046FDF735FE0020B5
:1011600070BD000040010020E1EE000870B50546AA
:101170000C4616460C480068C08A41F2B0318842DD
:1011800009D109480068008B218B884203D00648AA
:101190000068F9F70FFF0448046004492046FDF792
:1011A00013FE002070BD00004401002055EF000830
:1011B00070B505460C4616460C480068C08A41F2D8
:1011C000BA31884209D109480068008B218B8842D6
:1011D00003D006480068F9F7EDFE044804600449AE
:1011E0002046FDF7F1FD002070BD00004801002001
:1011F000CDEF000810B5FFF7E9F908480849006885
:101200000968084306D00022BDE810400549FA20CD
:10121000F9F702BD04490020886010BDF4000020E9
:10122000F8000020F51101082001002070B50446E7
:101230000D461646324629462046F2F7A7FC70BDF9
:1012400070B5044600252BE000224FF400711948C8
:10125000F0F7B4FE0120F9F737FC04F0800028B164
:10126000012211461448F0F7A9FE04E000220121F2
:101270001148F0F7A3FE6006040E0120F9F724FCE4
:10128000012251020B48F0F799FE0220F9F71CFCED
:101290004FF480710748F0F77FFE0443681CC5B225
:1012A000082DD1DB00224FF400710248F0F786FED2
:1012B000204670BD00040240001002402DE9F04FAE
:1012C000ADF2144D044600250020CDF804046078EA
:1012D000217840EA012AE078A17840EA01262079C5
:1012E000CDF80C04012E78DB502E76DCDDF80C04F2
:1012F000C000B042F7DBBAF15F0F6FDC0AEB06000B
:1013000060287FDC0027A94636E009F10500205C53
:10131000CDF808044FF0000B21E0012000FA0BF09B
:10132000DDF80814084020B14FF47F40CDF81004D8
:1013300002E00020CDF810040AEB070188B2DDF8C6
:101340001014F3F797FE781C87B2B74203DB012035
:10135000CDF8040406E00BF1010000F0FF0BBBF137
:10136000080FDADB00BFDDF80404012800D107E034
:1013700009F1010000F0FF09DDF80C048145C4DB30
:1013800000BF274802782846691CCDB20DF800201E
:101390000F222846691CCDB20DF800200DEB050088
:1013A00021680160281DC5B229466846F3F728F870
:1013B000804608F0FF022846691CCDB20DF80020D7
:1013C0004FEA28222846691CCDB20DF800201548A6
:1013D000008AA84203DB284603E017E012E0114828
:1013E000008A104948824A8AC8686946EFF7EAF8D5
:1013F0000C48428AC1680C48FFF718FF0DF2144DE3
:10140000BDE8F08F0220CDF8000402E00320CDF803
:1014100000040F20DDF80014F7F768F800BFEDE7CF
:101420005C00002058060020C80200202DE9F04F83
:10143000ADF2144D0546894600240020CDF8040481
:101440006878297840EA012AE878A97840EA0126F4
:101450002879CDF80C04012E7EDB502E7CDCDDF8E3
:101460000C04C000B042F7DBBAF15F0F75DC0AEB89
:1014700006006028FADC0027A04636E008F10500E7
:10148000285CCDF808044FF0000B21E0012000FAA1
:101490000BF0DDF80814084020B14FF47F40CDF880
:1014A000100402E00020CDF810040AEB070188B216
:1014B000DDF81014F3F7DEFD781C87B2B74203DBCA
:1014C0000120CDF8040406E00BF1010000F0FF0B51
:1014D000BBF1080FDADB00BFDDF80404012800D1FE
:1014E00007E008F1010000F0FF08DDF80C0480457A
:1014F000C4DB00BF344802782046611CCCB20DF832
:101500000020314842782046611CCCB20DF8002002
:101510002D4882782046611CCCB20DF800202A4864
:10152000C2782046611CCCB20DF8002009F10200FF
:10153000C0F307222046611CCCB20DF8002009F14F
:101540000200C2B22046611CCCB20DF800201F4838
:1015500002782046611C01E02CE027E0CCB20DF8B7
:1015600000200F222046611CCCB20DF800200DEBAC
:10157000040029680160201DC4B2FF2C01DC204654
:1015800000E0FF2012490880084602886946114899
:10159000EFF718F801230E4802880E490E4800683C
:1015A000FFF7ACF80DF2144DBDE8F08F0220CDF836
:1015B000000402E00320CDF800040F20DDF8001441
:1015C000F6F7D4FF00BFEDE7600000205C000020CC
:1015D0005601002080A30020380100202DE9F04FA3
:1015E000ADF2044D044600261CB90DF2044DBDE8D1
:1015F000F08F6078217840EA0128E078A17840EA0D
:10160000012794F804A0012F63DB602F61DCBAEBA3
:10161000470F5ED1B8F15F0F58DC08EB0700602878
:1016200054DC002514E0062000EB4500205C052179
:1016300001EB4501615C40EA0120CDF8000408EBB4
:10164000050188B2DDF80014F3F70CFD681C85B2C3
:10165000BD42E8DB234802783046711CCEB20DF85B
:10166000002010223046711CCEB20DF800200DEB88
:10167000060021680160301DC6B231466846F2F7A7
:10168000BFFE814609F0FF023046711CCEB20DF854
:1016900000204FEA29223046711CCEB20DF80020FE
:1016A0001148008AB04201DB304601E00E48008A52
:1016B0000D4948824A8AC8686946EEF783FF0A489E
:1016C000428AC1680948FFF7B1FD8EE74FF0020B6F
:1016D00001E04FF0030B0BF0FF011020F6F706FFBF
:1016E00000BF82E75C00002058060020C8020020EE
:1016F0002DE9F04FADF2044D0546894600241DB991
:101700000DF2044DBDE8F08F6878297840EA012891
:10171000E878A97840EA012795F804A0012F7FDB3B
:10172000602F7DDCBAEB470F7AD1B8F15F0F74DC24
:1017300008EB0700602870DC002614E0062000EBB0
:101740004600285C052101EB4601695C40EA012066
:10175000CDF8000408EB060188B2DDF80014F3F7B9
:1017600081FC701C86B2BE42E8DB3248027820461B
:10177000611CCCB20DF800202E4842782046611C36
:10178000CCB20DF800202B4882782046611CCCB2E8
:101790000DF800202748C2782046611CCCB20DF815
:1017A000002009F10200C0F307222146601CC4B2E8
:1017B0000DF8012009F10200C2B22046611CCCB232
:1017C0000DF800201C4802782046611CCCB20DF8B0
:1017D000002010222046611CCCB20DF800200DEB39
:1017E000040029680160201DC4B2FF2C01DC2046E2
:1017F00000E0FF2011490880084602886946104829
:10180000EEF7E0FE01230D4802880D490D480068FF
:10181000FEF774FF74E703E0FFE74FF0020B01E00F
:101820004FF0030B0BF0FF011020F6F79FFE00BFF7
:1018300066E70000600000205C00002056010020E8
:1018400080A30020380100202DE9F047ADF5806D20
:1018500005468A4600246878297840EA0129E87814
:10186000A97840EA012717B1B7F57F4F46D1B9F102
:101870005F0F40DC39464846F3F7FCFB234802780B
:101880002046611CCCB20DF8002005222046611CC8
:10189000CCB20DF800200DEB040029680160201D7A
:1018A000C4B221466846F2F7ABFD0646F2B22046C6
:1018B000611CCCB20DF8002032122046611CCCB263
:1018C0000DF800201248008AA04201DB204601E00A
:1018D0000F48008A0E4948824A8AC8686946EEF76E
:1018E00071FE0B48428AC1680A48FFF79FFC0DF55C
:1018F000806DBDE8F0874FF0020801E04FF003086B
:1019000041460520F6F7F2FD00BFF0E75C0000203D
:1019100058060020C80200202DE9F043ADF2044D26
:1019200005460E4600246878297840EA0129E878BF
:10193000A97840EA012717B1B7F57F4F60D1B9F117
:101940005F0F5ADC39464846F3F794FB304802787B
:101950002046611CCCB201A90A542D484278204689
:10196000611CCCB201A90A54294882782046611C26
:10197000CCB201A90A542648C2782046611CCCB2D8
:1019800001A90A54B01CC0F307222046611CCCB246
:1019900001A90A54B01CC2B22046611CCCB201A9F4
:1019A0000A541C4802782046611CCCB201A90A5492
:1019B00005222046611CCCB201A90A5401A820448A
:1019C00029680160201DC4B2FF2C01DC204600E024
:1019D000FF20114908800846028801A90F48EEF748
:1019E000F1FD01230C4802880C490D480068FEF700
:1019F00085FE0DF2044DBDE8F0834FF0020801E0D2
:101A00004FF0030841460520F6F7B0FD00BFF0E7B0
:101A1000600000205C0000205601002080A3002010
:101A2000380100202DE9F047ADF5806D05468A4666
:101A300000241DB90DF5806DBDE8F0876878297820
:101A400040EA0127E878A97840EA01285F2F3DDCC9
:101A500041463846F3F706FB204802782046611CD1
:101A6000CCB20DF8002006222046611CCCB20DF845
:101A700000200DEB040029680160201DC4B221463E
:101A80006846F2F7BDFC0646F2B22046611CCCB2B5
:101A90000DF8002032122046611CCCB20DF8002057
:101AA0000F48008AA04201DB204601E00C48008A72
:101AB0000B4948824A8AC8686946EEF783FD0848A0
:101AC000428AC1680748FFF7B1FBB3E74FF002094C
:101AD00049460620F6F70AFD00BFABE75C00002090
:101AE00058060020C80200202DE9F043ADF2044D55
:101AF00005460E4600241DB90DF2044DBDE8F083E5
:101B00006878297840EA0127E878A97840EA01282E
:101B10005F2F57DC41463846F3F7A4FA2D48027888
:101B20002046611CCCB201A90A542A4842782046BA
:101B3000611CCCB201A90A54264882782046611C57
:101B4000CCB201A90A542348C2782046611CCCB209
:101B500001A90A54B01CC0F307222046611CCCB274
:101B600001A90A54B01CC2B22046611CCCB201A922
:101B70000A54194802782046611CCCB201A90A54C3
:101B800006222046611CCCB201A90A5401A82044B7
:101B900029680160201DC4B2FF2C01DC204600E052
:101BA000FF200E4908800846028801A90C48EEF77C
:101BB00009FD01230948028809490A480068FEF71F
:101BC0009DFD99E74FF0020949460620F6F7CEFC45
:101BD00000BF91E7600000205C000020560100205B
:101BE00080A30020380100204FF04070E1EE100A81
:101BF00070470006101600061016000000000000D6
